:100000000C949A190C94BB190C949E390C94433A95
:100010000C94BB190C94BB190C94BB190C94BB1910
:100020000C94BB190C94BB190C94616A0C945F6A14
:100030000C94BB190C94BB190C94944C0C94B23BCB
:100040000C94BB190C94BB190C94BB190C94BB19E0
:100050000C948C3A0C94BB190C94BB190C94BB19DE
:100060000C94BB190C94BB190C94BB190C94BB19C0
:100070000C94BB190C94BB190C94BB190C94BB19B0
:100080000C94BB190C94BB190C94BB190C94BB19A0
:100090000C94BB190C94BB190C94BB190C94BB1990
:1000A0000C94BB190C94BB190C94BB190C94BB1980
:1000B0000C94BB190C94BB190C94BB190C94BB1970
:1000C0000C94BB190C94BB190C94BB190C94BB1960
:1000D0000C94BB190C947D4A0C94BB190C94BB195D
:1000E0000C94BB190C94BB190C94BB190C94783369
:1000F0000C94BB190C94BB190C94BB190C94BB1930
:100100000C94BB190C94BB190C94BB190C94BB191F
:100110000C94BB190C94BB190C94BB190C94BB190F
:100120000C94BB190C94BB190C94BB190C94BB19FF
:100130000C94BB190C94C43B0C94BB190C94BB19C4
:100140000C94BB190C94BB190C94BB190C947E7ABB
:100150000C94BB190C94BB190C94BB190C94BB19CF
:100160000C94BB190C94BB190C948F3B0C94BB19C9
:100170000C94BB190C94BB190C94BB190C94BB19AF
:100180000C94BB190C94BB190C94BB190C94BB199F
:100190000C94BB190C94BB190C94BB190C94BB198F
:1001A0000C94E93E0C94BB190C94BB190C94BB192C
:1001B0000C94636A0C94BB190C94BC730C94BB191B
:1001C0000C94BB190C94BB190C94BB190C94BB195F
:1001D0000C94BB190C94BB190C94BB190C94BB194F
:1001E0000C94BB190C94BB190C94BB190C94BB193F
:1001F0000C94BB190C94B7780C94E8780C94DB55EC
:100200000C9487340C9424590C94C75E0C945A585F
:100210000C944A5D0C94E5330C94645E0C94AC55DC
:100220000C9424790C94B65F0C94CE580C941B62F9
:100230000C9488590C94D75D0C94585D0C94455DD2
:100240000C941B5F0C9480790C9447620C94FD59BC
:100250000C94985D0C9403580C946D570C947E5A32
:100260000C945C340C9426610C944D590C944556B6
:100270000C94125E0C945E550C94875C0C94CE5AD0
:100280000C9452340C94465C0C9471340C94965E2D
:100290000C94EA600C94EA580C9479790C943D5AC9
:1002A0000C9487570C94BE340C94A4570C946B5F39
:1002B0000C94255E0C94EC550C94CB330C945A5C46
:1002C0000C9458340C94235F0C94C9330C947434FC
:1002D0000C945F5D0C94A05C0C94865B0C94BA5DEE
:1002E0000C9456790C941D620C9421790C94AF5A9D
:1002F0000C94C1580C94A85D0C94A7610C94E95E11
:100300000C94B75C0C94E15C0C94435F0C94D55452
:100310000C94EE5B0C9401620C9408620C94575F91
:100320000C94B5590C94D65B0C9420340C94285A38
:100330000C9431590C940B5F0C94E3590C94885D28
:100340000C945A5A0C9446580C9411620C941879D7
:100350000C94F65A0C946C5A0C94A25B0C94853451
:100360000C94045E0C94EC610C94445E0C9437582D
:100370000C944F340C94C4570C94DB5A0C94CB550A
:100380000C94325C0C94E85D0C9418620C94F75851
:100390000C94335F0C94135B0C947C570C94745E38
:1003A0000C9474580C94335E0C94E0570C943B5BA3
:1003B0000C94C65F0C9409590C94F1560C94893432
:1003C0000C9441340C94F65D0C94A65E0C94453468
:1003D0000C94F5600C9428580C944C5B0C94665D5E
:1003E0000C943D790C94765D0C94F45C0C94AB34D5
:1003F0000C946E5C0C94075D0C9455340C94BE5BAD
:100400000C94485A0C9467580C94B65E0C940B5C90
:100410000C94905A0C94CE5C0C942F570C94175A51
:100420000C942F620C94A0590C945C610C949F3432
:100430000C94F6570C94F75E0C9417580C94B05823
:100440000C94D85E0C9438620C94845E0C94545EC8
:100450000C94DB580C94C35D0C94205C0C94C9592B
:10046000506C617965727320204C6576656C202034
:100470005374617274004C6576656C3A2000F0F13B
:10048000EF0001100001100F11000E121F210007D4
:10049000FF0B060803060603050704050306000212
:1004A0000207FF080C1700000017D0000000000032
:1004B000017F7EC00000000016BBFF70000000003E
:1004C0002B5EF7DC00000000D6F7BFFF0000000144
:1004D000FFFFEFFF80000007BFBFFDFFE000000D42
:1004E000EEFDFFFFB8000013FFF7BFDFFC00000FB9
:1004F000F7FFFFFFFE00007FBFBFF7FBFF0000CA52
:10050000FDEF7FFFFF80003577FBFFFFFF8000CF0F
:10051000DFFFEFFFEDC003BB7EFFFFFFFFE000CD7D
:10052000DBEEFFFEFFE007B7A7FFFFFFFAD00A4BA5
:100530007FFBFFFFDFF01196CFBFFFFFFDF80E6FCF
:10054000BFFFFFFFFEF81497FFFEDFFFFFA82B2D74
:100550005FBBFFFEEDFC1CDFF7FFF76FFFDC2F2B0F
:10056000BFFFBDD7DFDE7ADF4FDDFF3EBDFE6F464A
:10057000BFFFFF4756FE56B97FF7AEBAFFDEDFC6B4
:100580009EFDF95773FFAA3967FF76AE8FFDDFC472
:100590009BFFED56F1FF672B6F7DFABDCFF7DDD4E2
:1005A0009FF7D5E6B37FAF252FFF7B5BC5FFF6DA5C
:1005B000DFBDF5AE3BFF7FA535F3EBD2DF7FDDFA84
:1005C000DEFEBEAC77FD7F6569556B57BEFFBFDAB7
:1005D000B6BEDEDD55FE6FE52D696BB2AB6E7DAA52
:1005E000DEB6166D56FE7FD5A94BEFB2A97E76EA30
:1005F00056B4F5ED56F43F75ABFB5B54C9BC2ECA3F
:1006000047BDBFFB16FC1FB5BFC7FEA6E9581DDEE0
:100610005DBD775D1AF81F6DAB6ADFBF65F00FFA3D
:10062000FED5AAB48BF007DFEBAADDDF75E007B7D4
:10063000BE7D6AB08BC003FEF3CA976F7BC001AF6B
:10064000EE356CB4878001FDBFCADB4B3B0000F781
:10065000F27524F4C600007DFD8ADB5B3C00003FA0
:10066000777535ACC800001FBAAACEF3300000077A
:10067000EF55312CE0000003FFEADED380000001DB
:10068000F7FFEDAD000000007EBFF2540000000057
:100690000FF6ADB00000000003FFD68000000000A0
:1006A000001FF80000000000C5078D07530725074D
:1006B000F706C006D607A70771073A070C07DA0640
:1006C0000D10FFFF04F7FFF9F7FC17FE17D017FE18
:1006D00017FC17F9F7F702FFFF050D1000000208DD
:1006E00000161C09F404142E1450142E14041409BA
:1006F000F4161C080000030D10FFFF07F7F3E7FADC
:1007000007F207FA07F3E7FFF7FFFF060D100000F7
:10071000050C1E1413E40A0412040A0413E41E1444
:10072000000C0000040D10FFFF07F7F8E7F447CEB8
:1007300047F447F8E7FFF7FFFF060D100000050C30
:10074000071408E434444E44344408E40714000C0D
:100750000000040D10FFFF02FE7FFC3FFC1FFC1792
:10076000EE17D1D7EE17FC17FC1FFC3FFE7FFFFFF3
:10077000020D1003C006600430041C3C146E1451BA
:10078000D46E143C14041C0430066003C00D10FF2A
:10079000FF04FE3FF83FE47FF07FE0E7F007F0075B
:1007A000F807FE07FFFF040D1000000201C006203D
:1007B00018202440105C20E41004100408040604EF
:1007C00001FC0000020D10FFFF09F7F967F807F9B7
:1007D00067FFF7FFFF080D100000070C069409647F
:1007E000080409640694000C0000060000A80EC569
:1007F0000B8A09F50760400000C101F00000020308
:10080000F0000002031E000002061C00000201832B
:1008100080000C06000003C0C002001802000003A4
:10082000606002003003000003303002006181008C
:10083000000240181000C301000002E00C180186FD
:1008400021000002B00408030C6100000298040CAF
:100850000618C30000028C0C040C318600000286CE
:10086000180418630C000002C3300C30C6180000D6
:100870000241E008208C3000000260000C2018606B
:10088000000002200006303002C0000002300003E9
:100890001801800000021800319C030000030C00C6
:1008A00048B606000003070044630C00000301CEB5
:1008B0002227980000047B111CF000000401888CA2
:1008C000000006C4460000066223000006311180C5
:1008D0000000053888C00000056C4460000005C6B3
:1008E0002230000004018F11180000040319888CC5
:1008F0000000040630C4460000040C6062230000BF
:100900000418C031118000000331801888C0000035
:100910000363000C4460000003C60006243000009E
:1009200002018C00031818020000020F1800018059
:100930000C0000021830000002C006000002306007
:10094000000002606300000260400000023091007D
:100950000002C040000002189100000260C00000C8
:10096000020C610000023180000002060300000258
:100970001B00000303060000020E000003018C00B0
:10098000000204000004F80000C1604000005F386D
:1009900000000778000007B800000601B800000456
:1009A0000F8007B80000041FD00FB80000043FEF0D
:1009B000FBB80000043FEFFBB80000043FEFFBB8BA
:1009C0000000043FEFFBB80000043FEFFBB800005D
:1009D00003103FEFFBB8000600281FD0FFB8000B44
:1009E00000680F8187B80004C2A8000E01B8000A91
:1009F0003D2FFFF100B8000A0528000100F800149F
:100A00000528000100B8006405280001009000A23C
:100A100005280001009000A205280001009E006446
:100A20000528000100F200140529FE0100D2000A89
:100A3000052902010312000A1D2F0101020C1200F8
:100A400004E2A9F1FFF012000B0068110008120087
:100A5000060029F10008120000031101000812002D
:100A60000003010102000812000003010102000856
:100A70001200000301010200081200000301F1004E
:100A800008120000041100081200000301F1FFF039
:100A9000120000030701000C12000003190280334A
:100AA0001200000323FEFFC4D200000201460280B0
:100AB0000432000002028E0280043E000002028E18
:100AC00002800424000002028E02800424000781B8
:100AD0004702800424000FC4A3E2800424001F7B8B
:100AE0005806FFE4241E3F7B5C0FFFF4241E5F7B4F
:100AF0005FFFFF02D8246CDF7B5FFFFF02DE247FF5
:100B0000DF7B5FFFFF02DF247FDF7B5FFFFF02DF12
:100B1000A46CDF7B5FFFFF02DFFC1E5F7B5FFFFFDC
:100B200002DF7F1E3F7B5FF007DF69001F7B5FC036
:100B300000FFC9000FC4D083FC1F89000780511C2F
:100B400000E6090000032120001109000003022033
:100B50007C010900000302400389090000030287A9
:100B6000004109000003020880210900000303C0BE
:100B70007C11090000030620231109000003050071
:100B800020D10900000304C0102109000003044023
:100B900010010900000302A40C0109000003015424
:100BA0000B86090000040818798900000406140067
:100BB000490000040104002900000588001F00000E
:100BC000057000006260400FFFFF06C008000006CD
:100BD000400800000640080000064008FFFF04FE31
:100BE0007C40088008080204124440088004103C3D
:100BF000F2544008800420200282544008800420DF
:100C0000200282547C0880081020F254440880108E
:100C10000820124444020880600420127C440881A9
:100C200080043CF2004408820008048200440884E6
:100C30000010048200440888002004F2007C088828
:100C400000200412004008880010041200400884AC
:100C5000000804F2004008820004040282004008F8
:100C600081800404028200400880600804F2004091
:100C700008801010020412004008800820041200AE
:100C800040088004203CF2004008800410208200CC
:100C90004008800408208200400880080420F200F8
:100CA00040088010042012004008806008201200D4
:100CB000400881801020F20040088200202002823B
:100CC0000040088400202002820040088800102094
:100CD000F200400888000820120040088800042024
:100CE000127C40088400043CF2444008820008045E
:100CF00082544008818010048244400880602004AF
:100D0000F254400880102004124440088008100467
:100D1000125440088004083CF24440088004040255
:100D20002082544008800404022082444008800845
:100D3000080220F25440088010100220124440089B
:100D40008060202002125440088180203CF2444000
:100D50000882001004825440088400080482444041
:100D6000088800040402F2544008880004040212B7
:100D7000444008FFFF04FE7C4008000006400800D5
:100D8000000640087C7C05004008444405004008FB
:100D900044440500400844440538400844440640A3
:100DA000087C7C055440080000054440080000050C
:100DB0003840080000064008000006400800000413
:100DC0007000400838000002E08838400844000104
:100DD0001104444008440001110454400844000137
:100DE000110444400838000002E088384008000040
:100DF0000470004008001C0000044008006300006C
:100E000004400800808002000002384008010040D1
:100E10000070444008010040E0885440080200216E
:100E20001104444008020021110438400802002146
:100E30001104007C08010040E088004408010040E3
:100E4000007000440800808002000002384408005E
:100E50006300000344440208001C000003544408DB
:100E6000000004704444020838000002E088387C26
:100E7000084400011104004008440001110400402E
:100E80000844000111040402400838000002E08810
:100E90006C40080000047004400800000640080090
:100EA0000006400FFFFF06C0604000000210000077
:100EB000022000000410078020000004100480209D
:100EC00000000410048020000004100780200000AF
:100ED00004100000022000000410000002200000A6
:100EE0000410000002200000041000000220000096
:100EF0000410000002200000041000000220000086
:100F00000410000002200000041000000220000075
:100F10000410000002200000041000000220000065
:100F20000410000002200000041000000220000055
:100F300004100000022000000301F00000023E0047
:100F40000003013000000232000003033000000201
:100F500033000003023800000271000003022C007D
:100F60000002D10000030627FFFF0291800000026B
:100F7000042E0001D08000000204380000027080BE
:100F80000000020400FFFC00800000020C03800748
:100F900000C0000002080E0301C040000002083833
:100FA000030070400000021860000002186000009A
:100FB0000210C600018C200000021186000186206C
:100FC000000002330000030330000002260000038B
:100FD00001900000026C0000022000D8000002C84E
:100FE00000000260004C0000029B000002E003646D
:100FF00000000293000002E00324000002B00000A1
:1010000002E000360001A0000002C0001200012032
:10101000000002C00012000160000180001A0003FD
:1010200040000180000B0002400001800009000226
:101030004000010000020900024000030000020914
:1010400000025800030000026900025800FFC000BF
:1010500069000240FF01F800090002400000027E22
:1010600000090002400000021F00090003400000C8
:101070000207C00B00016000000203E01A0001201B
:10108000000003E012000120000004160001B0007F
:101090000004340000029300000303240000029BBC
:1010A0000000030364000002C80000044C000002BA
:1010B0006C000004D800000226000003019000002C
:1010C0000233000003033000000211860001862075
:1010D00000000210C600018C200000021860000011
:1010E0000218600000020838030070400000020887
:1010F0000E0301C0400000020C03800700C0000086
:10110000020400FFFC0080000002043800000270AE
:1011100080000002042E0001D0800000020627FF9C
:10112000FF029180000002022C000002D1000003A7
:101130000238000002710000030330000002330097
:10114000000301300000023200000301F000000241
:101150003E00000410000002200000041000000205
:101160002000000410000002200000041000000213
:101170002000000410000002200000041000000203
:1011800020000004100000022000000410000002F3
:1011900020000004100000022000000410000002E3
:1011A00020000004100000022000000410000002D3
:1011B00020000004100000022000000410000002C3
:1011C00020000004100000022000000410000002B3
:1011D00020000004100000022000000410000002A3
:1011E000200000021008FF818102808193B63C6DCF
:1011F000C98101818102FF181008FF81810DFF184C
:1012000010087FFFCCCC03FF7F00FFFF026030306F
:101210000260FFFF021008FFFF02CCCC03FC780045
:10122000FFFF026030300260FFFF02A51381135BF5
:101230001335130A13E312BD1293126D12461206F0
:1012400008183C3C04180C180FC0003FF0007FF851
:10125000007FFC0EF87C3EF03CFEF03FFEF87FF88D
:101260007FFFE07FFF803FFE000FF000000C180FB3
:1012700083E03FEFF87FFFFC7FFFFEF87C3EF03815
:101280001EF0381EF87C3E7FFFFE7FFFFC3FEFF82C
:101290000F83E00C18F0000002F0000002F00000E4
:1012A00002F0001EF001FEF00FFEF07FFEF3FFE003
:1012B000FFFE00FFF000FF8000FC0000020C1800A1
:1012C0001FE000FFF803FFFC0FFFFC3FFC3EFFF8B0
:1012D0001EFE781EF87C3EE07FFC003FFC001FF8FD
:1012E0000007E00C1803F860FFF8F802FFF8FCFFB5
:1012F000F87CFE783EF0781EF0781EF07C3EF07FA1
:10130000FCF03FFCF01FF8F007E00C180003E000D1
:101310000FE0003FE000FFE003FCE00FF0E03FC023
:10132000E0FFFF02FEFFFF02FEFFFF02FEFFFF02E3
:10133000FE000002E00C180C00603E00F87E00FC8D
:101340007C007CF8003EF0381EF0381EF87C3E7FB2
:10135000FFFC7FFFFC3FEFF80F83E00C180C007ED2
:101360003E01FE7E03FE7C07FEF80F9EF01F1EF07E
:101370003E1EF87C1E7FF81E7FF01E3FE01E0F8091
:101380001E0C180000061C0000021C0000023C009D
:101390000002FFFF02FEFFFF02FEFFFF02FEFFFF53
:1013A00002FE0000090C180FFFE03FFFF87FFFFC72
:1013B0007FFFFCF8003EF0001EF0001EF8003E7FAC
:1013C000FFFC7FFFFC3FFFF80FFFE012150415E064
:1013D00014BD14951472144F1425140214DF130B4A
:1013E000187FC000BFC008DFA018E07038E0703878
:1013F000E07038E07038E07038DFAFD8BFDFE87FEA
:10140000DFF00B187FDFF0BFDFE8DFAFD8E0703828
:10141000E07038E07038E07038E07038DFAFD8BF87
:10142000DFE87FDFF00B1800000380000002C0003F
:101430000002E0000002E0000002E0000002E00024
:101440000002E0000002DF8FC0BFDFE07FDFF00BB3
:10145000187FDFF0BFDFE8DFAFD8E07038E070382A
:10146000E07038E07038E07038C02FD8801FE80096
:101470001FF00B187FC000BFC008DFA018E0703855
:10148000E07038E07038E07038E07038C02FD880F5
:101490001FE8001FF00B187FC0003FC0001FA00016
:1014A0000002700000027000000270000002700074
:1014B000000270001FAFC03FDFE07FDFF00B1800BD
:1014C0000003800008C02018E07038E07038E07039
:1014D00038E07038E07038DFAFD8BFDFE87FDFF08A
:1014E0000B18001FF0801FE8C02FD8E07038E070A4
:1014F00038E07038E07038E07038DFA018BFC008FE
:101500007FC000000B180000181F8FC03FDFE07F76
:10151000DFF00B187FDFF0BFDFE8DF8FD8E00038A7
:10152000E00038E00038E00038E00038DF8FD8BF56
:10153000DFE87FDFF00410701CF83EF83E701CEC12
:1015400019BB1908198218FE176C17DA167516E4FC
:1015500015531516303FFFFC0000033FFFFE00004F
:1015600003DFFFFE00000206EFFFFD0000020EF7A2
:10157000FFFB80001EFBFFF7C0003EFDFFEFE00019
:101580007EFE000FE000FEFE02000FE000FEFE0205
:10159000000FE000FEFE02000FE000FEFE02000F62
:1015A000E000FEFE02000FE000FEFE02000FE00081
:1015B000FEFE02000FE000FEFDFFEFE0007EFBFFFD
:1015C000F7DFFFBEF7FFFBBFFFDEEFFFFD7FFFEEA4
:1015D000DFFFFEFFFF02F63FFFFEFFFF02F83FFFC7
:1015E000FC7FFFF816303FFFFC7FFFF83FFFFEFF58
:1015F000FF02F8DFFFFEFFFF02F6EFFFFD7FFFEEC9
:10160000F7FFFBBFFFDEFBFFF7DFFFBEFDFFEFE0F5
:10161000007EFE000FE000FEFE02000FE000FEFE76
:1016200002000FE000FEFE02000FE000FEFE0200DE
:101630000FE000FEFE02000FE000FEFE02000FE0E1
:1016400000FEFE02000FE000FEFDFFEFE0007EFB6B
:10165000FFF7DFFFBEF7FFFBBFFFDEEFFFFD7FFF02
:10166000EEDFFFFEFFFF02F63FFFFEFFFF02F83F47
:10167000FFFC7FFFF8163000000CC0000005E00002
:101680000005F0000005F8000005FC000005FE0064
:101690000005FE000005FE000005FE000005FE003E
:1016A0000005FE000005FE000005FE000005FDFF30
:1016B000E0000003FBFFF01FFF80F7FFF83FFFC0D3
:1016C000EFFFFC7FFFE0DFFFFEFFFF02F03FFFFECA
:1016D000FFFF02F83FFFFC7FFFF816303FFFFC7F63
:1016E000FFF83FFFFEFFFF02F8DFFFFEFFFF02F6FD
:1016F000EFFFFD7FFFEEF7FFFBBFFFDEFBFFF7DF36
:10170000FFBEFDFFEFE0007EFE000FE000FEFE02E8
:10171000000FE000FEFE02000FE000FEFE02000FE0
:10172000E000FEFE02000FE000FEFE02000FE000FF
:10173000FEFE02000FE000FEFE02000FE000FEFCD5
:10174000000FE0007EF80007DFFFBEF00003BFFFE0
:10175000DEE000017FFFEEC0000002FFFF02F600A6
:101760000003FFFF02F80000037FFFF816303FFF81
:10177000FC0000033FFFFE000003DFFFFE0000024D
:1017800006EFFFFD0000020EF7FFFB80001EFBFFCF
:10179000F7C0003EFDFFEFE0007EFE000FE000FE20
:1017A000FE02000FE000FEFE02000FE000FEFE025F
:1017B000000FE000FEFE02000FE000FEFE02000F40
:1017C000E000FEFE02000FE000FEFE02000FE0005F
:1017D000FEFC000FE0007EF80007DFFFBEF0000314
:1017E000BFFFDEE000017FFFEEC0000002FFFF024E
:1017F000F6000003FFFF02F80000037FFFF8163039
:101800003FFFFC0000033FFFFE0000031FFFFE0040
:1018100000030FFFFD00000307FFFB800000020331
:10182000FFF7C000000201FFEFE00000040FE0003E
:1018300000040FE00000040FE00000040FE00000CF
:10184000040FE00000040FE00000040FE0000004BB
:101850000FE000000201FFEFE000000203FFF7DFEE
:10186000FF8007FFFBBFFFC00FFFFD7FFFE01FFFF3
:10187000FEFFFF02F03FFFFEFFFF02F83FFFFC7F8D
:10188000FFF8163000000CC000000406E000010064
:1018900000020EF0000380001EF80007C0003EFCAE
:1018A000000FE0007EFE000FE000FEFE02000FE0F1
:1018B00000FEFE02000FE000FEFE02000FE000FE50
:1018C000FE02000FE000FEFE02000FE000FEFE023E
:1018D000000FE000FEFE02000FE000FEFDFFEFE063
:1018E000007EFBFFF7DFFFBEF7FFFBBFFFDEEFFF72
:1018F000FD7FFFEEDFFFFEFFFF02F63FFFFEFFFF73
:1019000002F83FFFFC7FFFF816300000037FFFF86E
:10191000000003FFFF02F8C0000002FFFF02F6E034
:1019200000017FFFEEF00003BFFFDEF80007DFFFDE
:10193000BEFC000FE0007EFE000FE000FEFE020095
:101940000FE000FEFE02000FE000FEFE02000FE0CE
:1019500000FEFE02000FE000FEFE02000FE000FEAF
:10196000FE02000FE000FEFE02000FE000FEFDFFA1
:10197000EFE0007EFBFFF7C0003EF7FFFB80001E9C
:10198000EFFFFD0000020EDFFFFE000002063FFF3A
:10199000FE0000033FFFFC00000308181C000002CB
:1019A0001C0000023C000002FFFF02FEFFFF02FEDF
:1019B000FFFF02FEFFFF02FE000003163000005A88
:1019C00001FFE000000303FFF01FFF8007FFF83F67
:1019D000FFC00FFFFC7FFFE01FFFFEFFFF02F03F95
:1019E000FFFEFFFF02F83FFFFC7FFFF816303FFFCE
:1019F000FC7FFFF83FFFFEFFFF02F8DFFFFEFFFF67
:101A000002F6EFFFFC7FFFEEF7FFF83FFFDEFBFF84
:101A1000F01FFFBEFDFFE00000027EFE000004FE9E
:101A2000FE02000004FEFE02000004FEFE020000B2
:101A300004FEFE02000004FEFE02000004FEFE02A0
:101A4000000004FEFE02000004FEFDFFE0000002B4
:101A50007EFBFFF01FFFBEF7FFF83FFFDEEFFFFC4E
:101A60007FFFEEDFFFFEFFFF02F63FFFFEFFFF02FC
:101A7000F83FFFFC7FFFF800000000000000FA00C4
:101A80000000E000E00028FE28FE282454FE544810
:101A9000C4C81026466C92AA440A00A0C0000038B0
:101AA0004482000082443800001054385410101052
:101AB0007C10100506000000101010101006060023
:101AC000000004081020407C8A92A27C0042FE02A2
:101AD00000468A929262448292926C182848FE08CC
:101AE000E4A2A2A29C3C5292920C808E90A0C06C68
:101AF0009292926C6092929478006C6C0000003527
:101B000036000010284482002828282828824428EB
:101B1000100040808A90604C929E827C7E909090D3
:101B20007EFE9292926C7C82828244FE8282443853
:101B3000FE92929282FE909090807C8292925EFEC3
:101B4000101010FE0082FE8200040282FC80FE1053
:101B5000284482FE02020202FE403040FEFE2010B7
:101B600008FE7C8282827CFE909090607C828A84D7
:101B70007AFE90989462649292924C8080FE80806B
:101B8000FC020202FCF8040204F8FC021C02FCC67F
:101B9000281028C6C0201E20C0868A92A2C2FE82BB
:101BA00082000040201008048282FE000020408055
:101BB000402001010101018040200000042A2A2A5E
:101BC0001EFE1222221C1C222222041C222212FE91
:101BD0001C2A2A2A18107E904000182525253EFE32
:101BE0001020201E0000BE0000000121BE00FE08E3
:101BF0001422000082FE02003E2018201E3E10200B
:101C0000201E1C2222221C3F242424181824243F96
:101C1000003E10202010122A2A2A040020FE220052
:101C20003C0202043E38040204383C020C023C220E
:101C3000140814223805053E0022262A3222106C90
:101C40008200000000FE0000826C100000408080D6
:101C50004080FEFEFEFEFE043C7E3C0410925438A2
:101C6000101F7FFFE0C0C0E0FF7F1FF0FCFE0E06EC
:101C7000060EFEFCF0000818387FFFFF0000000091
:101C8000000000FEFEFE0000003070F0E0C0C1E386
:101C9000FF7F3E0E1E3E7EF6E6C68606063070F0DC
:101CA000E3C3E7FF7F3D00181C1E0E06068EFEFCF8
:101CB000F80001030F1E78FFFFFF0070F0F0B03056
:101CC00030FEFEFE300FFFFFFEC6C6C7C7C3C130E1
:101CD0003C3E0E06060EFEFCF81F7FFFE3C3C3E387
:101CE000F37130F0FCFE8E06068EFEFCF8C0C0C01C
:101CF000C1C7DFFEF8E0C000003EFEFEC0000000ED
:101D000000387CFFE7C3C3E7FF7C3878FCFECE8653
:101D100086CEFEFC783E7FFFE3C1C1E3FF7F1F1844
:101D20001C9E8E86868EFEFCF0043E0404043C0657
:101D300018200E020E0A1E0850781000000E0C0823
:101D40000E0618200A3E000C020C0E320E00000097
:101D5000003A003000303E143E147E28240812144D
:101D60002A160030001C2200221C001C1C1C081C0F
:101D7000080102000808080002000408101C221CC8
:101D8000123E02262A12222A1438083E3A2A243EFB
:101D90002A2E202E303E2A3E3A2A3E0014000214FB
:101DA00000081422141414221408202A101C323A99
:101DB0001E281E3E2A141C22223E221C3E2A223E9F
:101DC00028201C222C3E083E223E2204023C3E08D3
:101DD000363E02023E103E3E203E3E223E3E28104F
:101DE0001C221E3E2816122A24203E203E023E3C83
:101DF000023C3E043E360836380638262A32003E7B
:101E000022100804223E00102010010101201000C1
:101E1000161A0E3E120C0C12120C123E0C161A0858
:101E20001E280D151E3E100E002E00012E003E0C29
:101E300012003C021E181E1E100E0C120C1F120C5B
:101E40000C121F0E10100A1E14103E121E021E1C31
:101E5000021C1E061E120C1218051E161E1A08362B
:101E6000220036002236081030203E3E3E02021E7E
:101E700010101E020210101E02021E1010000000A0
:101E8000FE010001FF01FE01FD02FE000201000152
:101E900001010201030202FF000000FE010001FF38
:101EA00001FE01FD02FEFF00000002010001010130
:101EB0000201030202FF7EFF8189898F0600062F3F
:101EC00029293F1F00FFFF21213F1E001E3F212126
:101ED0003F1E0020FEFF2121003F3F103030001E3A
:101EE0003F21213F1E001F3F20203F1F00BFBF009A
:101EF0001E3F21212100193D2D2F26544F47474CCD
:101F00004500524553544F524520204C4F414420E8
:101F1000202020534156450020536C6F743A200016
:101F20005253543A004275696C64204461746520D0
:101F3000323000204275696C643A20004F464653A7
:101F4000455420204C4947485420202053504545B3
:101F50004400436C6F636B3A202000565265663A2A
:101F6000202020005643433A202020200056696E4E
:101F70003A202020200052657365743A2020004CDE
:101F80006F6769633A202000584D4547413A202049
:101F90007265760054696D6572463A200054696D29
:101FA0006572433A2000204275696C643A20008BC8
:101FB000959FA9B2BBC3CBD3DAE1E8EEF4FA0005F2
:101FC0000B1014191D2125292D3134373A3D40437A
:101FD00045484A4C4F51535557585A5C5D5F6061B4
:101FE000636465666768696A6B6C6D6E6F6F70714C
:101FF000717273737474757576767677777878788E
:102000007979797A7A7A7A7B7B7B7B7B7C7C7C7C26
:102010007C7C7D7D7D7D7D7D7D7E7E7E7E7E7E7EEB
:102020007E7E7E7E7E7F7F7F7F7F7F7F7F7F7F0044
:10203000000000000000000000000001010101019B
:102040000202020303030404040505060607070849
:1020500009090A0B0C0C0D0E0F1011121314151692
:102060001718191A1C1D1E202122242527282A2B67
:102070002D2F3032343537393B3C3E4042434547C3
:10208000494B4D4E5052545657595B5C5E606163EC
:10209000656668696B6C6E6F70717374757677784E
:1020A000797A7B7B7C7D7D7E7E7F7F7F7F7F7F00DB
:1020B000000000000000000101010202030304040B
:1020C0000506060708090A0A0B0C0D0E0F1011125F
:1020D00014151617181A1B1C1D1F2022232426272F
:1020E000292A2C2D2F3032333536383A3B3D3E40AD
:1020F0004143454648494B4C4E4F5153545657580F
:102100005A5B5D5E5F616264656667696A6B6C6D90
:102110006E6F70717273747576777878797A7A7B6E
:102120007B7C7C7D7D7E7E7E7F7F7F7F7F7F7F0946
:102130000909090A0A0A0A0A0B0B0B0C0C0D0D0EF1
:102140000E0F1010111213131415161718191A1B4D
:102150001C1D1E1F20212324252627292A2B2D2E36
:102160002F313234353638393B3C3E3F40424345CF
:102170004648494B4C4D4F505253555657595A5B50
:102180005D5E5F61626364666768696A6B6C6E6FEF
:10219000707172727374757677777879797A7B7BE0
:1021A0007C7C7D7D7E7E7E7E7F7F7F7F7F7F7F06C6
:1021B000067F7F7F7F7F7F7FFFFF7F0AFCFFFFFF20
:1021C000FFFF4002FFFF7FFF05FFFFFFFFBE000193
:1021D00001402060602060200080000080A0601826
:1021E000E020000001FF1080018000E0AB0000064D
:1021F000010108FF8000C129001C40010000000A05
:1022000000000064000000E803000010270000A0A8
:1022100086010040420F0080969800424D3E040027
:1022200000000000003E00000028000000800000C8
:102230000040000000010001000000000000040058
:10224000000000000000000000000000000000008E
:102250000000000000FFFFFF0053504920534E498B
:10226000464645520A424954343A2F53530A42498A
:1022700054353A4D4F53490A424954363A4D495321
:102280004F0A424954373A53434B00554152542068
:10229000534E49464645520A424954323A52582012
:1022A000424954333A54580049324320534E494628
:1022B0004645520A424954303A5344412042495417
:1022C000313A53434C0029681434091A040D82062C
:1022D00040032A021501FDEDDCCCBCACA8A403012F
:1022E000FDF5E5C56E17474F00444953434F4E4E29
:1022F000454354204348312C434832004E4F205828
:102300005400480DAC0DF20D380E7E0EC40E0A0FAF
:10231000500F960FDC0F221068104D6F6F6E20501B
:102320006861736500582000485A204D41580031BB
:102330002053544F5042495400322053544F50427E
:102340004954004E4F20504152495459004556457A
:102350004E20504152495459004F4444205041525C
:10236000495459004D4F56452D2020202020202033
:10237000204D4F56452B000B340C340F340E34FDDA
:102380003305340634011020304000E0C0A080C086
:10239000E0002040014080C0FF004080C0FF40209E
:1023A00000E0C0402000E0C0313230302020003258
:1023B000343030202000343830302020003936309E
:1023C0003020200031393230302000333834303082
:1023D0002000353736303020003131353230300092
:1023E0002020314D003530304B003235304B00313C
:1023F00032354B002036324B002033314B00203138
:10240000364B002020384B002020344B00312E3634
:102410004B0020383030002038303000203332304C
:1024200000203136300020203830002020333200A8
:102430002020313600202020380020332E3200208A
:10244000312E360020302E3800302E33320020203E
:102450003817002031361700203332170020363469
:102460001700313238170032353617003530301743
:102470000020311A1B0020321A1B0020351A1B00C5
:1024800031301A1B0032301A1B0035301A1B002065
:10249000302E310020302E320020302E350020200A
:1024A0002031002020203200202020350020203143
:1024B00030002020323000202035300035312E32DF
:1024C0000032352E360031322E3800362E343000B0
:1024D000332E323000312E363000302E3830003579
:1024E0002E313200322E353600312E323800302E69
:1024F000363400302E333200302E31360038301A68
:102500001B00130F0F0F03101312101311130102EE
:1025100003000F101111130B171411101906031CCF
:102520001D081F200E032213230C0D272814162329
:102530001914080808161613162B2B2B190C0D0648
:1025400006060606060F0C0D0E00101B12100011D9
:102550001500002210111311002B14001611001980
:10256000001D1E00202100000000090400000000E2
:10257000001604191408080816160F162B2B2B1911
:102580000C0D0606060606060000010203040506F9
:102590000708090A0A0B0C0D0E0F10112122231F28
:1025A00020121314151617151618191A1B1C1D1DA9
:1025B00025251E24204348204F4E20202000202087
:1025C000202020204741494E2D202020200020207F
:1025D000204741494E2B004C4F474943204F4E2046
:1025E00000202020202053454C454354202020002B
:1025F0002050524F544F434F4C00204E4F524D41AC
:102600004C202020002020202053494E474C4520BC
:102610002020002043495243554C415200204E4F48
:10262000524D414C202020002020202053494E476D
:102630004C4520202000202020204155544F2000D0
:102640002056435552534F522000202020484355D6
:102650005220434831202000202048435552204337
:102660004832002048414D4D494E4720202000204F
:1026700020202048414E4E202020002020424C4166
:10268000434B4D414E002020434831202020200064
:1026900020202020202020434832202020202000FD
:1026A00020204C4F474943200020475249442020D6
:1026B00020002020464C495020444953504C415959
:1026C00020002020494E56455254200020205644D8
:1026D00043202020202020002020205620502D5054
:1026E000202000204652455155454E435920002098
:1026F0002053494E452020202000202020205351E7
:10270000554152452020002020545249414E474C0B
:102710004500504F534954494F4E2020200020205F
:10272000414320434F55504C452000202020204D50
:102730004154482000504F534954494F4E202020C7
:1027400000202020494E56455254202000202020B1
:10275000544849434B30200020434831200020207A
:10276000202020202020202043483220002020202C
:1027700020202020204C4F474943005452494754C1
:10278000595045202000202020545249475352439D
:1027900020202000204D4F524554524947002053DD
:1027A000434F50452020202000202020204D45541C
:1027B0004552202020002020202020204646542062
:1027C0000020495120464654202020002020464623
:1027D000542057494E444F57202000202020204CA1
:1027E0004F472000435552534F5253200020202082
:1027F0002020444953504C415920200020202020C3
:1028000020202041574700574156452054595045F4
:102810002020002020205357454550202020002014
:102820004652455155454E4359002057494E444F55
:1028300057202020002020202045444745202020EC
:10284000200020202020534C4F50452000202041C4
:1028500055544F2020202020002020205452414356
:102860004B20202000205245464552454E4345000E
:102870002020414C4C2020202020002020202042DD
:1028800049545F302020202000202020204249543D
:102890005F3100204249545F322020202000202058
:1028A00020204249545F3320202020002020202077
:1028B0004249545F3400204249545F352020202093
:1028C00000202020204249545F3620202020002074
:1028D0002020204249545F3700204558542054524C
:1028E00049472000202020204249545F30202020EA
:1028F0002000202020204249545F310020504152C6
:10290000414C4C454C202000202020534552494149
:102910004C20200020202020202050554C4C00200E
:102920004932432020202020200020202020205534
:1029300041525420202020002020202020535049A4
:102940002000204E4F2050554C4C202000202020AD
:1029500050554C4C2055502020002050554C4C20B8
:10296000444F574E002050455253495354454E54FE
:1029700020200020204C494E4520202000202020EF
:10298000202053484F5720002043504F4C202020F8
:1029900020200020202020435048412020202000DB
:1029A00020494E5645525420535300204F50455213
:1029B00041544F522000202020494E564552542069
:1029C0002020002020415645524147452000414DDE
:1029D000504C49545544452000202044555459201A
:1029E0004359434C4520002020204F464653455430
:1029F0000020524F4C4C2020202020002020204539
:102A00004C415354494320200020205859204D4F19
:102A100044452000545249474D4F44452020002052
:102A200020504F53545452494720002020205452E4
:102A30004947484F4C440020455850202020202032
:102A40002000202020204E4F4953452020200020E8
:102A50002020435553544F4D2000205350454544AA
:102A60002020202000202020204D4F4445202020E1
:102A700020002020202052414E474520005357205F
:102A80004652455120202020002020535720414D00
:102A90005020202000202053572044555459200016
:102AA0002020444F574E2020202000202050494E07
:102AB00047504F4E47202020002020414343454CA3
:102AC000000000205355425452414354200020201E
:102AD0004D554C5449504C592020002044494646FD
:102AE000524E544C2000C800900120034006800C38
:102AF0000019D430190032007D00FA00F401E2041C
:102B0000C4098813D430190032007D00FA00F401A2
:102B1000E20400C2EB0B00E1F50580F0FA02407818
:102B20007D0120BCBE00105E5F0000D430000010AC
:102B30005E5F0008AF2F00D012130068890900689B
:102B400089090090D0030048E8010024F40000A89F
:102B5000610000D43000006A180000C4090000E2DF
:102B600004000071020000FA0000010002000400ED
:102B70000800140028005000C80090012003D0076E
:102B8000F900F301E703C3098713506C617965729B
:102B900020322057696E7300506C61796572203164
:102BA0002057696E7300506C6179657220323A006B
:102BB000506C6179657220313A00506F6E67004742
:102BC000616D65204F76657200536E616B6500081C
:102BD000010202040404040808080808080808019F
:102BE0000102010401020108010201040102017055
:102BF0006D00616D0020323A200020313A20004300
:102C000050552020200020486F75726C7920426555
:102C1000657020202020200020323420486F7572FB
:102C200020466F726D61742020002059656172200A
:102C300061742074686520656E642000204D6F6E9D
:102C400074682061667465722064617920002020B8
:102C5000204E6577204D6F6F6E2020202000576139
:102C600078696E67204372657363656E74002046F1
:102C700069727374205175617274657220005761B6
:102C800078696E6720476962626F75732000202043
:102C90002046756C6C204D6F6F6E202020005761B0
:102CA0006E696E6720476962626F75732000204C01
:102CB00061737420517561727465722020005761D0
:102CC0006E696E67204372657363656E7400205091
:102CD000726F66696C657300507265762E464D2082
:102CE000546F646179204E6578742E464D00506CA7
:102CF000617965723120506C61796572322053744C
:102D00006172740048756D616E2000506C61796568
:102D1000722000426C61636B3A202000576869742E
:102D2000653A2020005375204D6F2054752057655B
:102D3000205468204672205361002053756E6461F0
:102D400079202000204D6F6E64617920200020548E
:102D500075657364617920005765646E657364619D
:102D60007900546875727364617920002046726935
:102D70006461792020005361747572646179200068
:102D80004A414E00464542004D41520041505200DA
:102D90004D4159004A554E004A554C004155470097
:102DA000534550004F4354004E4F56004445430096
:102DB0004A616E7561727900000000466562727545
:102DC0006172790000004D617263680000000000CC
:102DD00000417072696C0000000000004D617900D4
:102DE000000000000000004A756E65000000000051
:102DF00000004A756C790000000000000041756712
:102E0000757374000000000053657074656D626531
:102E10007200004F63746F626572000000004E6FB5
:102E200076656D626572000000446563656D62657C
:102E30007200000054696D65202043616C656E640A
:102E400061722020417374726F0050726F66696CFA
:102E50006520496D6167652020205374617274009C
:102E6000536E616B65202020506F6E6720202020FC
:102E7000436865737300436F6E66696720446961D8
:102E8000676E6F73652041626F757400202020208B
:102E9000576174636820202000000000004F7363B6
:102EA000696C6C6F73636F70650000000000202D0B
:102EB0002047616D6573202D202000000000002058
:102EC0002053657474696E67732020000000000051
:102ED00046323A200046313A2000531C1D1E00564F
:102EE0001C1D1E00205600201A1B560053544F5024
:102EF000004B434E54004B485A001F563D002031B2
:102F0000161F543D00465720322E38300032300014
:102F10003139002032300020313900416C61726D4E
:102F200020003C2D2020202020204E657874202079
:102F3000202020202D3E004C617020002B482020B6
:102F400020202020202B4D202020202020202B530B
:102F50000020204C61702000202020202020200014
:102F60002020001F1C1F1E1F1E1F1F1E1F1E1F0EA6
:102F7000035800530063006F0070006500000018E4
:102F8000034700610062006F00740072006F006E02
:102F900000690063007300000004030904090220B3
:102FA0000001010080FA0904000002FF0000000790
:102FB00005810240000007050102400000120110D7
:102FC00001FF000040D016F906000101020001DAFD
:102FD00032CD32C832BF327A326B325E321D32E4C9
:102FE00031E32F144F0A00144F2800144F460014E9
:102FF0004F2800144F0A00144F2800144F460014A5
:103000004F280014460A00144628001446460014AF
:10301000462800143E0A00143E2800143E460014C0
:103020003B2800145E0A00145E2800145E4600145B
:103030005E2800145E0A00145E2800145E46001428
:103040005E280014690A00146928001469460014F7
:1030500069280014760A00147628001476460014B5
:10306000762800144F0A00144F2800144F4600140D
:103070004F280014460A001446280014464600143F
:10308000462800143E0A00143E2800143E46001450
:103090003E2800143B0A00143B2800143B46001451
:1030A0003B2800145E0A00145E2800145E460014DB
:1030B0005E2800145E0A00145E2800145E460014A8
:1030C0005E280014690A0014692800146946001477
:1030D00069280014760A0014762800147646001435
:1030E00076280014580A0014582800145846001472
:1030F000582800144F0A00144F2800144F4600149B
:103100004F280014460A00144628001446460014AE
:10311000462800143B0A00143B2800143B460014C8
:103120003B2800143B0A00143B2800143B460014C3
:103130003B2800143B0A00143B2800143B460014B3
:1031400034280014420A0014422800144246001495
:1031500042280014420A0014422800144246001477
:1031600042280014420A0014422800144246001467
:1031700042280014420A0014422800144246001457
:103180003B2800144F0A00144F2800144F46001427
:103190004F2800144F0A00144F2800144F46001403
:1031A0004F2800144F0A00144F2800144F460014F3
:1031B0004F280014690A0014692800146946001495
:1031C000692800143B0A00143B2800143B460014F5
:1031D0003B2800143E0A00143E2800143E4600140A
:1031E0003E280000149E190014761900144F19008F
:1031F00014761900144F190014761900149E190042
:1032000014761900144F1900147619001458190077
:10321000147619001469190014764B0000147619FD
:1032200000147619001476190014761900144F1939
:1032300000144F1900144F1900144F190014581995
:1032400000145819001458190014581900144F1973
:1032500000144F1900144F1900144F4B0000197639
:103260001969195E194F195E196900149E148D149D
:103270007E14761469145E144F0014761400149EA4
:10328000140014761400149E140014761400149E76
:10329000140014761400149E140014693C00149E4B
:1032A0003C0014693C00149E3C0014763C00144F12
:1032B000140014583C00145E3C0014768C0000325C
:1032C0003E14003258140000193E6100000A5E14DA
:1032D000000A4F14000A3E6400000A3E14000A3E31
:1032E00014000A3E640000089E107600143B0A0099
:1032F00014340A00282E00000D1A27333F4A545E6A
:10330000666D74787C7E7F7E7C78746D665E544AD0
:103310003F33271A0D00F3E6D9CDC1B6ACA29A937C
:103320008C888482818284888C939AA2ACB6C1CD29
:10333000D9E6F30011241FBECFEFCDBFDFE5DEBF1E
:1033400000E00CBF10E2A0E0B0E2EAE2FAEF00E039
:103350000BBF02C007900D92A032B107D9F724E548
:10336000A0E2B0E201C01D92A13DB207E1F70E94C8
:10337000BE3C0C94477C0C940000E091E321F0915A
:10338000E42192E1899FE019F1091124962F969585
:1033900096959695E90FF11D677080E801C08695B6
:1033A0006A95EAF786930895E091E021E395E0932A
:1033B000E021EA95F2E1EF9FE091E321F091E42131
:1033C000E019F10911240090DF21E00DF11D869331
:1033D0000895E091E321F091E42192E1899FE019C1
:1033E000F1091124A62FA695A695A695EA0FF11D21
:1033F000261B6770B0E801C0B6956A95EAF70B2EF8
:103400000692481B9EEE8FEF44231AF4419592E1F9
:1034100080E0A1E030E022231AF42195AFEF3FEFE6
:103420004217E8F0742F7695542F552309F4089528
:10343000720F741770F0741BAA2332F0B69548F41B
:10344000B0E8EF5FFF4F05C0BB0F18F4B1E0E150EB
:10345000F040E90FF81F0B2E06925A95E6CF722F17
:103460007695522F552309F40895740F721718F0AA
:10347000721BE90FF81FAA2332F0B69548F4B0E8A2
:10348000EF5FFF4F05C0BB0F18F4B1E0E150F04013
:103490000B2E06925A95E6CF8058860F1BF48FE7C5
:1034A00067FD80E880580895222730E8422F432B9B
:1034B000449F0816190610F009F001C0242F369514
:1034C000A9F7822F11240895E9E6FAE1E80FF11D2A
:1034D000099408C010C018C020C028C030C038C02F
:1034E00040C048C058990895D099FCCF5899089584
:1034F000D09BFCCFC7C058990895D199FCCF58995B
:103500000895D19BFCCFBEC058990895D299FCCFA5
:1035100058990895D29BFCCFB5C058990895D39976
:10352000FCCF58990895D39BFCCFACC0589908950F
:10353000D499FCCF58990895D49BFCCFA3C0589937
:103540000895D599FCCF58990895D59BFCCF9AC082
:1035500058990895D699FCCF58990895D69BFCCFD9
:1035600091C058990895D799FCCF58990895D79B41
:10357000FCCF88C0589908959299FCCF5899089526
:10358000929BFCCF7FC0E8ECFAE1E80FF11D0994B3
:1035900008C010C018C020C028C030C038C040C00B
:1035A00048C058990895D09BFCCF58990895D09958
:1035B000FCCF68C058990895D19BFCCF58990895C5
:1035C000D199FCCF5FC058990895D29BFCCF5899F0
:1035D0000895D299FCCF56C058990895D39BFCCF3B
:1035E00058990895D399FCCF4DC058990895D49B0C
:1035F000FCCF58990895D499FCCF44C058990895A8
:10360000D59BFCCF58990895D599FCCF3BC05899CC
:103610000895D69BFCCF58990895D699FCCF32C017
:1036200058990895D79BFCCF58990895D799FCCF06
:1036300029C058990895929BFCCF58990895929962
:10364000FCCF20C083580090240280151CF4589BA6
:10365000FACF08958A5F0090240280159CF0589B51
:10366000FACF08958D570090240280151CF0589BC6
:10367000FACF089586500090240280151CF4589BC0
:10368000FACF089589E0809340085D9A80B18B302D
:1036900058F484E100904C0800FEFCCF1092400AE0
:1036A0008093010258995D980895835800906402B0
:1036B00080151CF4589BFACF08958A5F009064022D
:1036C000801504F3589BFACF08958D57009064023B
:1036D00080151CF0589BFACF089586500090640224
:1036E000801584F6589BFACF08957F9300902402AA
:1036F000709124020716072E24F0589BF9CF7F9172
:10370000089570912402071A8015072ED4F4589B4F
:10371000F8CF7F9108957F93009024027091240246
:103720007015072E24F0589BF9CF7F910895709162
:103730002402071A0816072E24F4589BF8CF7F910D
:1037400008957F919FCF7F930090640270916402EF
:103750000716072E24F0589BF9CF7F91089570919A
:103760006402071A8015072E64F7589BF8CF7F91E3
:1037700008957F9300906402709164027015072E83
:1037800024F0589BF9CF7F91089570916402071A35
:103790000816072EB4F6589BF8CF7F9108958058ED
:1037A00060580090240280156CF206165CF2589B5B
:1037B000F8CF08958058605800906402801514F284
:1037C000061604F2589BF8CF0895FF7F0000F57F9E
:1037D0002403D87F4806A67F6A09617F8C0C097F85
:1037E000AB0F9C7EC8121D7EE215897DF918E37C23
:1037F0000B1C297C1A1F5C7B23227C7A2825897963
:10380000262884781F2B6B77112E4176FB300475A8
:10381000DF33B573BA3654728C39E270563C5E6F42
:10382000173FC96DCE41236C7A446D6A1C47A66868
:10383000B449CF663F4CE864BF4EF1623351EB6050
:103840009B53D75EF555B35C4258825A825A425810
:10385000B35CF555D75E9B53EB603351F162BF4EBD
:10386000E8643F4CCF66B449A6681C476D6A7A4449
:10387000236CCE41C96D173F5E6F563CE2708C39A8
:103880005472BA36B573DF330475FB304176112EAE
:103890006B771F2B84782628897928257C7A232228
:1038A0005C7B1A1F297C0B1CE37CF918897DE215CF
:1038B0001D7EC8129C7EAB0F097F8C0C617F6A094C
:1038C000A67F4806D87F2403F57F0000FF7FDCFC3D
:1038D000F57FB8F9D87F96F6A67F74F3617F55F02F
:1038E000097F38ED9C7E1EEA1D7E07E7897DF5E3A2
:1038F000E37CE6E0297CDDDD5C7BD8DA7C7ADAD714
:103900008979E1D48478EFD16B7705CF417621CCEA
:10391000047546C9B57374C65472AAC3E270E9C08F
:103920005E6F32BEC96D86BB236CE4B86D6A4CB65F
:10393000A668C1B3CF6641B1E864CDAEF16265ACB3
:10394000EB600BAAD75EBEA7B35C7EA5825A4DA3DF
:10395000425829A1F555159F9B530F9D3351189B34
:10396000BF4E31993F4C5A97B44993951C47DD930C
:103970007A443792CE41A290173F1E8F563CAC8DB1
:103980008C394B8CBA36FC8ADF33BF89FB30958883
:10399000112E7C871F2B7786262884852825A484D2
:1039A0002322D7831A1F1D830B1C7782F918E3810A
:1039B000E2156481C812F780AB0F9F808C0C5A808F
:1039C0006A09288048060B802403008040C020A09C
:1039D00060E0109050D030B070F0088848C828A837
:1039E00068E8189858D838B878F8048444C424A4EF
:1039F00064E4149454D434B474F40C8C4CCC2CACD7
:103A00006CEC1C9C5CDC3CBC7CFC028242C222A2B2
:103A100062E2129252D232B272F20A8A4ACA2AAAD6
:103A20006AEA1A9A5ADA3ABA7AFA068646C626A68E
:103A300066E6169656D636B676F60E8E4ECE2EAE76
:103A40006EEE1E9E5EDE3EBE7EFE018141C121A164
:103A500061E1119151D131B171F1098949C929A9A6
:103A600069E9199959D939B979F9058545C525A55E
:103A700065E5159555D535B575F50D8D4DCD2DAD46
:103A80006DED1D9D5DDD3DBD7DFD038343C323A322
:103A900063E3139353D333B373F30B8B4BCB2BAB46
:103AA0006BEB1B9B5BDB3BBB7BFB078747C727A7FE
:103AB00067E7179757D737B777F70F8F4FCF2FAFE6
:103AC0006FEF1F9F5FDF3FBF7FFF77278894881FBF
:103AD000771F881F771F672F71FD6250EDECF7E3AA
:103AE000E80FF61F849171FD819508953F922F9202
:103AF0005F924F927F926F929F928F92BF92AF92FE
:103B0000DF92CF92FF92EF921F930F93DF93CF93A9
:103B1000FC0181E090E0A0E8B0E004E0809F60015B
:103B2000909FD00C7C019F938F93EF01A09FC00DBD
:103B3000D11DB09FD00DFF93EF93BB24AA249927EA
:103B40000081118115950795688179817595679533
:103B5000A801061B170B460F571F41935193208155
:103B60003181359527956A817B8175956795A90186
:103B7000261B370B460F571F419351930F01EAEC59
:103B8000F7E3EA0DFB1D4591559165917591F001A3
:103B9000950320010C031001491E9C03590A300CA7
:103BA000411C591ED803590A300C411C591EB70339
:103BB00040012E033001891EBE03990A700C811C3E
:103BC000991EFA03990A700C811C991E260C371C49
:103BD000481C591C49925992B50320012C0310012D
:103BE000491EBC03590A300C411C591EDA03590AFC
:103BF000300C411C591E970340010E033001891EF1
:103C00009E03990A700C811C991EF803990A700C86
:103C1000811C991E2618370848085908499259925C
:103C2000AC0CBD1CB1FE8CCF04E0A09FC00DD11D1B
:103C3000E00DF11DB09FD00DF00D81E0E81AF90AFA
:103C400009F07BCFEF91FF918F919F91880F991F82
:103C5000B695A795109609F060CFCF91DF910F919F
:103C60001F91EF90FF90CF90DF90AF90BF908F901B
:103C70009F906F907F904F905F902F903F9008950E
:103C80000002030405060708090A0B0C0D0E0E0FAF
:103C90003F922F925F924F927F926F929F928F925C
:103CA000BF92AF921F93DF93CF935C01EB0160E46F
:103CB00070E0EAECF9E3992710E844991127A591FF
:103CC000BB27AA0FBB1FAA0FBB1FAA0DBB1D2D919F
:103CD0003D914D915D91B30320012A031001491ECE
:103CE000BA03590A300C411C591EBA03590A300C48
:103CF000411C591ED50340014C033001891EDC03D1
:103D0000990A700C811C991EDC03990A700C811CA5
:103D1000991E260C371C481C591C662477248824BD
:103D200022273327442770E1220F331F441F220C20
:103D3000331C441C551C661C771C881C220C331C2D
:103D4000441C551C661C771C881C26153705480525
:103D500028F42395621A730A840A23957A9521F729
:103D60004695379527951124439B1FC0621773070B
:103D700010F020E020C0261B370BFF93EF93E0E804
:103D8000FCE340EF37FD04C0221F331F4051FACF40
:103D9000330F3695369536953695E30FF11D5491D0
:103DA000450F342FEF91FF9106C0220F331F220FD2
:103DB000331F08F43FEF39931A9509F080CFCF9164
:103DC000DF911F91AF90BF908F909F906F907F90E9
:103DD0004F905F902F903F900895FF920F931F9305
:103DE000CF93DF9300D0CDB7DEB70E94492C1B8262
:103DF00010E0F12E1A828B81825F8983F0FE08C069
:103E000000E02A81215F49816A818B810E945A2FBB
:103E1000F3948A81805F8A83803881F7175F8B8172
:103E2000815F8B83183429F710E081E089831A823F
:103E300000E02A81822F8F5F8A8303FF0FC0095F12
:103E40001E5F81E089830F5FA2F70F900F900F90A4
:103E5000DF91CF911F910F91FF900895E02FF0E037
:103E6000EA5BFF4DE081EF70F0E0E050F04E8081C2
:103E7000E0ECE80F99F02170E73098F0211116C0BE
:103E8000EAEBE80F22E0F0E0EE0FFF1FEA55F94FF2
:103E900045915591612F89810E949F328981815F6F
:103EA000D1CF2111F0CFE6ECE80FEDCF23E0EBCF3F
:103EB0000F934130C0F49B01280F391F2F5F3F4FF4
:103EC0002170022F01956295607F9FE0899F802D70
:103ED00011242EE0260F4DE0480F6F5F8F5F0E9488
:103EE000232F0F91089529F001E0423061F300E0A3
:103EF000EACF082F060F0695000BE5CF3F924F92B1
:103F00005F926F927F928F929F92AF92BF92CF9269
:103F1000DF92EF92FF920F931F93CF93DF9300D026
:103F200000D0CDB7DEB72091394530913A45C9016F
:103F300082978093394590933A458953944380F50D
:103F40002093394530933A458091193490911A3431
:103F50009195819591098093CA209093CB2075E427
:103F60002933370739F040913834413008F494C48C
:103F700009F49BC4A9982696CDBFDEBFDF91CF91EF
:103F80001F910F91FF90EF90DF90CF90BF90AF9077
:103F90009F908F907F906F905F904F903F9008958B
:103FA0008091D0209091D1202091CE203091CF20AF
:103FB0002093193430931A342091CC203091CD20A5
:103FC00020931B3430931C342091432020932534BC
:103FD00020914220209326342091412020932734A1
:103FE0002091402020933834019780931734909388
:103FF00018348091C72098E189278093C7201092B8
:10400000373410922B341092363490912B3481E057
:10401000890F80932B3420912734921760F18330DD
:1040200050F141E02091D6203091D72020343F41FB
:1040300009F040E02091263430E02423232B09F4BA
:1040400006C44091DA205091DB206091DC20709111
:10405000DD2077FD02C0823670F0809137342091E8
:1040600036342093D6201092D72087778093C920AA
:1040700083E080932B349091363490932A3490933C
:10408000303490913734907890932C348330C0F151
:10409000A0913945B0913A4582E2E7E1F4E301901D
:1040A0000D928A95E1F72091193430911A348827BE
:1040B0009927821B930B8093D0209093D12081E08D
:1040C00090E0821B930B8093CE209093CF20809121
:1040D0001B3490911C349195819591098093CC204B
:1040E0009093CD2080E880934320109242208091CD
:1040F0002B34835090E0809341209093402013CF45
:1041000080E49FE18093233490932434EE27FF27AB
:10411000E81BF90B8091193490911A34E817F907CC
:1041200024F080914520843250F080912B34E0912E
:104130001B34F0911C34833010F0E0ECF0EEE0938F
:104140001D34F0931E348091DA209091DB20A091F1
:10415000DC20B091DD200197A109B1098093DA201C
:104160009093DB20A093DC20B093DD20409130348D
:10417000E42FF0E0EA5BFF4DE081E0932E34809184
:10418000C7208E2311F1E770E0932F34E093283499
:10419000E05FF0E0E258FB4FE491E0932934E091D6
:1041A000283480912F34833010F0E7FD09C0E0916E
:1041B0002934EF5FE0932934F0E0E258FB4FE491BB
:1041C000E195E0932834E1111CC2475F47774093A3
:1041D000303480912A344813C9CFB2C2682F62C2EA
:1041E000E0911B34F0911C34513019F4FB01EB19B0
:1041F000F109E0931F34F0932034052F10E0EB8099
:10420000FC800E191F09023011050CF4DEC1EB2CE5
:10421000F12C50904520442443940EE1501608F4AC
:10422000412C90E04D831E82870104501109F80152
:10423000E4290D811E810A5B1F4D68018C010A5B18
:104240001F4D0B831C83EF2B09F423C1470117E09B
:10425000811A910801E0E8E05E1608F400E0802A87
:10426000892809F419C1F6E0BF1638F4F601208553
:10427000EB81FC813085231B330BF6011082E98131
:10428000FA811082D09033340D2D10E00A5B1F4D5F
:10429000F801108270902E34172D1062EB81FC8192
:1042A00010831D2D187861F40091323410E00A5B00
:1042B0001F4DF6E0DF2ED60CF801D082225E3F4F74
:1042C000F3E0BF1608F066C00D811E81025011098F
:1042D000C02EE8E8CE22D12CC114D10409F0DFC0F1
:1042E0000A5B1F4D99249394F8011081171101C0A6
:1042F000912CC92CED81FE8132960E2F087810E0AA
:104300000115110509F0CEC0EA5BFF4D9924939485
:10431000E081E71101C0912C092DE0E1E427F0E0F4
:10432000EA5BFF4D4081E62DF0E0B496882483944B
:10433000912C4E171F0609F0812CC00ED11EF1E002
:10434000CF1AD108C80CD91C49E04C9DF0014D9DF5
:10435000F00D112456945694E519F1092E1B3F0BCC
:10436000E09128348C010E0F111DE7FD1A95F8011C
:104370003196E7FF99C087E892E08E199F09EB819B
:10438000FC814081480F4083680F791F6093D420DF
:104390007093D52080911B3490911C34680F791F45
:1043A000620F731F60931F34709320348091173411
:1043B000909118348A179B070CF4CD018093213417
:1043C0009093223421E0523009F020E0242980919A
:1043D00023349091243480549F41822B892B99F06F
:1043E0002FEF250F81E0563008F480E091E0F3E0F4
:1043F000BF1608F490E089233A2891E0311090E04C
:104400008923522F581B50932D34E0911F34F09183
:10441000203480912134909122348E179F071CF014
:10442000533008F449C0A0913945B0913A4582E231
:10443000E7E1F4E301900D928A95E1F78091193458
:1044400090911A349195819591098093D020909301
:10445000D1208091213490912234919581959109B8
:104460008093CE209093CF2080911F349091203460
:104470009195819591098093CC209093CD20809146
:104480003234809343201092422080912D3491E069
:1044900032CE27EF3FEFF1CE24EF3FEFEECEE1E05B
:1044A000CE2E28CF01E039CF4096F0E087219F2320
:1044B000880F8074992763CFE093D220F093D320A4
:1044C00081E020911734309118342E173F070CF0FB
:1044D00080E050912D345F5F50932D3490912B34B8
:1044E000591710F4811191CFE0931F34F0932034C9
:1044F00040913034242F30E07091313410913234B7
:10450000809126348115F1F18091D6209091D720A9
:1045100080340FE19007B1F1E03C50EEF50791F1E6
:104520005091C92057132EC08217930759F5209137
:10453000D4203091D52080911B3490911C349195DA
:1045400081959109821B930B8093D8209093D92059
:104550001093C820220F232F221F330B8091452058
:10456000820F809345202091394530913A452E5D48
:104570003F4F2093394530933A45809119349091BB
:104580001A34E9CC8091333490E08A5B9F4D50918E
:10459000C7205A5FDC015C93672F70E06A5B7F4D38
:1045A000DB011C92A12FB0E0AA5BBF4D1C922A5BDD
:1045B0003F4D80912E34D9018C93A0913434B0E0DA
:1045C000AA5BBF4D809135348C9380911D349091BE
:1045D0001E348E179F0774F4E0931D34F0931E343D
:1045E0004093363480913234807890913134892BE5
:1045F0008093373480912C34811509F4AEC0109229
:104600002C344093313480E88093333480933234B7
:1046100030902C34809137348325311005C080913F
:10462000313490912834890F80933134809334341D
:10463000982F987809F0B3CD50912534252F30E08C
:10464000B90160587109F901EA5BFF4DE081F0E0C2
:104650006E237F236115710569F0682FFB01E21B52
:10466000F30B32973CF4261B370BA0E4BFE122305A
:10467000310524F0A0911D34B0911E34A0931D3457
:10468000B0931E34B0902F3491E013E0B11608F0CF
:1046900090E05813A3CD911509F4A0CD60E16827EF
:1046A000609334349B012A5B3F4D29833A83F9019F
:1046B000A080A09235346090C72001E010E00B8309
:1046C0001C82A11411F01B821C82582F541B57709E
:1046D0009801511120E06B817C81261B370B70E023
:1046E000292337239A2D9621292B2115310509F0ED
:1046F00056CDEA2DE770F0E0E256FB4F059115919B
:104700006A2D607C95E20902600D711D1124609391
:10471000D4207093D52077FF02C0A0E4BFE1A0931E
:104720001D34B0931E3450912B34E0911934F09124
:104730001A34AE17BF070CF453CD523008F450CDE5
:1047400020911D3430911E34C9018854914E813717
:104750009D4308F064C0C90175C050912F34809109
:1047600028346091313470912E34209129342750AF
:10477000330B052F0450110BF801202B3F2B232B5B
:1047800009F04BC0E82FE595E77093E0940FE92717
:10479000E0933334AE2FB0E0AA5BBF4D2C919091E3
:1047A000C720291B330B2630310581F091E05530AD
:1047B00008F090E080913534890F80933534A998C2
:1047C00080913534811509F423CFE9CC91E0AE2FE7
:1047D000A927B0E0AA5BBF4D92E0E927F0E0EA5BD1
:1047E000FF4D9C912081922B31E0911101C030E06E
:1047F000982F990F990B840F911D861B9109272FD4
:104800002072822B21E0533008F420E02323822BF6
:10481000892B61F660933234D2CF31E0E9CF82E662
:1048200080932B3441E08091233490912434803460
:104830009F4109F040E0C901805C904E842B0097B5
:1048400009F089CF80931D3490931E34DECB809184
:10485000C72098E189278093C7202091394530915E
:104860003A452E5D3F4F2093394530933A45E091CC
:104870001D34F0911E3481E090E040911B34509142
:104880001C34E417F5070CF080E08E0F9F1F809317
:104890001D3490931E345FCB42E2F901A7E1B4E3EB
:1048A00001900D924A95E1F72DCC42E2F901A7E182
:1048B000B4E301900D924A95E1F7EE27FF27E81B3C
:1048C000F90BE093D220F093D320A99AF9CD8F92DF
:1048D0009F92AF92BF92CF92DF92EF92FF920F938F
:1048E0001F93CF93DF9300D00F92CDB7DEB789E34C
:1048F00095E48093394590933A455E9880E18093A2
:10490000C720109245201092D8201092D9201092E2
:10491000C8201092CA201092CB20E6E4F0E281E891
:10492000DF011D928A95E9F78091C92098E0A2E104
:10493000B9E0292F915098F5909344208093C92095
:10494000AA24AA948FEF8983BA2C1FEF35E1E32EB6
:1049500034E3F32E812C912C1B821A8240E4C42E66
:104960004FE1D42E8091CA209091CB20823C904E72
:1049700014F05E9B52C07D995E9A5E9BF3CF2496A5
:10498000CDBFDEBFDF91CF911F910F91FF90EF90D0
:10499000DF90CF90BF90AF909F908F900895492F58
:1049A00050E0FA01EA56FB4F34918A010A5B1F4D31
:1049B000BA016A547F4D88E0830FFB018083305F2A
:1049C000F8013083A08BB801605A7F4FFB01B083A0
:1049D0002550298388E0815008F4ABCF282F30E0A0
:1049E000220F331F2750310960E1869FF001112407
:1049F000EA5BFF4DE40FF51F229FB001239F700D6E
:104A0000700D11249B013595279535952795798152
:104A1000779F200D11242087DECF0E94ED1E95E1A7
:104A2000E91694E3F90609F0AEC00FEF27E04FE76F
:104A300062E08AE70E94232F00E02DE74FE768E756
:104A40008AE70E94232F89818A29883028F441E04F
:104A50006A2D89810E94581F7D995E9AD7018C9199
:104A6000843009F0C7C06298669B25C066987D991E
:104A70005E9A7B9B03C0BA81B150BA83799B03C015
:104A8000EA81EF5FEA837E9B03C0FB81F150FB83E9
:104A90008FB181702B81280F2B837A9B0CC03A81B8
:104AA00031137AC02B1178C040E06B818A810E945B
:104AB000581F1FEFB12EFA81FF3F09F491C0F83063
:104AC00008F091C03B813F3F09F48FC0383008F0B7
:104AD0008FC07A81791103C08B81881569F041E01C
:104AE0008B1040E081E0911280E04823682D892DF1
:104AF0000E94581F8B809A8042E06B818A810E94BD
:104B0000581F0E946B3B0E94A63BAA9888955E990D
:104B100002C0629BA9CFE0ECF0EEE093D020F093CE
:104B2000D120C092CE20D092CF208091D8209091D9
:104B3000D9208093CC209093CD208091C820809361
:104B40004320F1E0F093422023E020934120109293
:104B500040200E947E1FD7018C91843009F087C0CD
:104B60008091CA209091CB2080349F4109F074C07D
:104B7000E5E1EE16E4E3FE0609F47EC025E1E22E4F
:104B800024E3F22E6AC000E027E04FE762E08AE704
:104B90000E94232F0FEF51CF1F3F19F06FEFB61276
:104BA00014C0AB8170E1A79FC0011124BA818B0FA3
:104BB000911D8093D6209093D720BA2E1B2F41E0D1
:104BC0006B2D812F0E94581F76CF8B818295807F1D
:104BD000EA818E0F8093C920629AB62E1FEFEFCF25
:104BE00027E02A836FCF1A826DCF67E06B8371CF86
:104BF0001B826FCFC092D620D092D72080911434E0
:104C0000A0E8B0E002C0AA0FBB1F8A95E2F7CD0171
:104C1000A92FAA0FAA0B8093DA209093DB20A093F0
:104C2000DC20A093DD200E941D7A4091DA20509173
:104C3000DB206091DC207091DD20480F511D611D4B
:104C4000711D4093DA205093DB206093DC20709339
:104C5000DD200E946B3B5FCFAA9A2091C92027706C
:104C6000A090C9202983A2948FE0A8227BCEF5E1F1
:104C7000EF16F4E3FF0680CF96E1E92E94E3F92ED8
:104C8000ECCF0F931F93CF93DF93589A5E981092B7
:104C900014340E94492CC2E0D2E303E012E0589B96
:104CA00058C05898669B15C066987B99CF5FC430F2
:104CB00008F0C0E07A9B08C0809114348F5F803187
:104CC00008F054C08093143479990E9467247D9928
:104CD0005E9AD093E0211092DF218EE69EE20E9440
:104CE0004A311092E0211093DF218CE19DE20E9475
:104CF0004A31C0FF3EC08FEF9BE20E944A3185E0FF
:104D0000809315341092E0210093DF2183E19DE22E
:104D10000E944A31C1FF33C08FEF9BE20E944A31AB
:104D200085E0809316341092E02184E08093DF21A7
:104D300086E794E00E944A31809114340E94B43195
:104D40001092E0218FE08093DF2180E694E00E94C2
:104D50004A310E946B3B0E94A63B88955E9B9FCF89
:104D6000589ADF91CF911F910F91089510921434AA
:104D7000ABCF84E09DE20E944A3184E0C1CF84E061
:104D80009DE20E944A3184E0CCCFEF92FF920F93D4
:104D90001F934091103450911134609112347091EE
:104DA000133423E132E286E0F901E590F5900591B4
:104DB00015914E155F056007710780F481502450EE
:104DC00031098F3F89F794E0899FF0011124ED505C
:104DD000FE4D059115912591359104C001E010E03B
:104DE000823088F7619B11C0401B510B610971092A
:104DF00040931034509311346093123470931334F1
:104E00001F910F91FF90EF900895629B05C0400F96
:104E1000511F611D711DECCF811101C087E094E02D
:104E2000899FF0011124E950FE4D459155916591FE
:104E30007591DECFEF92FF920F931F93CF93DF9385
:104E400080910C34181614F410920C3480910E34A6
:104E5000811103C081E080930E34809110349091D1
:104E60001134A0911234B0911334892B8A2B8B2BDF
:104E700019F481E08093103480911234883128F540
:104E80008C3028F5863028F5833028F5811125C02F
:104E900081E08093DE2080910D34833009F489C055
:104EA000F0F4813009F473C0823009F057C0629A7F
:104EB000E4E1F4E32E2F9E2F8E2F821B0AF477C09D
:104EC00081E881939E13F8CF10C080E2E2CF80E1A9
:104ED000E0CF88E0DECF84E0DCCF82E0DACF843040
:104EE00009F47BC0853009F494C080910E34082FFA
:104EF00010E020E031E0281B3109220F331F60E071
:104F000070E0C0E0E4E1F4E3D72F472F50E0819157
:104F1000DA01AC5EBB4C7D014C5E5A4CDA018C93DD
:104F200062990CC04081982F990F990B840F911DA5
:104F300047FD9A9597FD019695958795DF3F21F05E
:104F4000D701AF5FBE4F8C93620F731FCF3709F04D
:104F500069C09801220F331FCF5FD6CF209160091F
:104F60003091610984E194E3A5E5B2E6482F2A9FD8
:104F7000B0012B9F700D3A9F700D11249B012F5F84
:104F80003F4FFC01019630834813F1CFAECFC4E10F
:104F9000D4E30C2F10E41C1B8C2F810F7E01219673
:104FA0000E94651DD7018C930C13F6CF9ECF8FE71F
:104FB00088CFE4E1F4E380E0982F9195990F915820
:104FC00091938F5F8038C1F7E4E9F4E3982F990F4C
:104FD0009F5791938F5FD1F788CFEFEAFFE184E18C
:104FE00094E32491DC01019621952C93319624E3DE
:104FF00084399207B1F720E8422F4058550BFA0147
:10500000E155F04EE491DC01EC9301962F5FA1F79E
:105010006CCF40E051E060E879E084E194E30E94E5
:10502000F07B63CFCF5F09F06FCFA091DE20B0E0BF
:1050300020E23CEB4EEB50E00E945D7B209110346F
:10504000309111344091123450911334E6E0E093E2
:10505000A200E32EF42EEF2899F5E0934009542F97
:10506000432F322F20E00E940D7B215031092093E5
:1050700076093093770920910C34E091DE20CE9FA1
:10508000E02D1124F0E0EC5EFA4C3081A303812D79
:10509000112460910F340E944D1AEC2FF0E0E15280
:1050A000FF4D8083CF5F39F75998629887E08093EE
:1050B000A200DF91CF911F910F91FF90EF90089583
:1050C000E1E0E0934009CFCFEF92FF920F931F935F
:1050D000CF93DF93589A629A5E98809173008C7F89
:1050E0008093730080EC80938001109220081092CE
:1050F00021088FE59AEE8093260890932708109256
:10510000600810926108809366089093670883E0B6
:105110008093000888E08093400882E08093050631
:10512000C0E0D0E0FF24F3948091200B80FD09C003
:10513000A99A8370823031F487EE92E30E94507A0C
:1051400001C0AA9A0E94492C1092E0211092DF21FE
:1051500085E09FE20E944A3186EA9FE10E944A313F
:105160008AE00E94C73185EF0E94C7311092E0218A
:10517000F092DF218DE99FE10E944A318091610820
:105180000E94C731809160080E94C7311092E021CF
:1051900082E08093DF2184E99FE10E944A3180917F
:1051A000210B0E94C7318091200B0E94C7311092C1
:1051B000E021E3E0E093DF2188E89FE10E944A31AB
:1051C000809193008F5B0E94FD301092E021F4E00B
:1051D000F093DF218FE79FE10E944A318AB30E945A
:1051E000C7311092E02185E08093DF2186E79FE1BF
:1051F0000E944A31809178000E94C7318E9A1092A5
:10520000E021E6E0E093DF218DE69FE10E944A3154
:1052100081E00E948A400E945831F8948FB789B982
:105220001092E021F7E0F093DF2184E69FE10E94F5
:105230004A310E9469410E94583189B18FBF7894E8
:105240001092E02188E08093DF218BE59FE10E94AE
:105250004A310E940C410E9458318E981092E021F0
:10526000E9E0E093DF2182E59FE10E944A318091ED
:1052700040000E94C731809150000E94C731809148
:1052800051000E94C731809153000E94C731F092B3
:10529000E021FFE0F093DF218CE39FE10E944A319F
:1052A000AA98A998E12C00E010E090E89E0D8BE010
:1052B000083010F49E2D8AE09093E0218093DF2146
:1052C000F80181918F010E94C731F0E1EF0E0031AA
:1052D000110559F7669B14C066987D995E9A7B9B71
:1052E00003C00E949A3F639A7A9B03C085B38F25BF
:1052F00085BB799B05C0D13091F10E94E33BD1E0A1
:10530000E091E321F091E421EC0FF11D9F01395070
:105310008081809580837297E217F307C9F7CF5F8A
:10532000C03109F4C0E00E946B3B0E94A63B889507
:105330005E9BFACEA89882E0809306061092000841
:105340001092400880917300836080937300589A94
:10535000DF91CF911F910F91FF90EF9008950E94E0
:105360002B3CD0E0CDCFCF938CEE92E30E94507ACD
:105370000E94492C8EE18093E021C1E0C093DF219F
:1053800065E486EB9EE10E94AE2C8AE08093E021EA
:1053900083E08093DF218DE99EE20E944A318FE80D
:1053A0009EE20E944A31C093E0218DE08093DF218C
:1053B00085E09FE20E944A3183E39FE10E944A31E7
:1053C0008AE00E94C73185EF0E94C731C093E02177
:1053D0008EE08093DF2185E29FE10E944A318AE1DD
:1053E0000E9496318FE20E94FD3081E00E9496314A
:1053F0008FE20E94FD3085E10E949631C093E0214A
:105400008FE08093DF2180E29FE10E944A3180910A
:1054100078000E94C731C9E78E9A0E94686A40E00E
:1054200050E066E082E20E94B87767E082E20E9484
:10543000F3770E946B3B0E94A63B0E940C418D5C5F
:1054400097408736910578F0AA9A8E988091400906
:1054500081110BC08895C15011F0669BDDCF669815
:10546000589ACF910895AA98F0CF8FEF0E94744078
:10547000F2CF1F93CF93DF93CDB7DEB7AC97CDBFFD
:10548000DEBFA99A811591F11FEF180F8CE0189FCC
:10549000B0011124605E764F4CE050E0CE01819661
:1054A0000E94F07B80E2189FB00111246050784F79
:1054B00040E250E0CE0101960E94F07B4CE050E0CB
:1054C00060E87AE0CE0181960E94947B40E250E051
:1054D00060E079E0CE0101960E94947BA998AC9699
:1054E000CDBFDEBFDF91CF911F9108954CE050E01A
:1054F0006FEE71E2CE0181960E94847B40E250E023
:105500006FEC71E2CE0101960E94847BD7CF1F938E
:10551000CF93DF93CDB7DEB7AC97CDBFDEBF182FEB
:10552000AA9A4CE050E060E87AE0CE0181960E94B1
:10553000F07B40E250E060E079E0CE0101960E940D
:10554000F07B8CE0189FB0011124605E764F4CE038
:1055500050E0CE0181960E94947B80E2189FB001BA
:1055600011246050784F40E250E0CE0101960E9435
:10557000947BAA98AC96CDBFDEBFDF91CF911F91EF
:1055800008950F931F93CF93DF935E98C0E00FE0D1
:1055900015E00E94492C1092E0211092DF218DE944
:1055A0009EE20E944A318EEC9CE20E944A31D0E099
:1055B0001093E02182E08D0F8093DF21CD1346C050
:1055C0008DE20E94FD3081E80E94FD3088E19FE17C
:1055D0000E944A3180E38D0F0E94FD30DF5FD8309A
:1055E00039F71092E0210093DF2182E09FE10E94D1
:1055F0004A31669B1EC06698789901C07C99CF5F3E
:105600007E9901C07F99C1507D995E9A7B9B03C0B2
:1056100080E00E94392A7A9B04C081E08C0F0E94AE
:10562000392A799B03C08C2F0E94872AC83008F042
:10563000C0E00E946B3B0E94A63B88955E9BA9CF71
:10564000589ADF91CF911F910F91089581E1809336
:10565000E021BCCFEF92FF920F931F93CF93DF9384
:105660000091E1211091E221E801229680E0E82EEC
:1056700080E0F82E0E5F164F8091CF0187FDFCCFA2
:1056800040E150E0B701CE010E94947B629680E138
:10569000E80EF11C0C171D0779F7DF91CF911F91D0
:1056A0000F91FF90EF900895EF92FF920F931F9349
:1056B000CF93DF935E980E94492C0091E1211091D5
:1056C000E221E801229680E0E82E80E0F82E0E5FCD
:1056D000164F8091CF0187FDFCCF40E150E0B7012C
:1056E000CE010E94F07B629680E1E80EF11C0C175F
:1056F0001D0779F7669B03C066987D995E9A0E94A4
:105700006B3B0E94A63B88955E9BF4CF589ADF9135
:10571000CF911F910F91FF90EF900895EF92FF921C
:105720000F931F93CF93DF935E98C0E0DFEF0CE100
:105730000E94492C0093E0211092DF218FEB9EE222
:105740000E944A3186E0E82E8CE2F82E10E082E0DA
:105750008093E021810F8093DF21C11312C08DE27D
:105760000E94FD3081E80E94FD30123009F447C0EC
:10577000133009F447C0113041F06F9B08C0619AA3
:1057800006C08EE08093E021F0CF6A99F8CFC70180
:105790000E944A3161981F5F82E1E80EF11C1430CB
:1057A000B1F60E94686A40E050E06DE081E00E943E
:1057B000B8776DE084E40E94F37781E08093E02184
:1057C0008FE08093DF218BEF9EE10E944A31669B40
:1057D00020C06698789901C07C99CF5F7E9901C0FE
:1057E0007F99C1507D995E9A7B9B3AC0C23079F116
:1057F00060F4C11125C08DB180588DB908C0689B77
:10580000C6CFBDCF699BC3CFBACFC33031F1C0E0A3
:10581000DFEF0E946B3B0E94A63B8895D11519F0E3
:10582000D1505E9B85CF6DB189E19DE00E94117CD6
:10583000589ADF91CF911F910F91FF90EF900895AB
:105840008DB194E089278DB9C1E0DFEFE2CF8DB152
:1058500091E089278DB9DFEFDCCF8DB192E0F9CFF0
:10586000C430A8F6F8CF67990EC0679A85EE91E22A
:1058700025ED3AE22093E3213093E4218093E12166
:105880009093E2210895679887EE9AE227ED33E33B
:10589000F1CFE091E121F091E2219F01375F8FEF9D
:1058A00082838383848385838683878380878187BC
:1058B000828783878487858786878787808B818B8C
:1058C0007296E217F30761F71092E0211092DF2140
:1058D0000895CF93DF93C7EED1E240E150E06FEF40
:1058E00070E0CE010E948D7B62968AE2C73ED807A7
:1058F000A1F7C9EEDAE240E150E06FEF70E0CE01CF
:105900000E948D7B629683E3C93ED807A1F7DF91A1
:10591000CF910895CF93DF9300D00F92CDB7DEB72C
:1059200089836A834B835C83EB81FC81849131960C
:1059300064918F3F69F02B813C812E5F3F4F2B8319
:105940003C833A81630F9981890F0E94BD19ECCF86
:105950002496CDBFDEBFDF91CF9108950F931F93A3
:10596000CF93DF93EC018C01060F111DC017D107F7
:1059700029F4DF91CF911F910F910895FE01849139
:105980000E94D4192196F2CF0F931F93CF93DF93E8
:1059900000D0CDB7DEB789838A30C9F1282F2451D2
:1059A000330BC901220F331F280F391F8901075DEF
:1059B000124E245D324E2A833B83F80184910F5F9F
:1059C0001F4F619B02C0806880950E94D4198A8114
:1059D0009B810817190789F7998186E09C3179F135
:1059E00029812D3181F48EE00E94D4198091E0212B
:1059F0008F5F8093E0218091E02187FD0CC0898139
:105A00008A3081F408C0398188E03A31C1F0809150
:105A1000E02187FF0FC01092E0218091DF218F5F8E
:105A20008093DF210F900F900F90DF91CF911F9106
:105A30000F9108959CB1892F827091FD8FE70E948C
:105A4000D419D9CFCF93DF93EC01FE01849181115A
:105A500003C0DF91CF91089521960E94C42CF5CF09
:105A6000CF93DF93C82F843658F0DCE9D80F81E359
:105A7000D43618F0D8E3DC0F82E30E94C42CCD2F7B
:105A800080E3CA3040F40E94C42C80E38C0FDF9185
:105A9000CF910C94C42C8F5FCA50F3CFCF93C82FF3
:105AA00082958F700E94E4790E94C42C8C2F8F7095
:105AB0000E94E479CF910C94C42C4F925F926F9224
:105AC0007F929F92AF92BF92CF92DF92EF92FF921E
:105AD0000F931F93CF93DF93CDB7DEB72897CDBF3A
:105AE000DEBF69017A015E012FEFA21AB20A98E0C7
:105AF000F50111929A95E9F7262F30E0F2E18F9F98
:105B00002019310911240091E3211091E421020FA1
:105B1000131F8093E0216093DF21F7FE9DC0F09476
:105B2000E094D094C094C11CD11CE11CF11C629B78
:105B30008FC08FE3F8018083729780837297808390
:105B4000729780830C5611098CB181FB992491F8CE
:105B500081FDBAC0F0E6CF16F3E4DF06F9E9EF06FF
:105B6000FBE3FF060CF0B3C021EED21625EFE206F0
:105B700025E0F2060CF474C0B601C70120EA36E84D
:105B800041E050E00E942F7B69017A0187E192E2B7
:105B9000D501AE0147505109FC01459055906590E3
:105BA0007590C414D504E604F70408F097C0049770
:105BB00011974A175B0781F797E0F92E619902C0A8
:105BC00083E0F82EF501EF0DF11D8081629B99C0F5
:105BD000E4E18E9FC00111249C012F59334ED8015E
:105BE00011978559934EF9012F5F3F4FE491E0954E
:105BF000EC93529782179307B1F79801245B310910
:105C0000D801FC01E4910196E095EC9352972A1794
:105C10003B07B9F7F801E85DF1099F1409F468C082
:105C20008F01FA94FFEFFF12CDCF2896CDBFDEBFD4
:105C3000DF91CF911F910F91FF90EF90DF90CF9068
:105C4000BF90AF909F907F906F905F904F9008951E
:105C50008DE20E94C42C78CF629974CF80E2F9CF94
:105C600080E8C81686E9D80688E9E806F1046CF0F1
:105C7000B601C70120E137E240E050E00E942F7BEF
:105C800069017A019924939481CF90E4C91692E432
:105C9000D9069FE0E906F1046CF0B601C70128EED1
:105CA00033E040E050E00E942F7B69017A0142E03E
:105CB000942E6CCFB601C70124E630E040E050E0FE
:105CC0000E942F7B69017A0133E0932E5FCF2FE092
:105CD000C22E27E2D22EE12CF12C58CF17962C9110
:105CE0002F5F2C931797C418D508E608F70859CFEB
:105CF00089EF8083F801EA5EF10980830052114048
:105D000090CF805D0E94C42C9F108BCF8EE20E94AA
:105D1000C42C87CFE62FF0E0EE0FFF1FEF5EFF4DA4
:105D200020813181DC010E94567B41FF06C0AAE040
:105D3000B0E09B01AC010E945D7B28E030E040E0D8
:105D400050E00E942F7B6091DF218091E0210C9434
:105D50005D2D8093E0216093DF21CA010C94222DF8
:105D6000FF920F931F93CF93DF93F42E982F962BD0
:105D7000F2F0C091E321D091E421262F26952695BB
:105D8000269530E092E1899F201931091124C20F34
:105D9000D31F677000E810E002C0159507956A955B
:105DA000E2F741110AC00095888180238883DF9142
:105DB000CF911F910F91FF90089581E0481303C088
:105DC00088818027F3CF9FEF491303C08881802B00
:105DD000EDCF0E94017A8F15C8F3E9CFCF93DF93FF
:105DE00000D00F92CDB7DEB749832A83803CF0F410
:105DF0008C83803810F08FE78C83603C10F56B83C8
:105E0000603810F09FE79B838C819B81891780F419
:105E1000892F9C819B838C839C818B81981740F474
:105E20002496CDBFDEBFDF91CF9108951C82E5CFD0
:105E30004A8169818B810E94B02E8B818F5F8B8319
:105E4000EBCF1B82E9CF0F93CF93DF9300D00F925C
:105E5000CDB7DEB789836C834A832B83202F462FEF
:105E60006A810E94EE2E202F4B816A8189810E94D7
:105E7000EE2E8C819B818917C0F0402F6B81898128
:105E80000E94B02E402F6B818A810E94B02E8B81A0
:105E90008F5F8B838C819B81891778F72496CDBF88
:105EA000DEBFDF91CF910F9108958B819C819B8301
:105EB0008C83F0CF0F93CF93DF9300D00F92CDB7A9
:105EC000DEB789836C834A832B836217A0F0202F6F
:105ED0004B816A8189810E94EE2E8B818F5F8B833B
:105EE0008C819B81891798F72496CDBFDEBFDF9107
:105EF000CF910F9108958B819C819B838C83F0CFF0
:105F00002F923F924F925F926F927F928F929F92C9
:105F1000AF92BF92CF92DF92EF92FF920F931F93B7
:105F2000CF93DF93CDB7DEB72A97CDBFDEBF89878A
:105F30006A87F42E122FCE82261708F454C1E61673
:105F400028F4EA86E62E89850987082FE11630F0C5
:105F50008E2DE12E182F802F0F2DF82E902E2985B3
:105F6000921A0AF04BC0922E901A3FEF3A838E2C71
:105F70008A85881A4F2C9985491A0AF042C0492E01
:105F80004F1855245A94712E2A85721A9814E4F1E8
:105F9000882D892C982E198266246394471424F046
:105FA000872D742C482E612CD72CD5944A85E41665
:105FB00009F480C0382C3594C984212CA82CB82C25
:105FC000BB0CBB08972D990F990B7F829887822D68
:105FD00090E02A141B040CF06DC029853C2DC216DC
:105FE00010F439852C2D1B821FC08E2DE12E1A85B1
:105FF0008A87802F0F2DF9848987B0CF41E04A83AB
:10600000B6CF55245394BFCF31E03983C5CF222476
:106010002394280E390C3A141B04BCF44981411115
:1060200007C001964A81C40E282E8A159B057CF371
:106030001C82D40C8F819885D81619066CF46110D7
:1060400010C09985950D9987F4CF3818498141156D
:1060500079F34A814B83DFCFD718611411F05C824A
:10606000E9CF6C2DC31608F4632F3985631708F444
:10607000632F8C2D2C1508F4822F4985481708F4BE
:10608000842F2E814A850E94EE2E8981811102C0C3
:106090009A81C90E2B81C20E611003C03985350D5E
:1060A000398749858C81480F49879A859F5F9A87F0
:1060B000E9128DCFCF2CC01AA2F5C02ECF182FEF2A
:1060C0002A83312E3E18C3147CF58C2DC32C382E18
:1060D00041E04983EC2CE594A12C8C2C9C2C990C50
:1060E0009908972D990F990B7C829D832A2D30E07A
:1060F0008A149104DCF42A96CDBFDEBFDF91CF91E4
:106100001F910F91FF90EF90DF90CF90BF90AF90D5
:106110009F908F907F906F905F904F903F902F90C7
:10612000089531E03A83CDCF1982D4CF9985802F5D
:10613000091710F48985902F590108C03981311150
:1061400011C04FEFA41AB40A2A81020FA814B9048F
:106150004CF4E30CE81419048CF3EC1829812A8020
:10616000211101C0212C1B820BC0D40C2C813D813C
:10617000D21613069CF5611006C03985350D398796
:106180004985F412F2CF602F081708F4682F89852B
:10619000681708F4682F802F901708F4892F9985C5
:1061A000981708F4892F2E814A850E94EE2E2981A6
:1061B000211102C03A81030F611003C04985450DCA
:1061C00049878A858F5F8A87181708F494CF020D54
:1061D00099852B81920F9987A39488CFD718611442
:1061E00091F25B82C3CFE21608F4FFCE8A852A873C
:1061F000182F89854987F82EA9CE9091DF218A3002
:1062000039F41092E02181E0890F8093DF21089515
:10621000482F4052550B9A0185E0829FA001839F31
:10622000500D11249A012958354E892F90E0609124
:10623000E02172E1679F8019910911246091E321A7
:106240007091E421860F971F4458554EDC01F901E7
:106250002F5F3F4F6491EE276199E395E150E62768
:10626000EC9352974217530791F72091E0212B5F4F
:106270002093E02127FD0DC0FC01EA55F109882794
:1062800061998395815080838091E0218F5F809315
:10629000E0210895CF93DF93EC01FE0184918111F9
:1062A00003C0DF91CF91089521960E94FD30F5CF74
:1062B000FF920F931F93CF93DF93EC0180E3C031E4
:1062C00097E2D90720F590E3F92EC83E93E0D9076D
:1062D00010F500E3C436D10510F510E3CA30D1053E
:1062E00010F5803311F00E94FD308F2D0E94FD309B
:1062F000802F0E94FD30812F0E94FD308C2F805D09
:10630000DF91CF911F910F91FF900C94FD308F5F23
:10631000C051D742D4CFF394C85ED340D6CF0F5FDD
:10632000C456D109D7CF1F5F2A97D8CFCF93DF9319
:10633000C82F843658F0DCE9D80F81E3D43618F042
:10634000D8E3DC0F82E30E94FD30CD2F80E3CA301A
:1063500040F40E94FD3080E38C0FDF91CF910C94CC
:10636000FD308F5FCA50F3CFCF93C82F80E3CA3080
:1063700048F4803351F00E94FD3080E38C0FCF91C0
:106380000C94FD308F5FCA50F2CF80E2F4CFCF93F0
:10639000C82F82958F700E94E4790E94FD308C2F67
:1063A0008F700E94E479CF910C94FD30CF93DF93EE
:1063B000382F5EEE5303C0011124680F792F711D31
:1063C0008091E3219091E421860F971F30E0BFEF89
:1063D000622F70E0EB016296341312C0DF91CF910F
:1063E0000895E52FFA2FB1935E2FAF2FE52FE81B0D
:1063F000E217B8F3860F971F8C1B9D0B3F5FECCF06
:10640000582FA92FF3CF0F931F93CF93DF93FA0148
:10641000D4919A012E5F3F4F31964491469546950F
:106420004695582F7EEE7503C0011124860F911DED
:106430006091E3217091E421860F971F60E0E0E016
:1064400050E012E1140F6D1328C0DF91CF911F911E
:106450000F910895E1110CC0D9011196F9015491E1
:10646000FD010491501316C03196E4912D5F3F4F0A
:10647000E150A72FBC2F752F70957D937A2FCB2FCE
:10648000F72FF81BF41730F3840F911D811B91092E
:106490006F5FD9CF9D01E1E0EBCF782FC92FF0CF0F
:1064A0001F93CF93DF9300D0CDB7DEB78B83698383
:1064B0004A83E0E0443638F0842F84568436B8F1BD
:1064C00084568A83E2E010E08A818A3098F523308E
:1064D00070F0F0E0EE0FFF1FE553FC4E4591559133
:1064E00069818B810E9403328B81835F8B83E12FD3
:1064F000F0E0EE0FFF1FE553FC4E45915591698189
:106500008B810E9403328A81E82FF0E0EE0FFF1F9B
:10651000E553FC4E4591559169818B81835F0F90C6
:106520000F900F90DF91CF911F910C9403328A83CB
:10653000E1E0C9CF1F5F8A818A508A83C5CF4F921D
:106540005F926F927F928F929F92AF92BF92CF9203
:10655000DF92EF92FF920F931F93CF93DF9300D0C0
:10656000CDB7DEB729834115510581F1FA01A49118
:106570003196E491E695E695E695EE2EF12C262FE0
:10658000660F330B89010E0F111D10161106F4F45E
:106590004E5F5F4FF9019EEE8902E00DF11D11245F
:1065A0006091E3217091E4216E0F7F1F982F990F66
:1065B000990BC12C712C4C018A0E911C5701E2E100
:1065C000AE0EB11C881599050CF462C00F900F90A7
:1065D0000F90DF91CF911F910F91FF90EF90DF907F
:1065E000CF90BF90AF909F908F907F906F905F9073
:1065F0004F900895C1100FC06A01FFEFCF1ADF0A54
:10660000FA017490F6016490761022C03196E491FC
:106610004D5F5F4FCE2ECA948038910560F4F0E153
:106620004F16510440F4E981E11116C0FC91D72CBA
:10663000D094FD21FC931196FFEF4F1A5F0A40168C
:106640005106C4F26E0D7F1D6A197B090196BACFFF
:10665000A601CC24C394DFCFF981F13029F4FC9159
:10666000D72CD094FD29E6CFE981E23019F4FC91D2
:10667000F721E0CFF981F33019F4FC91F729DACF53
:10668000E981F72DE43011F4FC91F725F095D2CF94
:106690002901DB01D4CF88EA91E62091A10A27FFE6
:1066A00003C08091A00A08952AE62A95F1F700C058
:1066B000019799F780E00895E091E9339091EB33E9
:1066C0009830E0F791E09E0FF0E0E751FC4C8383B7
:1066D000F8948091EB338F5F8093EB3383E1809369
:1066E000A30A7894983008F090E09093E9330895E5
:1066F0001F921FB61F9211248F938BB78F939F9376
:10670000EF93FF938091EB338115E1F081508093FB
:10671000EB33E091EA3381E08E0FF0E0E751FC4C7F
:1067200093819093A00A883008F080E08093EA3348
:10673000FF91EF919F918F918BBF8F911F901FBE03
:106740001F90189580E18093A30AF2CF8F929F92B9
:10675000AF92BF92CF92DF92EF92FF920F931F936F
:10676000CF93DF931092080410920904A9988937F7
:1067700068F4833470F08354863358F4E82FF0E0E3
:106780008827E75BF3488F4F0C944E7B8B3B09F4D3
:10679000B0C180E00DC0E8E0FFE2ABE8B4E58FE80F
:1067A00094E524912D9331968A179B07D1F784E0C5
:1067B000DF91CF911F910F91FF90EF90DF90CF90DD
:1067C000BF90AF909F908F900895C0914F5480914B
:1067D0004D54611105C00E944B33C82F0E944B33AA
:1067E000C11106C090B19B3008F05D98589A0EC058
:1067F000C630E0F3C332D1F3C632C1F394EF9C0F3D
:106800009230A0F398EE9C0F953080F3CE30A0F438
:106810001092144C1092154C1092164C1092174C6A
:106820005A9AEC2FF0E0CC3028F0CC50EC2FF0E06E
:10683000EC50FC4C8083ADCFC432B8F3599AF5CFFD
:10684000611591F080914F54909150548093103481
:106850009093113480914D5490914E548093123402
:1068600090931334599A95CFC0E1D4E38E012196C9
:106870000E944B33F8018083F4E3C431DF07B1F7A2
:10688000F1CFAA980E943D4D84CFAA9840E051E0F4
:1068900060E879E08FED90E20E94947B7ACF589A7D
:1068A0005C9A77CF589A5C9874CF589A5D9A71CF5A
:1068B000589A0E948F476DCF611561F080914D54B9
:1068C0008093FE3380914E548093FF330E94414960
:1068D000589A5FCF0E944B338093FE330E944B3314
:1068E000F3CF589A5A9ABECF8091144C9091154C80
:1068F000A091164CB091174C80938B5490938C546C
:10690000A0938D54B0938E5452CF679842CF679A1C
:1069100040CFEBE8F4E580E090E0DC0101962C91BB
:1069200021938C309105C9F780E2E4EFF3E3A7E906
:10693000B4E501900D928A95E1F78CE239CFC0E081
:106940008C2F90E08058964F0E94FC7B0E945C3315
:10695000CF5FB1F71ECF87E40E945C33CFEDD0E26A
:106960001C2F7E0121960E944B33F70180831C135C
:10697000F8CF599A84E50E945C330BCF81E00E94E6
:106980005C3381E00E945C338EEF0E945C330BE14C
:1069900012E239E5E32E32E2F32EC0E0D0E0F80156
:1069A0008491D8279C2F2D2FCD2FD295CD27C07F16
:1069B000DF709C272D27CC0FDD1FD927C2270E940F
:1069C0005C330F5F1F4FE016F10649F780EFE82EAA
:1069D00083E0F82E9EE3B92E992493942FE3A22E00
:1069E0006701E0E8CE228A2D87708824839401C055
:1069F000880C8A95EAF700E010E0E091E321F0913D
:106A0000E421EC0DFD1DE00FF11F80E098E0880F00
:106A10002191282131E0211130E0832B9150B9F7E9
:106A2000D8279C2F2D2FCD2FD295CD27C07FDF705B
:106A30009C272D27CC0FDD1FD927C2270E945C334E
:106A4000B394F0E8BF1219C08D2F0E945C338C2FD5
:106A50000E945C330E944B33863009F09ACE9394A7
:106A600081E00E945C33892D0E945C33892D8095E2
:106A70000E945C33B12CC0E0D0E0085F1F4F0038AB
:106A8000110509F0BACFAA94F0E1EF1AF1088FEFDF
:106A9000A812A6CF1AE1B7FE19C08D2F0E945C3351
:106AA0008C2F0E945C330E944B33863009F071CEEC
:106AB00084E00E945C330E944B33853109F069CE3B
:106AC00084E00E945C330E944B3363CED1278C2F2D
:106AD0009D2FCD2FD295CD27C07FDF708C279D278E
:106AE000CC0FDD1FD827C9278AE10E945C33B394FD
:106AF000D2CF6115B1F010922A2010922B208091F4
:106B000028208D7980932820809120208D7C80936F
:106B100020208091202085FD04C08091282085FFC1
:106B2000F8CFF8948AE00E94D43E8091C1048E7F11
:106B30008093C10484E60E94D43E8AEA95E580935E
:106B4000D4329093D5328FEF8093780061E089E75B
:106B500090E00E94BA791DCE8F929F92AF92BF9221
:106B6000CF92DF92EF92FF920F931F93CF93DF9319
:106B70000091F733C091F833359902C0CFE700E0B8
:106B8000DC2FDD0FDD0BC01BD10907FDD395F3E032
:106B9000CC0FDD1FFA95E1F780B18B3018F0CC0FE8
:106BA000DD1F000FF0900734F694F694F694102F42
:106BB00000E068E0C62ED12C70E8E72EA12C902EC4
:106BC000812E80B18B3098F52091F633922F802F53
:106BD000910F24B12E21C9F08C0F9D1F21E0322F7F
:106BE000337041F5BB0CA11411F0B394A12C8C0FA0
:106BF0009D1F2F5F213299F788E78093E021F09263
:106C0000DF218B2D0E944E2DF394E69421E0C21AD1
:106C1000D108B9F6DF91CF911F910F91FF90EF90BE
:106C2000DF90CF90BF90AF909F908F900895892D67
:106C3000982DCFCFE92FF0E0EA5CFC4A30813E216D
:106C4000B1F2A394D4CF809110018064809310019D
:106C5000809120018064809320018091A10887FDAC
:106C600043C08091C20881118091C30885E8809358
:106C7000120180E095E0809314019093150184E166
:106C800094E380931C0190931D018091083482301D
:106C900071F1811581F120E080E090E020931301F3
:106CA000909318018093190184E8379B84EA8093BC
:106CB000100185E88093220180E095E08093240113
:106CC0009093250184E199E380932C0190932D0109
:106CD0008EE19EE3809328019093290184E8379BFD
:106CE00084EA8093200108958091A008B6CF2BE418
:106CF00088E090EAD3CF2AE488E093ECCFCFDF920C
:106D0000EF92FF920F931F93CF93DF93D82E8111B1
:106D10003AC00091153E1091163E80E094E1E92EB4
:106D200094E3F92E8093E0211092DF21C0E51F9BB0
:106D300002C06695C0EA2C2F30E0C69FE001112406
:106D40002C9B15C0C8010217130738F1821B930B47
:106D500070E06F5F7F4F629FE001639FD00D729F75
:106D6000D00D1124C80FD91FD53008F0D55080910F
:106D7000DF218031A0F0DF91CF911F910F91FF9023
:106D8000EF90DF9008950091173E1091183E84E136
:106D9000E82E89E3F82E87E4C5CF9B5FD7CF2C99E7
:106DA00003C0C017D10738F7F701EC0FFD1F808132
:106DB0002196D53010F0C0E0D0E01F9B20C08A3073
:106DC000B1F484E10E94C42C8091E0218E5F809315
:106DD000E0218091E021D11018C08B3340F28091E6
:106DE000DF211092E0218F5F8093DF21C0CF8D30B3
:106DF00011F485E1E7CF803228F78FE5E3CF0E94D9
:106E00004E2D80E20E94C42CE4CF873408F0AFCF2F
:106E100087E48093E021ABCF8F929F92AF92BF9295
:106E2000CF92DF92EF92FF920F931F93CF93DF9356
:106E30000E94A63B0E94492CE4E1F4E382E09AE040
:106E4000DF019C011D9221503040E1F71092153E68
:106E50001092163E1092173E1092183E85B184FB98
:106E6000FF24F4F884FF02C0CFE0FC2E10927300E0
:106E700080910834813009F0F6C088EA92E20E94DD
:106E80004A3184E19CE380931A3E90931B3E84E157
:106E900094E380931C3E90931D3E80E880931E3EB9
:106EA00080915006887F82608093500683E08093B3
:106EB0004C0680934906C0E00E9423360E946B3B3B
:106EC0000E94A63B20E035E0C05C53E06CE080917E
:106ED000153E9091163E892B39F48091173E909182
:106EE000183E892B09F41CC140E1D42E00E015E0C6
:106EF0006EE3862E6BE3962E71E4C72E0E94492C1A
:106F0000A9988091382085FF1AC010923E201092D7
:106F10003F20649957C124E134E320933C2030930F
:106F20003D2080E892E080933A2090933B2080912E
:106F300038208D79809338208CB18D258CB9809143
:106F40000834813009F064C12C9B50C18091153EFA
:106F50009091163E8038910508F441C18091153E0C
:106F60009091163E80589109CF2DD0E02196D6956C
:106F7000DC2FCC27D795C795C80FD91FD83008F07C
:106F8000D85090E8B92E2C9907C08091153E909169
:106F9000163EC817D90788F5FE01EC5EFB4CA080B1
:106FA000FE01F695E795F695E795EC5EF34C80814A
:106FB0009C2F9370990F21E0290FE82E01C0EE0C51
:106FC0002A95EAF701C0880F9A95EAF787FF18C15A
:106FD0008A2D86950E944E2DA0FE0DC18CE3E7FE02
:106FE00088E20E94C42C80E20E94C42C2196D830F2
:106FF00010F0C0E0D0E0BA9431F60E94A63B0E94A7
:107000006B3B0E94332C669B2BC066987A9B05C015
:10701000799B03C083B1805883B97B9B12C08BB12D
:107020008D258BB9809108345C9B71C11092A408A6
:107030009091C0089F7B9093C008813011F410920A
:1070400049067A9B05C081E0F11001C080E0F81A82
:10705000799B04C02FE0F21608F4F3947D995B98B5
:107060005B994CCF84C0823009F044C08BE892E237
:107070000E944A318AB1877090E0FC01E252FD4DD6
:10708000E491E093A608FC01EA52FD4DE491E093FF
:10709000A7082AB1269526952695237035E0320F4C
:1070A0003093193E559B03C0569B22C020635799CD
:1070B00028602093A50820E12093A40821E02093D4
:1070C0004008FC01EE0FFF1FEA53FD4D859195919D
:1070D00080931F3E9093203E969587959695879531
:1070E000809366089093670883E080934608E3CE18
:1070F0002062DDCF8111DFCE89E592E20E944A3124
:1071000081E0569981E4CC275799C395CC0FCC0FD9
:1071100080935706559BD0CE80E480935406CCCE06
:10712000A89540910834413001F18091140190916B
:107130001501D901A81BB90BA093153EB093163EBB
:107140008091240190912501F901E81BF90BE0934E
:10715000173EF093183E411108C0D49B06C0C0935F
:10716000C00850934C06609349065B9927C01FB82E
:1071700086E391E580933C2090933D2082E28093CA
:10718000382064981092A3081092A4081092460820
:1071900010924008109249061092C0088CE7809324
:1071A0007300DF91CF911F910F91FF90EF90DF90CF
:1071B000CF90BF90AF909F908F9008957D9B87CE8A
:1071C0005B9885CEA4E9B6E3A0933C20B0933D2024
:1071D000E9E8F2E0E0933A20F0933B20A8CE8091DA
:1071E000153E9091163E8058984FBECE20E8F29EF4
:1071F000E0011124C6CE8EE3E7FCF3CE89E2F1CEA6
:107200008A2D0E944E2D8BE2E7FCEBCE8DE2E9CE7B
:107210008091140190911501D801A81BB90BA0937E
:10722000153EB093163E8091240190912501F801FE
:10723000E81BF90BE093173EF093183E379B18C0FC
:107240008091100187FD0BC010921401109215015E
:107250001092A4088091C0088F7B8093C008809111
:10726000200187FD05C010922401109225015C9A2F
:107270005C9B3CC02EE14FE368E08FE30E94E9197C
:10728000CCEEDEE28CE0E82E8092E021E092DF217D
:10729000FE0184910E94C42CE3942196F0E1EF1248
:1072A000F3CF8F2D1F998E7F8092E0211092DF21E6
:1072B0000E94E4790E94C42C809108349092E021CD
:1072C00081111BC081E08093DF2189E40E94C42CDE
:1072D000C092E0218FE40E94C42C6F2D80E00E94B8
:1072E0007F366F2D81E00E947F3687CE2FE74FE3F8
:1072F00068E08FE30E94E919D4CF81E08093DF2119
:1073000082E50E94C42CC092E02184E5E4CF813064
:1073100041F483E080934906379B93CE0E94233645
:1073200090CE823019F4D092A408F6CF8111F4CF18
:107330008091C00880648093C008EECF1F921FB672
:107340001F9211242F932BB72F933F934F935F934B
:107350006F937F938F939F93AF93BF93EF93FF931D
:1073600080911C3E90911D3EE0911A3EF0911B3E93
:1073700030911E3E28E12093200820910C082160C6
:1073800020930C08A99A40E021E0D19B0CC02091E9
:107390000C0820FFF8CFAC014451544311C0609158
:1073A0000C0860FDF8CFD19BFACF68E384319607D3
:1073B00051F5379B61C0109249065C9A40E058E055
:1073C0004093153E5093163E80931C3E90931D3E75
:1073D000E0931A3EF0931B3E30931E3E81E0809373
:1073E0004C06FF91EF91BF91AF919F918F917F914B
:1073F0006F915F914F913F912F912BBF2F911F90D4
:107400001FBE1F9018957AB3672F617070FD25C05D
:1074100070910C0870FDBFCFD19B04C0D09BF8CFFA
:10742000D199B9CF483021F5DC015D93CD0121958B
:1074300023234081242B611103C0432F4695242B25
:1074400036953695208320E040E03111ACCF118293
:10745000319620E040E030E8A6CF70910C0870FD36
:107460009ACFD19BDFCFD099F8CFD19BDBCF8BCFF9
:10747000550F562B4F5F97CF1092143CE4E1FCE37D
:1074800084E194E390CF2F932FB72F938F939F9303
:1074900092E09093200890910C08916090930C08D2
:1074A00098E0579914C0D79B2DC0880FD69981605A
:1074B000D7992DC09150B9F713C020910C0820FF27
:1074C00006C09F918F912F912FBF2F911895D79B19
:1074D000F4CFD79912C0880FD69981609150B9F72F
:1074E00080931E3E82E080934C065C99EACF8091A7
:1074F0002001806180932001E4CF20910C0820FFBF
:10750000E8CFDFCF20910C0820FFCDCFDACF20913C
:107510000C0820FFCDCFD5CF1F921FB61F9211248C
:107520002F933F934F935F936F938F939F939AB350
:10753000892F887093FD58C091E090934C089091EA
:107540004C0890FFFCCF20911F3E3091203E2093AD
:1075500066083093670890E050E061E04091193E82
:107560005417C8F0483020F1559925C091E0909308
:107570004C0890914C0890FFFCCFD39B2AC05799A0
:1075800043C080931E3E5C9924C08091200180619D
:10759000809320011EC060934C0840914C0840FF2E
:1075A000FCCF8695D39B02C080689F5F5F5FD6CF7C
:1075B00086954F5FD7CF41E040934C0840914C08EF
:1075C00040FFFCCF9170569B1AC09115D1F0D39B10
:1075D000CDCF36952795369527952093660830931D
:1075E000670881E080934C089F918F916F915F9124
:1075F0004F913F912F911F901FBE1F90189591158D
:1076000031F3D399B3CFE5CF91E090934C089091AB
:107610004C0890FFFCCFD399B4CFDBCF1F93CF930F
:10762000DF9300D00F92CDB7DEB780E88093E521DD
:107630008093E6218093E72A8093E82A2AEF3AE2B2
:107640002B833C8310E08B819C8183519940EB819B
:10765000FC817197E983FA8341E150E06FEF70E0BC
:107660000E948D7B41E150E06FEF70E089819A814B
:107670000E948D7B812F86958F5F8575912F990F45
:107680009C5F9A7A892B982F990F990F9C7C8695ED
:1076900086958373892B8295EB81FC81E250F940BA
:1076A0008083EB81FC8180831F5F7296EB83FC8378
:1076B000103849F62496CDBFDEBFDF91CF911F91E0
:1076C0000895E0EAF9E0168280EC858388E08483FF
:1076D000EA9A0C940E3BE89AE0E0F1E080A980641D
:1076E00080AB80E48A95F1F780E182AB82E099E09B
:1076F00084AB95AB80EA84AF89E085AF8CE683AB41
:107700009091E1218091E22190AF81AF84E880AB3C
:10771000E0EAF9E080EC818384E0838308951F929E
:107720001FB61F9211248F9385E18A95F1F700000F
:10773000E8981092A3098AE08A95F1F700C0A99809
:10774000AA988F911F901FBE1F901895A89580E250
:107750009EE4E89B06C02AE02A95F1F700C0019755
:10776000C1F708951F921FB61F9211248F93809125
:1077700006088B7F809306088FB18111609A8F91E4
:107780001F901FBE1F9018951F921FB61F921124A5
:107790008F93109200091092060980917400816005
:1077A000809374008FB18111609A8F911F901FBEDA
:1077B0001F901895AAECB1E092E09C93E82FF0E0BE
:1077C00084911C9208958BEC80935200809150001C
:1077D00089608093500082EC8093550080E0909106
:1077E000510093FD08C0EFE8F1E03197F1F700C0D8
:1077F00000008F5FA1F79091510093FF109252000B
:1078000099E1909350009091510094FD08C0EFE8E9
:10781000F1E03197F1F700C000008F5FA1F764E05D
:1078200080E490E00E94BA7988E1809350008091D2
:10783000400080FF06C04CEF52E267E080E00E940B
:10784000A92E8EE08093A6098CE08093CC018FE86E
:10785000809386010895809150008160809350004C
:1078600080E09091510090FD08C0EFE8F1E0319781
:10787000F1F700C000008150A1F760E080E490E0E3
:107880000E94BA7991E01092520010925500EFE8F0
:10789000F1E03197F1F700C0000090935000809123
:1078A0005000813081F71092A6098EE08093CC01C0
:1078B0008DE88093860108958E9A82E08093050674
:1078C000E0E7F0E088E18083118281E082838CE749
:1078D00083839CE6948385830C94E33BCF93DF936F
:1078E0000E94613B61E080E890E00E94BA7997E0F5
:1078F000909348008E98A6E0B6E082E08C93E0E09A
:10790000F8E010828FE08187E0E410828187E0E078
:10791000F9E010828187E0E410828187E0E0FAE0FC
:1079200010828187E0E410828187C0E0D1E0188274
:1079300080E488831092000210924002E0E8F1E0B7
:10794000108211821282138288E08483158217824A
:10795000E0E7F0E088E58083918392838FEF838373
:107960009FEE948385838EEF868384E28C930E94BE
:107970002B3C80E88883DF91CF91089598E5909320
:107980007000C7E0C0937100C09372008FEF8093C6
:1079900073002FEE20937400809375002EEF2093D8
:1079A00076002CE0F22EF092CC012EE2209300061D
:1079B000C0931406C0931606C093170623EC2093B9
:1079C0002006D1E0D0933206C0933306C09334062C
:1079D000C093350600E800932406D0934A0600932E
:1079E0004B061FE31093600620E220936406109379
:1079F0008006D0938E0620E4209394068093B000F6
:107A00009093B00632E0E32EE092A9068093AA0696
:107A100081E48093B20082E38093B3000E946E3CC5
:107A20000E94332C0E94492C0093000183E0809334
:107A300043008FEF91E080930A0490930B0490E051
:107A400080930C0490930D04E092000485E08093F1
:107A500002048FEB98EA8093260B9093270BF09209
:107A6000000BD093060B47E050E06AE17DE080E038
:107A700090E00E94F07B89E19DE00E94FC7B8DB943
:107A80000E943C74C093A2008091200B9091210B26
:107A90000E94EC790E94B3291093780066980E94A6
:107AA000A37411E044E0D42EF12E0E946E3C669B3C
:107AB0001EC066987E9902C0789B03C08EB18F5F0E
:107AC0008EB97F9902C07C9B03C08EB181508EB964
:107AD0008EB1833009F405C108F05EC0813009F42D
:107AE00069C0823009F473C088E789B9589A589BF5
:107AF00044C00E94E33B87EE92E30E94507A8EB12D
:107B00000BE9C1E0D5E7811749F08EB105E8C1EF77
:107B1000D1EF181718F00BE9CFE0DFE085E78D0F04
:107B20008B3E08F4EDC01EB18CE18093E021E09221
:107B3000DF212EB12150330B41E1429FC001439F11
:107B4000900D11248457914D0E944A31F092E0210A
:107B50008FE08093DF212EB12150330B46E1429F0D
:107B6000C001439F900D11248C5C914D0E944A31BD
:107B70000E94A63B0E946B3B589889B1811509F47D
:107B800010C10E94A63B8091400981118ECF89B11E
:107B9000815089B9889589CF843009F0A5CF7B9928
:107BA0000E948E2B7A990E94642879990E94B329A9
:107BB000DEB89ACF7B9B03C00E94A37411E07A9930
:107BC0000E94F375799B90CF0E94EB418DCF7B99FA
:107BD0000E94C12A7A990E94542B799B80C00E94EE
:107BE0005C3C0E94547847E050E06AE17DE080E030
:107BF00090E00E94947B109202041092070B109266
:107C0000060980E18093010980E880932909C091E9
:107C1000200BD091210B0E94674D1092C10410924D
:107C2000C3041092C004809150008D7F8093500057
:107C300047E050E06AE17DE080E090E00E94F07B68
:107C400082B18C3030F168948091200B9091210B9F
:107C50008C179D07F0F4E89486B18F5F86B986B1E2
:107C6000873008F016B883B18F5F83B9C3B180E065
:107C700090E00E94A8738C1760F491E093B984B1EE
:107C80008F5F84B984B18D3020F094B985B18F5F56
:107C900085B90E94686A1CB81BB889E19DE00E9402
:107CA000FC7B8DB9109201091092290910920302F0
:107CB00010924302809110018064809310018091A2
:107CC0003001806480933001809120018064809332
:107CD00020010E94866A85E080930204589AEEB8DB
:107CE00003CF7B990E94D6697A990E94F465799BAB
:107CF00004C00E94E33B0E94412683E08EB9F4CE8B
:107D0000669B1AC0669887EE92E30E94507A1EB175
:107D10007E9902C0789B06C08EB18F5F8EB905E850
:107D2000C1EFD1EF7F9902C07C9B06C08EB181501C
:107D30008EB90BE9CFE0DFE08EB1853008F0FEB8F8
:107D40008EB1811101C0DEB8C2303CF1C1500E9439
:107D5000332C0E94492CEEB1F0E0EE0FFF1FE551ED
:107D6000F84F4591559120E064E0802F8D0F0E94DF
:107D70009F32E12FF0E0EE0FFF1FE551F84F4591E4
:107D8000559120E064E080E18D0F0E949F320E94B7
:107D9000A63B0E946B3BDC0FC1CECF3FC4F6CF5F4A
:107DA000D6CF0E94A37481CEA895811101C00895F9
:107DB000815090914000911107C0EFEEF1E03197B2
:107DC000F1F700C00000F1CFE7E3FFE13197F1F7F1
:107DD000F8CF1F920F920FB60F9211240BB60F928D
:107DE0002F933F934F935F936F937F938F939F93C3
:107DF000AF93BF93CF93DF93EF93FF93A998AA9884
:107E0000C0E1D0E081E00E94D43E8091A8068D13AD
:107E100046C0C15009F044C0DFB97F9B10C07E9BB3
:107E20000EC07D9B0CC047E050E06AE17DE080E041
:107E300090E00E94947B60E08BEB0E94A6338FB1B0
:107E4000811509F446C0589A669A80917100811193
:107E500029C0809100088F3069F484E18093210863
:107E600080910C08826080930C08809106088460E1
:107E700080930608FF91EF91DF91CF91BF91AF9171
:107E80009F918F917F916F915F914F913F912F9132
:107E90000F900BBE0F900FBE0F901F901895C9E06A
:107EA000D82FB0CF809174008E7F80937400109291
:107EB00000098FE08093090984EF90E08093260900
:107EC0009093270981E0809306098EE08093000952
:107ED000D1CF80917100811108C0809106088B7FFD
:107EE000809306086098A898C5CF10920009109258
:107EF000060980917400816080937400F3CF0E9422
:107F0000714980E40E94D43E0E94AA4C80E10E9404
:107F1000D43E84E18093010280934102E0E0F1E0ED
:107F200080898F77808B80A98F7780AB80A18F77B6
:107F300080A308959F92AF92BF92CF92DF92EF926B
:107F4000FF920F931F93CF93DF931FB80E94492C8A
:107F500089EE92E20E944A318CE68093E0218FE024
:107F60008093DF2186EE92E20E944A310E946B3BB1
:107F70000E94A63B8FB18115E9F30E945C3C799B7E
:107F800045C00E94492C1092070B10B8B12C84E117
:107F900094E3A82E97E0992E80B1883008F444C06D
:107FA00090E19093010287E0809304029093410254
:107FB00080934402F12CC0E0D0E08E0183E8E82EEB
:107FC000E0922002E092600281E00E94D43E809123
:107FD000240290912502080F191F8091640290914C
:107FE0006502C80FD91FFA9459F7B80180E09BE0E9
:107FF0000E94347CBE018EEF9AE00E94347C60E0E7
:1080000082E09BE00E94117C0E94866A1FB8DF918B
:10801000CF911F910F91FF90EF90DF90CF90BF9085
:10802000AF909F900C946E3C1B2DC6E0D0E0012FCA
:108030001F5FC093F433C093F5330E947F3F84E108
:1080400094E3E12CF12C6701FC0101962081C20E22
:10805000D11C27FDDA94F85F2081E20EF11C27FD88
:10806000FA94A812F1CFA99A80B19E01989E200D92
:10807000311D1124C9016D2D8C53954F0E94117C27
:1080800080E28D0D803460F520E62D0D412F60E6F5
:10809000812F0E94E91980B19E01989E200D311D0B
:1080A0001124C9016F2D8457954F0E94117C80E2E5
:1080B0008F0D8034B8F481E4800F20E62F0D482F17
:1080C00060E60E94E9190E946B3B0E94A63B219743
:1080D00008F0ADCF87E0B80E80B18F5F80B95CCF7C
:1080E000AA9AD9CFAA9AEFCFA895811569F08150A5
:1080F00090914000911109C0EFEEF1E03197F1F756
:1081000000C00000669BF1CF0895E7E3FFE13197DF
:10811000F1F7F6CFCF93C82FAB9A809171008D7F86
:108120008093710081E08093000280E780930102D8
:1081300080E48093020284E380932102109204027F
:1081400080E1A0E0B0E04FE991E04093200220916F
:1081500006022115E1F3909306022091100230915E
:108160001102A20FB31F815081F7AB9827E731E0CE
:108170000E94567B472F582F692FE3E0659557954E
:108180004795EA95D9F7CA01109202022091710031
:10819000226020937100C1112EC04F3F20E1520791
:1081A000ACF5473620E15207A4F582E093E220E0E7
:1081B00030E0FC01A591B5914A175B0708F581E015
:1081C00090E02115C1F0F901EE0FFF1FE050FD4DC9
:1081D00085919591481BA81BB90BB695A795B695A7
:1081E000A795A41750F0220F331F220F331F2C0F17
:1081F000311DC9010397CF9108954A1BCF5FF1CF7D
:108200002F5F3F4F02962C30310599F680E090E0C9
:10821000F2CF8DE290E0EFCF0F931F93CF93DF93D8
:10822000809171008D7F8093710081E080930002C6
:1082300080E78093010280E4809302028FEF8093B5
:10824000060288E3809321028091400081113DC0A5
:108250001092040210E1C0E0D0E001E081E88093D8
:108260002002809106028115E1F3009306028091BD
:10827000100290911102C80FD91F809110029091A5
:1082800011020E94EC7981E00E94D43E115031F736
:10829000109202028091710082608093710027E742
:1082A00031E0DE010E94567BBB2797FDBA95A92FCE
:1082B000982F872F24E0A595979587952A95D9F72C
:1082C000DF91CF911F910F91089584E08093040274
:1082D000C1CF0F931F93CF93DF93809171008D7F58
:1082E0008093710081E08093000280E1809301021D
:1082F00080E48093020288E38093210281E00E945F
:10830000D43E8FEF8093060280914000811132C0ED
:1083100082E08093040210E1C0E0D0E001E081E857
:1083200080932002809106028115E1F300930602FA
:108330008091100290911102C80FD91F81E00E9414
:10834000D43E115061F71092020280917100826058
:10835000809371009E01DD0F440B542F60E070E0AC
:1083600080E094E00E942F7BC901DF91CF911F91A3
:108370000F91089587E0CDCFCF93DF9300D000D049
:108380000F92CDB7DEB729E12C8321E02D831E8229
:10839000BE016F5F7F4F0E944A77DC0190E080E072
:1083A000853D27E892072DE1A207B10578F4892FD2
:1083B0009A2FAB2F25E0A695979587952A95D9F703
:1083C0002796CDBFDEBFDF91CF910895845D97489A
:1083D000AD41B109E5CF2F923F924F925F926F92DC
:1083E0007F928F929F92AF92BF92CF92DF92EF9245
:1083F000FF920F931F93CF93DF93CDB7DEB76697AE
:10840000CDBFDEBF83B18C8384B18D8385B18E8374
:10841000639A5E98DD24DA94712C4E012FEF821A54
:10842000920A669B4AC0C4010E94BC416698F82C1F
:10843000092D7D995E9A7E9902C07F9B04C08F2D85
:10844000902F0E947377789902C07C9B04C08F2D77
:10845000902F0E9490777B9B11C010E08F2D902F62
:108460000E949077E12E8F2D902F0E94BC41182FF3
:1084700037E7E31698F3873788F7712C7A9B06C0A5
:1084800083B18C8384B18D8385B18E83DD24DA94AE
:10849000799B13C01FEF8F2D902F0E947377E12ED1
:1084A0008F2D902F0E94BC41182F86E7E81698F771
:1084B000163788F3DD24DA94712C8C81871509F442
:1084C000C5C00E94492C7C80C4010E94BC41182F69
:1084D00092E29093E0211092DF218AE193E20E94E0
:1084E0004A31A40161E082E20E94B8771730A8F017
:1084F00081E0143398F082E0123480F083E01F367C
:1085000068F084E01D3750F085E01A3A38F086E0D4
:10851000183B20F087E0153E08F080E0E8E1E093AA
:10852000E0219DE09093DF21F0E18F9FC0011124B5
:10853000825B934D0E944A311092E0218FE080933C
:10854000DF2188ED9CE20E944A310E946B3B409003
:10855000E3215090E4212CEB421A26E0520A30EE3F
:10856000E32E3FEFF32E46EA242E44E0342E36E786
:10857000311B3E8BEE9C9001EF9C300D300D112491
:10858000298B3A8B29863A86488A652C188602C040
:10859000E88B6F2EE985FA858491F885F052FB8B84
:1085A000A12CB12CC12C8C8B1D8A80E890E00A2C68
:1085B00002C0959587950A94E2F78B879C878C89F2
:1085C0009D89EB85FC858E239F23892B99F08B89D0
:1085D0008A0D8802900111242D873E8789899A8906
:1085E000820F931F813094402CF4163709F04EC04F
:1085F0008B85C82A3FEFA31AB30A88E0A816B104F6
:10860000A1F6E889F62DC094C19229853A852F5F9D
:108610003F4F29873A873885385F3887303409F0EB
:10862000B7CF88E0280E311C92E1490E511CE89B1F
:108630000E946B3BEFEFEE1AFE0AF0E2EF16F10438
:1086400009F098CF0E94A63B0E946B3B0E94A63B7C
:108650008895D11419F0DA945E9BE3CE6698589A07
:108660006696CDBFDEBFDF91CF911F910F91FF9036
:10867000EF90DF90CF90BF90AF909F908F907F90C2
:108680006F905F904F903F902F900895111509F4CF
:10869000B1CF163780F58E891F8660E28695869564
:1086A0000E94407A082F8115C9F08802A001112488
:1086B0009A01AD85BE850E94567B672F782F892F42
:1086C000869577956795869577956795CA01861BF8
:1086D000970B0E94541A10169CF4082FEF85E11591
:1086E00091F0202F332721950CF43095E216F306F4
:1086F0000CF07ECF7FCF8AE8810F91E09F87CDCFAE
:10870000082F0195EBCF0E15F3CFAF92BF92CF920A
:10871000DF92EF92FF921F93CF93DF9380B1C6EF6A
:10872000DEE2873010F0C7EFDEE211E0612F8091CA
:10873000F7330E94BD1962E0610F8091F8330E9407
:10874000BD191C5F113891F7E090F733F090F833C2
:108750001E2D1F19EF1410F41F2D1E19479B4AC020
:10876000E0B184E0E89FF0011124EE5EF44DA590A5
:10877000B590C590D590AB2CBC2CCD2CD12C449B66
:1087800004C08091F633E81AF81A45ED5EE260E025
:1087900080E00E94A92EAE2DEE0CBB0B9501A60128
:1087A0000E94687B9B01AC0160E080E10E945D2D2E
:1087B000CE010E94222D40ED5EE261E080E00E9449
:1087C000A92EAF2DFF0CBB0B9501A6010E94687B63
:1087D0009B01AC0161E080E10E945D2DCE01DF9143
:1087E000CF911F91FF90EF90DF90CF90BF90AF900F
:1087F0000C94222D4EEF5EE26CE080E40E94A92EE4
:10880000C12ED12CE12CF12C1115E9F0E0B184E05E
:10881000E89FF0011124EE5EF44D6591759185910C
:1088200095919601A7010E940D7B80B18B3020F0BD
:1088300056954795379527956CE088E50E945D2D04
:10884000CE010E94222D41E05FE26DE08CE40E94A7
:10885000A92EE0B1F0E0EE0FFF1FEA51F54D259192
:108860003591D6010E94567B9B01AC01AAEF0E9474
:108870005D7B9B01AC016DE088E50E945D2D80B1C0
:10888000873078F487E10E94C42C83E5DF91CF9193
:108890001F91FF90EF90DF90CF90BF90AF900C941E
:1088A000C42C80B1803188F78AE10E94C42C8BE10E
:1088B000EACF8F929F92AF92BF92CF92DF92EF92C8
:1088C000FF920F931F93CF93DF9300D00F92CDB7FA
:1088D000DEB7479918C1339B91C02091F4332C83A4
:1088E00081B02091F9333091FA3339838091053486
:1088F000EDE3F4E566E371E5329B90C04091F63319
:108900009091F733460F572F511DFA01E90FF11DD2
:1089100020819091F833490F511DFA01F081F983BC
:10892000122F1695469B85C050E8D52ED11A8091FE
:10893000F633E981E81BFF0BBF0175956795F62EAD
:1089400001E0602F8D2D0E94BD19FFE7FF1628F46E
:108950006F2D82E0800F0E94BD190C5F013889F7EE
:10896000298126952B8388B186FB992496F8198353
:108970001A8220E430E06901C11AD108FB81AF2ED0
:1089800086FF80C045E253E26DE08EE40E94A92E8E
:1089900041B16091F43380E09C2D0E948A2E809139
:1089A000F433843008F468C087EE9EE20E94222DE2
:1089B0004DE95AE26EE08EE40E94A92E42B1609128
:1089C000F53380E090E49A190E948A2E8091F53365
:1089D000843008F454C087EE9EE22496CDBFDEBFFB
:1089E000DF91CF911F910F91FF90EF90DF90CF908B
:1089F000BF90AF909F908F900C94222D8091F53373
:108A00008C8382B02091FB339091FC3399838091C9
:108A10000634E8E3F4E566E372E56ECF319905C00C
:108A2000220F3981330F39837BCF21819281998342
:108A300077CF982F990F990BBC01620F711D759517
:108A40006795E62E2981820F911D95958795F82EC1
:108A500001E03FE7E31620F46E2D802F0E94BD1940
:108A60008FE7F81628F46F2D82E0800F0E94BD1961
:108A70000C5F013871F774CF84EE9EE297CF84EEDD
:108A80009EE2ABCF9B8180E0191708F08EE0EC816D
:108A900027EEE22E2EE2F22EE43020F494EEE92EC0
:108AA0009EE2F92E98E09093E0218093DF21482DFB
:108AB0006C8180E09C2D0E948A2EC7010E94222D8D
:108AC000FB811F1710F48EE0982E88E08093E02140
:108AD0009092DF21482D6C8180E090E49A190E94E9
:108AE0008A2EC7010E94222D4AEF5EE26EE08CE4DE
:108AF0000E94A92E482D6C8180E099819A190E94CC
:108B00008A2EC7016ACF2496CDBFDEBFDF91CF91F9
:108B10001F910F91FF90EF90DF90CF90BF90AF909B
:108B20009F908F9008956F927F928F929F92AF92B5
:108B3000BF92CF92DF92EF92FF920F931F93CF934A
:108B4000DF93629A1092E02182E08093DF215E9BA6
:108B5000A5C05F99A3C08BB1482F407184FD78C038
:108B600010910102C091410200910402D09144028F
:108B7000709020026090600290E19093010287E083
:108B8000809304029093410280934402E12CF12CE3
:108B900067014601560153E850932002509360024A
:108BA0008FE79CE00197F1F700C0000020912402BC
:108BB000309125028091640290916502589948C0D5
:108BC000032E000C0008821A930AA008B008092E90
:108BD000000C0008C81AD90AE008F0084150E1F674
:108BE00080E09BE00E940C7C092E000C0008880E9F
:108BF000991EA01CB01C8EEF9AE00E940C7C65E0D0
:108C0000B594A794979487946A95D1F78092144C61
:108C10009092154C092E000C0008C80ED91EE01CBD
:108C2000F01C75E0F594E794D794C7947A95D1F742
:108C3000C092164CD092174C609260027092200243
:108C40000093040210930102D0934402C0934102A6
:108C500041B160E08091144C9091154C0E948A2E95
:108C600080E48093E02182E08093DF2142B160E0E4
:108C70008091164C9091174C0E948A2E6298DF9139
:108C8000CF911F910F91FF90EF90DF90CF90BF9009
:108C9000AF909F908F907F906F9008955F9B1DC0C5
:108CA0005E991BC041B1809140546091F43320E83B
:108CB000829FC00111240E948A2E80E48093E021CB
:108CC00082E08093DF2142B180913B546091F53383
:108CD00020E8829FC0011124CFCF5E99CAC0809145
:108CE00003088C3381F1109232511092335110925B
:108CF00034511092355110922E5110922F511092E2
:108D0000305110923151109200089FE09093090861
:108D100080E1809301082CE3209303082DE0209349
:108D2000000824EF35E0209326083093270810929E
:108D3000000A9093090A8093010A8CE28093030A47
:108D40008AE08093000AC0902E51D0902F51E0907D
:108D50003051F09031518091325190913351A09126
:108D60003451B0913551C81AD90AEA0AFB0A8091E8
:108D7000030481FF3CC05E9922C080912E519091E6
:108D80002F51A0913051B091315180933251909335
:108D90003351A0933451B09335518091280890916C
:108DA00029082091280A3091290ADC01C901209361
:108DB0002E5190932F51A0933051B09331518FEF9A
:108DC000809303045C9905C080912B518F5F809341
:108DD0002B5180912B518C3350F010922B5180915C
:108DE0002C518F5F8C3308F079C080932C515E99A1
:108DF0007DC0E0B184E0E89FF0011124EE5EF44D07
:108E000085909590A590B590892C9A2CAB2CB12C7F
:108E1000A0914154B0E09401A5010E945D7B9B01AB
:108E2000AC0162E080E00E945D2DA0913C54B0E076
:108E30009401A5010E945D7B9B01AC0162E080E48E
:108E40000E945D2D619A9601A70165E088E00E946D
:108E50005D2DC092144CD092154CE092164CF092BD
:108E6000174C61985E990ACF87E0809348545A9ACC
:108E700005CF809103088F3331F110922D5110925C
:108E80002C5110922B51109200089FE090930908EA
:108E900080E1809301082FE3209303082DE02093C5
:108EA000000824EF35E0209326083093270810921D
:108EB000000A9093090A8093010A8FE28093030AC3
:108EC0008AE08093000AC0902808D0902908760193
:108ED0008091280A9091290A6C0149CF10922C5157
:108EE00080912D518F5F80932D5181CF80E38093AE
:108EF000E02181E08093DF2180912D510E94302D6F
:108F00008AE30E94C42C80912C510E94302D8AE368
:108F10000E94C42C80912B510E94302D93CF5C98DD
:108F2000289829982A9887E0809348541EB81FB83B
:108F300008958091F4338115B1F0909140549132AD
:108F400090F081508093F43380910034811106C0F9
:108F5000809101340E94D0798093013480914054F3
:108F60008695809340548091F5338115B1F09091AE
:108F70003B54913290F081508093F53380910034CE
:108F8000813031F4809101340E94D0798093013492
:108F900080913B54869580933B5408951092485499
:108FA0008091455480B9809144548093F4338091EA
:108FB00043548093F533089580B180934554809154
:108FC000F433809344548091F5338093435410924A
:108FD000F4331092F53387E0809348540895CF938B
:108FE000DF93EFE2F1E2409908C0EFEAF0E2419945
:108FF00004C0EFE2F0E2429B629A38B1232F207165
:1090000034FF58C080E066E371E5349162993FE730
:109010008F3708F04AC03196DB01BF5F2C91205892
:10902000DB014C914058C303A0011124C4E08C9F84
:10903000D0011124AC5EBB4C4D935D93A303900112
:1090400011242D933D938F5F69F5629884E194E339
:109050000E94761D64E178E384E194E30E94481E57
:10906000809114389091153821E0981708F422E087
:1090700030E080E093E0F901EC5EF74C408194171A
:1090800010F4822F942F2F5F3F4F27FFF4CFE82F4C
:10909000F0E0EC5EF74C9081983008F480E0DF91CE
:1090A000CF9108956F5F7F4FB0CF87FFB5CF3197D6
:1090B000B3CFCD01449162994FE72F37D8F4319661
:1090C000DC018D918058382FB403812D112494E058
:1090D000299FA0011124BA016C5E7B4C4A5E5B4C57
:1090E000EB011A82EA018983EB01188289832F5FE1
:1090F00001F7ABCF27FFE4CF3197E2CF80B12FEF5D
:109100008B3008F42FE7479B09C08091415480932E
:10911000F73380913C548093F83308951092F733DD
:109120002093F833089B02C0109B08C080913B54E9
:10913000089B2AC090914054891730F58091405483
:10914000883080F1E091F633F0E0EA5CFE4A8695E3
:1091500090913F54890F9081981788F190E0319158
:10916000831708F446C09093F7339F5F3191381707
:1091700008F443C09093F8339F5F3081831778F5EC
:1091800031962913F9CF0EC0883060F0E091F633A4
:10919000F0E0EA5CFD4A869590913A54DBCF9F5F00
:1091A00029130EC080B18B3008F4B7CF8091F7330C
:1091B00086958093F7338091F8338695ACCF90E015
:1091C0003191381760F39093F7339F5F3191831794
:1091D00048F09093F8339F5F3081381730F09093C8
:1091E000F833E0CF2913F1CFDDCF31962913F3CF38
:1091F000D9CF9F5F2913B3CFD5CF2913B6CFD2CF05
:10920000CF93DF93EFEAF1E2A4EFB3E384919D9172
:10921000981728F09D0121503109E9018883319682
:10922000D4E3A431BD0791F780910A3490910934B9
:10923000891710F48093093480910B34811103C095
:1092400081E080930B3480910134833018F483E003
:10925000809301348091033490910234981710F474
:109260008093023480910434833018F483E0809337
:10927000043480B1863110F085E180B9DF91CF915F
:1092800008958091FE339091FF338F3F910520F533
:1092900090B1911102C08830C8F090B1913011F4B2
:1092A0008530B0F090B1923011F4853088F090B1F3
:1092B000963018F4843070F00895811106C081E072
:1092C00090E08093FE339093FF33089588E0F8CFC9
:1092D00085E0F6CF84E0F4CF97FFF7CF8FEF9FE7DD
:1092E000F0CF1F93CF93DF930E9400490E94414922
:1092F00084E08093A2001092400A1092410A1092DA
:10930000460A109240081092410888B1803240F419
:109310005E9B02C05F9B04C05E990FC05F9B0DC047
:109320008FE08093000882E08093040888E18093B6
:10933000270880910434809326088EE080930009EA
:1093400082E08093040987E28093260984B120E0BB
:10935000982F9170290F8695D9F788E090E0821BAD
:10936000880F880F880F90910734891710F4109296
:10937000073484E1809301028093410285E0809369
:1093800003028093430283E08093040280934402AB
:1093900090B19B3008F484C08093400A80B18B3038
:1093A00009F07BC087E893E18093660A9093670A8F
:1093B000E0B1F0E0EE0FFF1FEC5AF44D859195916E
:1093C000809346549093475481E0809300028093A9
:1093D000400280E280930202809342020E94DA3BC4
:1093E00080930C0281E20E94DA3B80930D0288E3B5
:1093F000809321029091F433892F880F880F836026
:109400008093200281E2809361021091F533812FD5
:10941000880F880F83608093600280E1809331021F
:10942000C0B180B1883008F0C7E027E0C29FE001FA
:1094300011249E01290F311DC9018C53954F0E94A3
:10944000FC7B819580933D54CE01810F911D845703
:10945000954F0E94FC7B81958093385484E00B9B50
:1094600044C08093050680E2139B42C080930506AA
:1094700081E01C9981E4199B03C01A993CC080616A
:109480009FEF9093B000809350065A9887E08093A6
:10949000A200DF91CF911F91089589E698E184CFD2
:1094A0001DB880B1863068F0E0B1F0E0EE0FFF1F2C
:1094B000EC58F44D859195918093660A9093670AD4
:1094C00083CF80B1811569F080B18F5F80930402F2
:1094D00080B18F5F80934402109203021092430286
:1094E00073CF82E080930402F5CF80930606BBCF52
:1094F00080930606BDCF8861C3CF1F920F920FB62F
:109500000F9211240BB60F92CF92DF92FF920F931E
:109510001F932F933F934F935F936F937F938F93FB
:109520009F93AF93BF93CF93DF93EF93FF93F0900D
:10953000E0210091DF218091240260913D540E943E
:109540004D1AC82F80916402609138540E944D1AC0
:1095500011270C99139511951C27CC271499C395A5
:10956000C195C82760E86C1B20E8210FA603D12C09
:109570001124D12F0E9B08C0D0E8DD0D0F9B04C035
:10958000812F0E944C1AD82F169B08C0179B37C1F9
:1095900060E8611B8C2F0E944C1AC82F80912751C4
:1095A00090912851A0912951B0912A518D0F911D70
:1095B000A11DB11D8093275190932851A09329514B
:1095C000B0932A518091235190912451A09125511B
:1095D000B09126518C0F911DA11DB11D8093235177
:1095E00090932451A0932551B093265180912151FD
:1095F0009091225101968093215190932251659A26
:10960000C0904654D090475480912151909122515E
:109610008C159D0508F456C01092215110922251CC
:109620000D9B0EC0960140E050E060912751709173
:1096300028518091295190912A510E940D7BD22F5F
:10964000159B0EC0960140E050E06091235170914F
:10965000245180912551909126510E940D7BC22F5B
:1096600010922751109228511092295110922A518C
:10967000109223511092245110922551109226518C
:109680003A9B10C0EDB1F0E0EA5CFE4A80818D0F9C
:109690008795EDB1F0E0EA5CFD4A90819C0F9795CB
:1096A000C92FD82FEDB1F0E0EA5CFE4AD083EDB1CE
:1096B000F0E0EA5CFD4AC083EDB18AB3F0E0EA5C19
:1096C000FC4A8083459B21C130991FC18091215163
:1096D00090912251892B09F495C00D9B93C0159B45
:1096E000C2C0DAB2C0910734189B21C0D7E310E89A
:1096F00084B18123C1F08DB1843059F41092E021FE
:109700008C2F8695869586958093DF218D2F0E94DC
:10971000C42C8D2D812309F4ECC08DB16C2F86955E
:109720000E94BD19C85F1695D150DF3209F71E9B04
:1097300012C08DB18F7079F4C93368F48DB18695FC
:109740008F5F8093E021C695C695C695C093DF21B3
:109750008D2D0E944E2D8091215190912251892B67
:1097600081F58DB18F5F8DB98DB1811101C0649A82
:109770003099D5C08DB1811109C01D9B03C0459999
:109780000E94AC351092460A5C991BC0459B19C0DB
:109790003D9917C0689915C01092DF212091E321EF
:1097A0003091E4219DB1969540E150E06FEF70E07B
:1097B000F901A2E19A9FE019F1091124CF010E9459
:1097C0008D7BF092E0210093DF21FF91EF91DF91FB
:1097D000CF91BF91AF919F918F917F916F915F9149
:1097E0004F913F912F911F910F91FF90DF90CF905C
:1097F0000F900BBE0F900FBE0F901F901895C0E8F2
:10980000CD0DCCCE609105348D2F0E944C1AD82FEF
:10981000D695EDB1F0E0EB5CFE4A609105348081B5
:109820000E944C1A3E9B4BC09DB1911509F447C054
:10983000282F2695D21304C0D11571F0DF3761F0BF
:10984000089B0AC04DB18DB14150550B55954795B8
:109850006D2F86950E94E919809121519091225196
:10986000892B09F03CCF609106348C2F0E944C1A52
:10987000C82FC695EDB1F0E0EB5CFD4A609106346F
:1098800080810E944C1A3E9B26C09DB1911519F112
:10989000282F2695C21306C0C11509F422CFCF3751
:1098A00009F41FCF109B1DCF4DB18DB14150550B09
:1098B000559547956C2F86950E94E91912CF089B04
:1098C000CBCFD11549F2DF3739F28DB16D2F8695A7
:1098D0000E94BD19C1CF109B04CFC11509F401CF5F
:1098E000CF3709F4FECE8DB16C2F86950E94BD193D
:1098F000F8CE8DB166E06C0F86950E94BD191B9B5A
:1099000011CF8DB165E06C0F0ACF479B24CF3F9BF1
:1099100022CF8DB16FE386950E94BD191CCF5C9B51
:1099200050CF1092460A4DCF8F938FB78F938BB73E
:109930008F93EF93FF93E0E0F8E086818E7F86833C
:10994000589A5D9AFF91EF918F918BBF8F918FBF46
:109950008F911895FF920F931F93CF93DF93809170
:1099600010018064809310018091200180648093B5
:10997000200185E0F82EF0921201D0E1D09313017E
:1099800000E012E0009314011093150184E194E3C8
:1099900080931C0190931D01C4E2C093180182E0E2
:1099A00080931901C0931001189B1CC00E94A63B14
:1099B00080913001806480933001F0923201D09325
:1099C0003301009334011093350184E194E48093D2
:1099D0003C0190933D018AE1809338011092390156
:1099E000C093300185E08093220180E180932301C0
:1099F000009324011093250184E19CE380932C01C2
:109A000090932D0184E68093280182E080932901C0
:109A100084E280932001189B05C08091300180680A
:109A200080933001809110018068809310018091B3
:109A3000200180688093200180B1863040F48CE161
:109A4000809301028093410280E090E006C082E0B2
:109A50008093400AF9CF019751F02091110124FD24
:109A600006C020E22A95F1F7589BF5CF5D98DF916B
:109A7000CF911F910F91FF90089588B1803258F4D3
:109A80008091455480B9809144548093F4338091FF
:109A900043548093F5334CE050E060E87AE080E096
:109AA00090E00E94947B40E250E060E079E084EF37
:109AB00093E30E94947B80B1809345548091F4336A
:109AC000809344548091F5338093435408952F92AA
:109AD0003F924F925F926F927F928F929F92AF923E
:109AE000BF92CF92DF92EF92FF920F931F93CF938B
:109AF000DF93CDB7DEB72897CDBFDEBF4CE050E097
:109B000060E87AE080E090E00E94F07B40E250E084
:109B100060E079E084EF93E30E94F07B88EE80932D
:109B2000800180E28093810188ED8093830180EE43
:109B3000809385018FE88093860190ED9093870153
:109B400082E28093210381E18093220383E080936A
:109B5000230329E0209320039093420196E29093FF
:109B6000430120E031E020934401309345012FED83
:109B700030E220934801309349019BE390934C01DC
:109B800080934D0184EA8093400180E88093000136
:109B900080B1809345548091F433809344548091F4
:109BA000F533809343541EB8589A5A9A599A669A34
:109BB000639A1FB826E331E52E835A990E947149B2
:109BC0005B9B08C01FB85C980E943D4D0E940C37FB
:109BD0000E947149609950C05C9B72C080910608D8
:109BE0008E7F809306085D9B30C288B1803220F45E
:109BF0005E9B02C05F9929C280B18B3008F094C38C
:109C00008FE99FE00197F1F700C000001092400A31
:109C100084E18093010280934102809136548F5FEA
:109C200080933654EFE7F2E03197F1F700C000007F
:109C30005D9810924008189B05C0809130018F7785
:109C40008093300180E091E0209110012F772093E4
:109C50001001209120012F77209320010091140101
:109C60001091150120B1211509F415C120E032E051
:109C7000201B310B89011AC17B9B03C05C990E9498
:109C80008F478EB18E3220F07A9901C07999669A09
:109C90007D9BA2CF2896CDBFDEBFDF91CF911F91D4
:109CA0000F91FF90EF90DF90CF90BF90AF909F907B
:109CB0008F907F906F905F904F903F902F9008957E
:109CC0005D998CCF3091FD3339835981511115C085
:109CD00080B18B3010F40E94AA4C289902C02A9BB4
:109CE00008C0309B03C080B18B3018F488B180323B
:109CF00068F4589973CF5D9A71CF5899E9CF81E094
:109D00000E94D43E498141504983DFCF10926008C0
:109D10001092610881E080934C088091FE3390910D
:109D2000FF3320B1211511F0880F991F20B12111A7
:109D300034C008978093660890936708809126083E
:109D40008093200880910C08816080930C082A9BE6
:109D500005C08091060881608093060869E280E86A
:109D600090E00E94BA7980910034813008F050C0B0
:109D700060913D546195809101340E944C1A2E9B54
:109D800021C060910334809102340E94CF1B6BE2AA
:109D900080E890E00E94BA7921CF20B1213011F4FF
:109DA0000597C8CF20B12230D9F320B1263010F466
:109DB0000497C0CF21E030E0009709F420E0821B37
:109DC000930BB8CF2D9B14C09091013480E8890F7C
:109DD000811544F480E8891B2B9B07C081950E9464
:109DE000751BD5CFC9F781E0F7CF0E948B1BCFCF72
:109DF0002F9B05C02B9B09C00E94221BC8CF20911E
:109E0000240290E8980F2917BCF30E94321BBFCFA1
:109E1000B1F5609138546195809101340E944C1ADB
:109E20002E9B07C060910334809102340E94DA1B9C
:109E3000AECF2D9B14C0909101349058292F220F42
:109E4000220B822F8927291301C081E02B9B04C09C
:109E500080950E94A31B9BCF0E94B91B98CF2F9B7C
:109E600005C02B9B09C00E94551B91CF2091640215
:109E700090E8980F2917BCF30E94651B88CF8B30A0
:109E800008F085CF82502B9B03C00E94C31A7FCF5E
:109E90000E94641A7CCF980121503140323008F082
:109EA0001BC293E0FC01E01BF10B8F01A8014C5E8B
:109EB0005B4C7A01C8018C5E934C4C01F801EC5E5E
:109EC000FB4B6F0126E332E529833A83412C66E39D
:109ED000A62E61E5B62EF6018081F501FE5F808336
:109EE000F7012081822FF40190819B830F5F1F4F28
:109EF000123008F0F5C13FEFC31AD30A4FEFE41A4E
:109F0000F40A5FEF851A950A30B13115F9F00D9B0F
:109F100005C0F701808185952595820F159B06C0A8
:109F2000F401F081F5959595F90FFB830F5F1F4FB5
:109F3000011522E0120709F4E2C13FEFE31AF30A28
:109F40004FEF841A940A5FEFC51AD50A0A9B06C020
:109F5000411421F0F7019081981B892F129B07C0B3
:109F6000411429F0F4019081FB819F1B9B83609138
:109F70003D540E944D1A66240C996394619468269E
:109F8000609138548B810E944D1A22271499239591
:109F900021952827288760E8621B20E8260DA60364
:109FA000312D11243B83562C0E9B09C05B8040E869
:109FB000540E0F9B04C0862D0E944C1A582E169BDF
:109FC00008C0179BABC160E8661988850E944C1ACF
:109FD000888795012F5F3F4FF5013A9BA3C1808190
:109FE000850D87958083E981FA818081F8858F0FBF
:109FF00087958887E981FA8148854193E983FA83C7
:10A00000439409F06BC18091382085FF0FC01092F6
:10A010003E2010923F2082E093E880933A20909374
:10A020003B20809138208D7980933820F894299BAB
:10A0300009C05C9A80B18B3028F48EB1853011F064
:10A0400085E38EB9669B58987894189B05C08091DB
:10A0500030018F7780933001809110018F7780934A
:10A060001001809120018F77809320015C9905C0B9
:10A07000309903C088B1803210F40E94A63B8BB1A6
:10A08000982F9072998385FDE6C03D990CC0479941
:10A0900008C0469906C0459B06C080B18B3008F0C9
:10A0A00030990E94492CF89480B18B3020F0309B7D
:10A0B00002C0649B9CC064984C9B2EC0E0B124E01D
:10A0C000E29FF0011124EE5EF44D2591359145910A
:10A0D0005591E0B1232F342F452F50E0A4E0469551
:10A0E00037952795AA95D9F7D1010E94687BE7306B
:10A0F00008F039C18C01169507950F3B08F027C170
:10A100009695879577956795609310347093113481
:10A1100080931234909313344D9B09C0C10175E0B4
:10A12000959587957A95E1F7819580930C344E9BB0
:10A1300009C0C10164E0959587956A95E1F780585B
:10A1400080930F344F9B08C0C10154E095958795CB
:10A150005A95E1F780930E34711002C070900B3461
:10A16000972D4A9991958091093430E1839FA00100
:10A17000112420910A3460E1269F90011124290EB8
:10A18000311C97FD3A94221533050CF0FAC04B9B15
:10A190009A01629A1901499B06C0489BFBC09FE740
:10A1A000791608F47394629B08C070900B344B9B33
:10A1B00004C099B124E0922799B9629899B190317D
:10A1C000B0F0599A3F9B13C06FE786950E94BD1966
:10A1D00080910A346FE786950E94BD196FE7C1012F
:10A1E00045E0959587954A95E1F70E94BD197894C9
:10A1F00090913651809136529C014981E42FF0E0D4
:10A20000EA5CFE4A5081FF5F4081951708F4952F64
:10A21000531708F4352F841708F4842F421708F4D5
:10A22000242F59815F5F59835111E7CF492F431B79
:10A2300040934054482F421B40933B5490933E54CC
:10A2400030933F548093395420933A54319B03C048
:10A2500045990E947E48459B7FC1369BBDC080B119
:10A26000F090F6338B3008F0F12C88E09BE00E94F0
:10A27000FC7BE82E87E09BE00E94FC7BD82E1982B5
:10A280000F2D10E0C801875F934F0E94FC7BC82E02
:10A29000C801875F944F0E94FC7B182F6E2D8C2D78
:10A2A0000E944C1ABC8086958C836D2D812F0E9454
:10A2B0004C1ACD8086958D830981015080B119811A
:10A2C0008B3010F0169506953E9B9AC069816111FE
:10A2D00067C081E08983D4CF9C01CACC5901FBCDF2
:10A2E00000E010E034E1C32E34E4D32E44E1842EA8
:10A2F0004CE3942E54E1E52E54E3F52E05CE00E018
:10A3000010E0B4E1CB2EB4E4DB2E94E1892E9CE383
:10A31000992E24E1E22E24E3F22E18CE5B815058D0
:10A32000588757CE508266CE309B07C05D985C99A7
:10A330007DCE82E08093460A79CE649BFACF649802
:10A340005D98809136548F5F809336546FCE8FEF37
:10A350009FEFAEEB8093103490931134A09312349E
:10A3600010921334D9CE20ED37E040E00E940D7BEF
:10A37000209310343093113440931234509313349B
:10A38000CBCE241635060CF006CF4B9BA901629A62
:10A390001A0101CFE2E07E1608F405CF7A9403CFCC
:10A3A000089B06C02B2D402F6C81812F0E94E9193C
:10A3B000109B06C02C2D402F6D81812F0E94E91922
:10A3C00080B18B3018F499819F3730F4F394E98190
:10A3D000EF5FE983E11154CF80B18B3010F0309BF7
:10A3E000BBC080B18B30C8F0309B17C08DB1B82E88
:10A3F0006894B0F81982812C00E0912CC12C12C015
:10A40000089B04C06C81812F0E94BD19109BD8CF7E
:10A410006D81812F0E94BD19D3CFB090F633EACF62
:10A42000812E0D2D8B2D8C0D90B19B3028F0309B03
:10A4300003C0FC2DF695F98390E09C012A5C3E4A0E
:10A4400079018A5C9C4AFC01608010910734189B5A
:10A450003CC020E8A22E37E0D32E84B18A2181F1BE
:10A46000F981F11124C0512E5694569456941092AD
:10A47000E0215092DF2180E38D0D0E94C42C809159
:10A4800000348250990BD816190689F42F812E3783
:10A4900070F4289902C02A9B0AC03F813093E021C2
:10A4A0005092DF2189E12B9B88E10E94C42C862DEC
:10A4B0008A2109F454C1612F89810E94BD19185F56
:10A4C000A694DA944FEFD412C8CF1E9B10C0898196
:10A4D0008F7069F4193358F459815093E02116951F
:10A4E000169516951093DF21862D0E944E2D6091B2
:10A4F0000534F70180810E944C1AD82EF701FF5FC6
:10A500006091063480810E944C1AD694182F1695BB
:10A510003E9B38C1F981F115B1F0D01204C001158C
:10A5200051F00F3741F0089B06C0202F492D6D2DAB
:10A5300089810E94E91918111CC1111519F01F37E2
:10A5400009F017C1998039813F5F3983C39437FF80
:10A5500067CF1D990E94AC3546992CC1479B44C0DA
:10A560008BB1182F107285FD3FC0089B6BC11099ED
:10A570006CC167E76983DD24D39488B184FBFF2431
:10A58000F4F884FF6BC187B1837079F060E180914A
:10A59000F6330E94BD1960E28091F6330E94BD1926
:10A5A00060E38091F6330E94BD1980E090E00E9444
:10A5B000EF47E091F633F12FFE1BEF2FF0E0EC5E5A
:10A5C000F74C60816695669527E7261B622F3E9BB8
:10A5D00041C127E7412F812F0E94E9191F5F1038E1
:10A5E00041F731990E947E4888B1803208F057C007
:10A5F0005D9B04C05E9B53C05F9B51C0409148541B
:10A60000498341114CC084E0809348540E94492CF6
:10A610005E9B02C05F990CC049E557E260E08CE0A8
:10A620000E94A92E48E657E260E08CE40E94A92E21
:10A630005E9B02C05F9B04C05E9969C15F9B67C15E
:10A6400044EE5EE260E081E30E94A92E44EE5EE209
:10A6500060E081E70E94A92E86E3E82E81E5F82ECE
:10A660008701F7016081FFEFEF1AFF0A6695669593
:10A670006695645E89810E94BD19F801FF5F608163
:10A68000669566956695645E8981805C0E94BD19B9
:10A6900029812F5F2983203419F70E949345659BF8
:10A6A00017C065988091382085FF12C08DB18093C6
:10A6B000375410923E2010923F2042E053E84093DE
:10A6C0003A2050933B20809138208D798093382018
:10A6D00080914854811509F41EC21091F433009101
:10A6E000F533F0B058B1598343980E98169886E325
:10A6F00091E50E94EF478093415486E392E50E94E2
:10A70000EF4780933C54698168B988B1803208F082
:10A7100043C15F9944C15E9945C185E089838091B9
:10A72000F4332981281710F42093F4338091F53302
:10A730003981381710F43093F53380B18B3010F035
:10A740004AE040B920914854283008F0D7C1E22FA0
:10A75000F0E08827E158F3488F4F0C944E7B66E079
:10A76000610F89810E94BD191B9BA9CE65E0610F15
:10A77000A3CE109BE7CE282D492D612F89810E9401
:10A78000E919E0CE089B09C0D11439F02FE7D216A1
:10A7900021F06D2D89810E94BD19109BD3CE11151A
:10A7A00009F4D0CE1F3709F4CDCE612F89810E94E4
:10A7B000BD19C8CE3F9B06C04AE05AE260E080E087
:10A7C0000E94A92EE6E3F1E580B18B3050F130997B
:10A7D00028C09DB18E2F46E351E5841B981321C0FC
:10A7E000369BBCCE86E09BE00E94FC7BE82EF12CE1
:10A7F0000F2D10E0C801875F944F0E94FC7B8E19DB
:10A80000898387FD0BC0C801875F934F0E94FC7B43
:10A8100069816695809586950E94BD19F39441F7EC
:10A820009DCE8F010F5F1F4FDF01BF5F6C9166955B
:10A830008081809586950E94BD195E81501781F2B6
:10A84000F801C2CF87E7898396CE9BE3998392E094
:10A85000D92E93CE812F0E94BD19C0CE089928C051
:10A86000109BBFCE86E392E50E94EF4780933C5455
:10A8700004E118E3F80161918F0187B170E00D2CBC
:10A8800002C0759567950A94E2F7F981F61708F406
:10A890006F2F27E7261B622F86FF35C027E74F2D36
:10A8A0008F2D0E94E919F39430E8F312E3CF99CE8B
:10A8B00086E391E50E94EF478093415404E118E359
:10A8C000E12CF80161918F0187B170E00D2C02C07D
:10A8D000759567950A94E2F7F981F61708F46F2FDA
:10A8E0002981261B622F86FF0AC029814E2D8E2DBD
:10A8F0000E94E919E39430E8E312E3CFB1CF8E2D43
:10A900000E94BD19F7CF8F2D0E94BD19CCCF809129
:10A910000034823010F08A30C1F44AED58E263E02E
:10A9200080E10E94A92E0AE5F02E5E9B1DC01092C8
:10A93000485441EF5EE263E082E60E94A92E5C9BF0
:10A94000F982398130938201A8CE1EE5F12EF80EEE
:10A9500042EA56E263E080E10E94A92E8091003431
:10A96000825D0E94C42CE1CF46EF5EE263E082E6A6
:10A970000E94A92E80B106EF1EE2873010F007EF8B
:10A980001EE2A80160E08DE20E94A92EA80160E00D
:10A990008DE60E94A92ED4CF95E09983C0CEE3E046
:10A9A000E983BDCEF3E0F983BACE88B1803208F4F2
:10A9B00058C02D982E982F9A089A109A909140542A
:10A9C000903108F4089880913B54803108F4109835
:10A9D000089904C0109902C0089A109A30E4309384
:10A9E000F633E0E8E093FE331092FF339695309112
:10A9F0003F54930F869530913A54830F089B49C07A
:10AA000030914154323008F444C040913C543417E2
:10AA100008F43FC02A9A1092003490930134392FE1
:10AA20000C9946C0459B1DC0969530E4432F491BA9
:10AA3000409305348695381B30930634089B0FC02D
:10AA4000109B0DC040E2491B942F303E14F420E6C9
:10AA5000281B90930534209306340E9499470E9446
:10AA6000994788B1803220F45E9902C05F9B46C04E
:10AA700090913C5480914154891708F4892F829514
:10AA80008F7090B18917C0F490B1981B892F80B94D
:10AA900035C0109BC7CF30913C54323018F22A9AFF
:10AAA00031E03093003480930134149BBBCF382FB6
:10AAB000309530930134B6CF81E0E9CF80913E5498
:10AAC0008C3B60F480913F548A3440F08091F433A1
:10AAD000F9818F1718F48F5F8093F4338091395484
:10AAE0008C3B60F480913A548A3440F08091F53385
:10AAF0002981821718F48F5F8093F5338091F433A6
:10AB0000811308C08091F533801304C080B18F1584
:10AB100009F464C05A9A669BDFC09091003466982D
:10AB20007D9B66C08EB1811162C02896CDBFDEBF0D
:10AB3000DF91CF911F910F91FF90EF90DF90CF9019
:10AB4000BF90AF909F908F907F906F905F904F904D
:10AB50003F902F900C943D4D80913E548A3F20F4BD
:10AB600080913F54823138F48091F433811519F08B
:10AB700081508093F433809139548A3F28F4809136
:10AB80003A54823108F0BACF8091F533811509F437
:10AB9000B5CF8150B1CF809141548D3728F4809149
:10ABA0003C548D3708F4AACF80B1823008F4A6CF88
:10ABB00080B181506CCF80914154823308F09ECF98
:10ABC00080913C54823308F099CF80B18A3008F0EC
:10ABD00095CF80B18F5F5BCF10B890CF80914854F4
:10ABE000811509F498CF81508093485498CD1EB8B0
:10ABF0007E9B02C07F993B9A789B0AC08EB18430BD
:10AC000009F45B9AEEB1F0E0EB5BFA4DE491EEB93A
:10AC10007C9B06C0EEB1F0E0EE5FFA4DE491EEB938
:10AC20008EB1863340F18EB18D3328F57B9B23C0E6
:10AC3000EEB1F0E0EE0FFF1FE55FFC4DA591B59181
:10AC40008091425421E0280F209342542EB1265384
:10AC5000330B45E0429FF001439FF00D1124E80FB4
:10AC6000F11DEB57FC4DE491EC93809142548530FB
:10AC700010F010924254EEB1E334B0F4F0E08827C3
:10AC8000E957F3488F4F0C944E7BF8947B9B04C09C
:10AC9000299B5EC01DB85C987A9B62C0799B60C09E
:10ACA00080E48093F63378948EB18D3338F08EB192
:10ACB000833420F480B18B3008F0639A8EB1811117
:10ACC00009C05C9B07C080B18B3010F0469B02C06E
:10ACD00085E38EB90E940049589B0AC058980E948B
:10ACE0007149639902C03D9BA5C663980E94492C97
:10ACF0008EB1811511F40C944F628EB18D3208F42F
:10AD0000A6C68EB18E3210F00C947E5F1092E021B8
:10AD10008FE08093DF218091003481110C94B05F2B
:10AD2000F090F43341B1498364E007EE1EE2F61679
:10AD300010F404EE1EE2EEB1E652E53110F00C9490
:10AD4000C65FF0E08827E653F3488F4F0C944E7BA4
:10AD50008BB190E189278BB95C9B9ECF58989CCF93
:10AD60007A9B1DC09BB1892F807194FD18C090B152
:10AD70009531A8F590B19F5F90B990E8E82FF0E089
:10AD8000EA5CFE4A9083DF01BF5F9C93FE5F108206
:10AD90008F5FA1F7639A1DB81092460A5D98799B60
:10ADA00082CF9BB1892F807194FD7DCF90B1911599
:10ADB00019F090B1915090B990E8E82FF0E0EA5C7A
:10ADC000FE4A9083DF01BF5F9C93FE5F10828F5F1E
:10ADD000A1F7639A1DB81092460A5D9864CF95E179
:10ADE000CBCF639A7B9B04C081B191E0892781B965
:10ADF0007A991CC0799B58CF8091F433863008F043
:10AE000053CF8F5F8093F43319822981022F10E092
:10AE10000A5C1E4AF80180810E94D979F80180837A
:10AE2000F981FF5FF983F111F0CF3ECF8091F433C8
:10AE3000811501F381508093F43319823981032FF6
:10AE400010E00A5C1E4AF80180810E94D079F80166
:10AE50008083F981FF5FF983F111F0CFCBCF639A43
:10AE60007B9B04C082B191E0892782B97A991CC08A
:10AE7000799B1ACF8091F533863008F015CF8F5F1C
:10AE80008093F53319822981022F10E00A5C1D4A54
:10AE9000F80180810E94D979F8018083F981FF5FF0
:10AEA000F983F111F0CF00CF8091F533811501F3D3
:10AEB00081508093F53319822981022F10E00A5CBA
:10AEC0001D4AF80180810E94D079F8018083F981C0
:10AED000FF5FF983F111F0CFCBCF7B9B04C083B12F
:10AEE00091E0892783B97A9B02C08CE18EB9799B66
:10AEF000DBCE83E28EB9D8CE7B9937987A99379A90
:10AF0000799BD2CE85B190E1892785B9CDCE7B9B47
:10AF100006C0289B11C029990FC028985C987A9B7D
:10AF200004C02A98289A299A5C98799BBDCE2A9BBE
:10AF300007C02A985C98B8CE2A982998289AEECF0C
:10AF40002A9A29982898F6CF7B9B03C0359B18C076
:10AF500035987A9B09C086B198E0892786B9339BDA
:10AF600003C034988FE38EB9799B9ECE86B190E171
:10AF7000892786B9349B98CE339881E48EB994CED4
:10AF8000359A8DE38EB9E5CF7B9B03C0409B0CC007
:10AF900040987A9B03C0419B0BC04198799B84CE1B
:10AFA000429B0AC0429880CE409A41984298F1CF85
:10AFB0004098419A4298F2CF40984198429A74CE74
:10AFC0007B9B06C01092003481E32E9B80E38EB9F8
:10AFD0007A9B07C081E08093003481E32E9B80E35D
:10AFE0008EB9799B61CE8FE18EB95ECE7B9B5CCEB4
:10AFF000389B04C087B192E0892787B987B191E077
:10B00000892787B951CE7B9B02C05E9A5F987A9B55
:10B0100002C05E985F9A799B47CE5E9905C05F99A2
:10B0200003C05E9A5F9A40CE5E985F983DCE7B9B50
:10B0300003C081E080930D347A9B03C082E080934B
:10B040000D34799B03C083E080930D34599A2CCE44
:10B050007B9B02C08BE38EB97A9B04C081B198E0E0
:10B06000892781B9799B20CE87E28EB91DCE7B9B43
:10B0700002C08CE38EB97A9B04C082B198E0892724
:10B0800082B9799B11CE88E28EB90ECE7B9B05C02A
:10B0900080910734885F809307347A9B04C083B122
:10B0A00090E1892783B9799BFFCD83B198E0892707
:10B0B00083B9FACD7B9B02C081E08EB97A9B02C036
:10B0C00082E08EB9799BF0CD83E08EB9EDCD7B9B8C
:10B0D00002C085E08EB97A9B02C088E08EB9799B68
:10B0E000E3CD89E18EB9E0CD88B1803210F40E94C1
:10B0F000CE4728B129837B9B19C0799B17C0469BFB
:10B1000012C04598469A479A8FB18111FDCF88B1F8
:10B11000803210F40E94DC4788B13981831709F42A
:10B12000C3CD639AC1CD459A4698EDCF7B9B09C0AC
:10B13000479902C0469903C0459A4698479888E1C6
:10B140008EB97A9B05C04598469847988AE08EB993
:10B15000799BDDCF45984698479A82E18EB9D7CF43
:10B160007B9B04C088B190E1892788B97A9B02C093
:10B1700087E08EB9799B98CD88B198E0892788B906
:10B1800093CD7B9B02C086E08EB97A9B02C085E29C
:10B190008EB9799B89CD84E18EB986CD7B9B02C027
:10B1A0008BE08EB97A9B02C087E18EB9799B7CCD0A
:10B1B0008FE28EB979CD7B9B03C084E080930D3400
:10B1C0007A9910920D34799B03C085E080930D34F9
:10B1D000599A6ACD7B9B02C086E38EB97A9B02C0E6
:10B1E0008CE28EB9799B60CD83E38EB95DCD7B9B7C
:10B1F00004C089B190E1892789B97A9B04C089B1DB
:10B2000090E2892789B9799B4FCD89B1805889B956
:10B210004BCD7B9B06C086B191E0892786B93099DA
:10B220003A987A9B06C087B194E0892787B93A9902
:10B230003098799B39CD639A469B03C0459A4698CE
:10B2400033CD4598469A30CD7B9B02C08AE18EB9BA
:10B250007A9B02C08EE28EB9799B26CD8AE38EB9A5
:10B2600023CD7B9B03C02E9B0CC02E987A9B03C0E2
:10B270002F9B0BC02F98799B17CD2D9B0AC02D9823
:10B2800013CD2F982D982E9AF1CF2F9A2D982E9876
:10B29000F2CF2F982D9A2E9807CD7B9B04C086B1B4
:10B2A00092E0892786B97A9B04C086B194E0892709
:10B2B00086B9799BF9CC86B190E4892786B9369B0B
:10B2C000F3CC6091053488E09BE00E94117C609192
:10B2D000063487E09BE00E94117C6091F63386E0A3
:10B2E0009BE00E94117C8091CF0187FDFCCF40E064
:10B2F00051E069E07CE086E391E50E94947B40E0C8
:10B3000051E069E07BE086E392E50E94947BCCCC3F
:10B31000109207347B9B04C084B18F3F71F414B842
:10B320007A9B04C084B191E0892784B9799BBCCC15
:10B3300084B192E0892784B9B7CC8FEF84B9F0CF7C
:10B34000109207347B9B04C084B194E0892784B9B0
:10B350007A9B04C084B198E0892784B9799BA4CCF6
:10B3600084B190E1892784B99FCC109207347B9BEC
:10B3700004C084B190E2892784B97A9B04C084B167
:10B3800090E4892784B9799B8FCC84B1805884B9A3
:10B390008BCC7B9B03C08AE0809300347A9B03C0F4
:10B3A00082E080930034799B03C083E08093003473
:10B3B0007C997ACC80910034891376CC85B198E061
:10B3C000892785B971CC7B9B03C084E080930034CE
:10B3D0007A9B03C085E080930034799B03C086E0AC
:10B3E000809300347C9960CC8091003489135CCCCC
:10B3F00085B198E0892785B957CC7B9B03C087E04E
:10B40000809300347A9B03C088E080930034799B5A
:10B4100003C089E0809300347C9946CC809100344D
:10B42000891342CC85B198E0892785B93DCC7B9BB7
:10B4300004C083B190E4892783B97A9B04C083B1A7
:10B4400090E2892783B9799B2FCC84E28EB92CCCEA
:10B450007B9B05C081E08093083484E08EB97A9BA1
:10B4600005C082E0809308348DE28EB9799B1CCCB4
:10B470001092083486E28EB917CC7B9919987A9B82
:10B4800002C0199A1A9A799B0FCC199A1A980CCC67
:10B490007B9B04C087B190E2892787B97A9B04C05F
:10B4A00087B190E4892787B9799BFECB87B1805813
:10B4B00087B9FACB7B9B04C08AB190E489278AB90B
:10B4C0007A9B03C08AB180588AB9799BEDCB8AB147
:10B4D00090E289278AB9E8CB7B9B02C089E28EB9CA
:10B4E0007A9B05C081B190E1892781B9639A799BE4
:10B4F000DBCB81B190E2892781B9D6CB7B9B02C09F
:10B500008AE28EB97A9B05C082B190E1892782B91F
:10B51000639A799BC9CB82B190E2892782B9C4CB67
:10B520007B9B07C00E9B15C081B1805881B90F9BD2
:10B530000E987A9B07C00E9B0FC081B1805881B9CD
:10B540000F990E98799BB0CB81B194E0892781B98E
:10B55000ABCB0E9A0F9AEDCF0E9A0F98F3CF7B9B41
:10B5600007C0169B15C082B1805882B9179B1698E8
:10B570007A9B07C0169B0FC082B1805882B9179979
:10B580001698799B91CB82B194E0892782B98CCBB4
:10B59000169A179AEDCF169A1798F3CF7B9B02C095
:10B5A00087E38EB97A9B02C089E38EB9799B7CCB05
:10B5B00088E38EB979CB7B9B04C089B194E089275D
:10B5C00089B97A9B04C089B198E0892789B9799BA8
:10B5D0006BCB499B05C0489B03C04998489864CBF6
:10B5E000499B02C0489A60CB499A5ECB7B9B09C0BD
:10B5F0008AB19AB1907E9AB99AB18F5F8F71892B77
:10B600008AB97A9B04C0559908C0559A5698799B77
:10B610004BCB8AB180588AB947CB569902C0569A0B
:10B62000F6CF5598F4CF8091FE339091FF337B9BFA
:10B630000DC080389105E1F021E08115914009F4B9
:10B6400020E0922F969520FB882787F97A9B07C0E8
:10B6500021E030E0009709F420E0821B930B7999F8
:10B6600001968093FE339093FF330E9441491CCB97
:10B6700080E091E0EBCF7B990E94C5267A9B03C0C6
:10B68000619A0E94C526799B03C0629A0E94C526D2
:10B6900061986298599A08CB7B9B21C080910134B4
:10B6A000803891F580910034813070F4809140545D
:10B6B000869590913F54890F809301340C9B0FC065
:10B6C0008095809301340BC051F480913B54869552
:10B6D00090913A54890F809301341499F1CF7A9B59
:10B6E00008C0809101348F3F19F08F5F809301343F
:10B6F0002B9A799BD9CA80910134811519F0815018
:10B70000809301342B98D0CA80E8DBCF7B9B02C0AA
:10B7100082E38EB97A9B07C0809102348E3F18F481
:10B720008E5F80930234799BBFCA8091023481304E
:10B7300008F4BACA19F410920234B6CA825080933F
:10B740000234B2CA7B9B02C081E38EB97A9B07C0E8
:10B75000809103348E3F18F48E5F80930334799B7D
:10B76000A3CA80910334813008F49ECA19F4109260
:10B7700003349ACA82508093033496CA7B9B02C0DA
:10B7800084E38EB97A9B07C080910934811519F042
:10B79000815080930934799B87CA809109348F3F07
:10B7A00009F482CA8F5F809309347ECA7B9B02C0F2
:10B7B00083E38EB97A9B07C080910A34811519F012
:10B7C000815080930A34799B6FCA80910A348F3FED
:10B7D00009F46ACA8F5F80930A3466CA7A9B06C0EE
:10B7E000799B04C080E48093F6335ECA7B9B02C0E1
:10B7F0005C981EB87A9B07C08091F633811519F0CA
:10B8000081508093F633799B4FCA8091F6338F5FD6
:10B810008093F63349CA7A9B07C080910B348230FB
:10B8200018F0815080930B34799B07C080910B34C2
:10B830008F3718F48F5F80930B3470900B3434CAB9
:10B840007A9B05C080910C348F5F80930C34799B78
:10B8500007C080910C34803819F0815080930C34EB
:10B86000599A22CA7A9B07C080910F348F3719F0FA
:10B870008F5F80930F34799B07C080910F3480389D
:10B8800019F0815080930F34599A0ECA7A9B07C0E1
:10B8900080910E34811519F0815080930E34799B7C
:10B8A00007C080910E348F3F19F08F5F80930E3464
:10B8B000599AFAC97A9B07C08091FD33811519F016
:10B8C00081508093FD33799BEFC98091FD338F3F89
:10B8D00009F4EAC98F5F8093FD33E6C97A9B05C0FE
:10B8E000809105348E5F80930534799BDDC980910A
:10B8F0000534803809F4D8C99FEF980F813819F4BE
:10B9000090930534D1C9825080930534CDC97A9B78
:10B9100005C0809106348E5F80930634799BC4C93C
:10B9200080910634803809F4BFC99FEF980F8138A1
:10B9300019F490930634B8C9825080930634B4C980
:10B940007B9B02C08EE38EB97A9B08C031988091B0
:10B95000F733811519F081508093F733799BA4C98F
:10B9600031988091F7338F5F8093F7339DC97B9B2C
:10B9700002C08DE38EB97A9B08C031988091F8336C
:10B98000811519F081508093F833799B8DC93198D6
:10B990008091F8338F5F8093F83386C97B9B02C018
:10B9A00080E48EB97A9B05C08091F9338F5F8093D4
:10B9B000F933799B79C98091F93381508093F933B8
:10B9C00073C97B9B02C08FE38EB97A9B05C08091BF
:10B9D000FA338F5F8093FA33799B66C98091FA338B
:10B9E00081508093FA3360C97B9B02C082E48EB998
:10B9F0007A9B05C08091FB338F5F8093FB33799BEB
:10BA000053C98091FB3381508093FB334DC97B9B9D
:10BA100002C081E48EB97A9B05C08091FC338F5FB0
:10BA20008093FC33799B40C98091FC338150809393
:10BA3000FC333AC9E091E321F091E421CF01995020
:10BA40002FEF278772978E179F07D9F751C910924A
:10BA5000E0218FE08093DF21EEB1E150FF0BE8574A
:10BA6000FA4D049153E2059F800111240C541A4DA4
:10BA700019826198EEB1E150EC3260F4F0E0882771
:10BA8000E152F3488F4F0C944E7B6981611102C0E3
:10BA90000899619A0F5F1F4FF801319784918111C6
:10BAA0002AC2619839813F5F3983333011F729C940
:10BAB00089818111EFCF109BEDCF619AEBCF9981F6
:10BAC0009111E8CF189BE6CF619AE4CFE981E111AB
:10BAD00004C03799DFCF619ADDCFF981F13019F4D5
:10BAE000379BD8CFF8CF2C9BD5CFF5CF298121110B
:10BAF00006C0289BCFCF2999CDCF619ACBCF398172
:10BB0000313019F42999F9CFC5CF2A9BC3CFF5CF8E
:10BB10004981411104C0359BBDCF619ABBCF59818A
:10BB2000513019F43399F9CFB5CF349BB3CFF5CF5A
:10BB30006981611104C0409BADCF619AABCF89810F
:10BB4000813019F44199F9CFA5CF429BA3CFF5CF0E
:10BB5000809100349981911105C0811509F09ACF27
:10BB6000619A98CFE981E13011F48130F7CF8230CA
:10BB7000B8F790CFF981F1118DCF87B1837009F4B7
:10BB800089CF619A87CF2981211105C05E9B82CF21
:10BB90005F9B08C07FCF3981313031F45F9B7ACF12
:10BBA0005E9978CF619A76CF5E9974CFF1CF80910C
:10BBB0000D344981411105C0813009F06BCF619A84
:10BBC00069CF5981513011F48230F7CF8330F5CFEE
:10BBD0006981613021F40B9B5DCF619A5BCF8981D4
:10BBE000823009F057CF0E9B55CFF7CF9981913016
:10BBF00021F4139B4FCF619A4DCFE981E23009F0D8
:10BC000049CF169B47CFF7CFF981F13021F41C9B28
:10BC100041CF619A3FCF2981223009F03BCF1B9B56
:10BC200039CFF7CF3981311106C0459902C0469B03
:10BC300031CF619A2FCF4981413021F488B18032D0
:10BC4000C0F328CF479B26CFF4CF5981511104C0B0
:10BC5000449B20CF619A1ECF6981623009F01ACFD0
:10BC6000439B18CFF7CF80910D349981911105C076
:10BC7000843009F00FCF619A0DCFE981E13011F4E2
:10BC80008115F7CF8530F5CFF981F11104C04C9BB8
:10BC900001CF619AFFCE2981213019F44D99F9CF56
:10BCA000F9CE4F9BF7CEF5CF3981311104C0309BCF
:10BCB000F1CE619AEFCE4981413019F43A99F9CF2A
:10BCC000E9CE469BE7CEF5CF5981511104C02E9B9A
:10BCD000E1CE619ADFCE6981613019F42F9BDACE13
:10BCE000F8CF2D9BD7CEF5CF8981811104C0319B30
:10BCF000D1CE619ACFCE9981913019F43299F9CF92
:10BD0000C9CE369BC7CEF5CFE981E11106C084B11B
:10BD10008F3F09F0BFCE619ABDCEF981F13019F4A1
:10BD20002099F9CFB7CE219BB5CEF5CF298121112E
:10BD300004C0229BAFCE619AADCE3981313019F467
:10BD40002399F9CFA7CE249BA5CEF5CF49814111E8
:10BD500004C0259B9FCE619A9DCE5981513019F424
:10BD60002699F9CF97CE279B95CEF5CF80910034B9
:10BD70006981611105C08A3009F08CCE619A8ACE42
:10BD80009981913011F48230F7CF8330F5CF8091D3
:10BD90000034E981E11105C0843009F07BCE619A5D
:10BDA00079CEF981F13011F48530F7CF8630F5CFB7
:10BDB000809100342981211105C0873009F06ACEB5
:10BDC000619A68CE3981313011F48830F7CF8930EB
:10BDD000F5CF4981411104C01E9B5CCE619A5ACEB9
:10BDE0005981513009F056CE1D9B54CEF7CF698151
:10BDF000611104C019994ECE619A4CCE898181306F
:10BE000029F4199B47CE1A99F7CF44CE199B42CEFD
:10BE10001A9940CEF1CF9981911104C03D9B3ACE41
:10BE2000619A38CEE981E13019F43E99F9CF32CEEA
:10BE30003F9B30CEF5CFF981F23009F02BCE559BE8
:10BE400029CE619A27CE2981211104C00E9B22CED2
:10BE5000619A20CE3981313019F40C99F9CF1ACE7C
:10BE60000D9B18CEF5CF4981411104C0169B12CE0F
:10BE7000619A10CE5981513019F41499F9CF0ACE34
:10BE8000159B08CEF5CF6981611106C00E9B02CECD
:10BE90000F9B00CE619AFECD8981813029F40E9BE3
:10BEA000F9CD0F9BF7CFF6CD0A9BF4CDF3CF998157
:10BEB000911106C0169BEECD179BECCD619AEACD91
:10BEC000E981E13029F4169BE5CD179BF7CFE2CD50
:10BED000129BE0CDF3CFF981F11104C04A9BDACD7A
:10BEE000619AD8CD2981213019F44B99F9CFD2CD5F
:10BEF000499BD0CDF5CF0E94C42CCCCD8EB18334DC
:10BF000018F01EB80C94865644E653E26FE088E3BE
:10BF10000E94A92E8EB18B3310F40C948656109289
:10BF2000E0218FE08093DF218EB18D3330F482E108
:10BF300097E20E94222D0C9486568EB18F3370F4B6
:10BF400086E50E94C42C82E496E20E94222D81E3C1
:10BF5000709B82E30E94C42C0C94865688E4F1CF37
:10BF6000F090F53352B159830C94945681E2569B6C
:10BF70002BC18093E02168E08DE69EE10E94AE2C0B
:10BF800069E786E2579B83E20E94BD1988B180323F
:10BF900008F432C347993FC0469987C2809105345F
:10BFA000982F990F990B80589F4F95958795898366
:10BFB00080910634982F990F990B80589F4F959533
:10BFC0008795182F87B183708230A9F0833009F4E8
:10BFD00080C2813001F58091E3219091E421FC0140
:10BFE000EE57F4408057944020812F77208332967B
:10BFF000E817F907C9F700E1089B04C06981802FA1
:10C000000E94BD19109B04C0612F802F0E94BD1992
:10C01000005F003889F7339B02C0089903C0349B46
:10C0200003C010990E945944469903C035990E9453
:10C0300085433F9B53C081B1F82FF170F98380FF96
:10C040001BC00E9B56C288E58093E0211092DF2131
:10C050008DE20C9B80E20E94C42C89E597E20E944D
:10C06000222D0F9B38C28BE2149B8DE20E94C42CC0
:10C0700087E697E20E94222D109B1FC0169B67C285
:10C0800088E58093E02139813093DF218DE2149B94
:10C0900080E20E94C42C88E697E20E94222D179B22
:10C0A00048C28BE20C9B8DE20E94C42C88E597E28B
:10C0B0000E94222D69816F5F6983479B69C240B1ED
:10C0C00085E0489FA001112440525C4D698189E5BB
:10C0D0000E94A92E88E293E20E94222D289902C094
:10C0E0002A9B8AC2459B88C280B18B3020F4809104
:10C0F000FF338111E8C22E9B59C2E0910234EB83D9
:10C100001091033480910034813008F056C20C9BAA
:10C1100008C02B8120952B8310958CB194E0892742
:10C120008CB9809105343B81380F3B83180F80B167
:10C130008B3008F454C286B1682F61706F8380FD24
:10C14000BFC280910034823008F055C2EB81E69581
:10C15000E98387B18370823061F460E18F810E944E
:10C16000BD1960E28F810E94BD1960E38F810E943A
:10C17000BD192E9B70C21695F981FD3748F448E928
:10C180005EE16F2F629909C0898183508D3740F439
:10C19000629906C047EA5EE169818F810E948A2C1C
:10C1A0001D3748F447EA5EE1629909C08DEF810FBF
:10C1B0008D3708F020C262991EC248E95EE1612F06
:10C1C0008F810E948A2C17C28093E02168E085E766
:10C1D0009EE1D4CE8CE78093E021499BD7CE88E1C5
:10C1E000489B89E10E94C42CD1CE8AB18695869560
:10C1F000869583708B5C0E94C42C4AB1477087E09F
:10C20000489FA001112448555C4D6FE088E00E94D2
:10C21000A92E43E453E26FE080E3559B0AC049E551
:10C2200053E26FE08CE2569904C04DE453E26FE0B4
:10C2300088E20E94A92E49E353E2579902C04FE2D7
:10C2400053E26FE08CE50E94A92EA0CE80B18B3026
:10C2500008F09CCEE0B1F0E0EE0FFF1FEA51F54D83
:10C2600025913591A091FE33B091FF330E94DE7A83
:10C270009B01AC01213797E039079DE34907510540
:10C2800024F020E737E04DE350E0AAEFB0E00E9451
:10C290005D7B9B01AC016FE080E00E945D2D80B171
:10C2A000873028F487E10E94C42C83E59BCF8AE184
:10C2B0000E94C42C8BE1F7CFA091DE20B0E020E2F9
:10C2C0003CEB4EEB50E00E945D7B009110341091EE
:10C2D00011342091123430911334003A1648214021
:10C2E000310528F5009166091091670920E030E0DA
:10C2F000E0914009E13021F030E0212F102F00E0E3
:10C30000A90198012F5F3F4F4F4F5F4F0E940D7B58
:10C31000A8EEB3E00E945D7B9B01AC016FE080E082
:10C320000E945D2D87EF9EE20E94222D2FCE20914C
:10C330006609309167092F5F3F4F40E00E940D7BF7
:10C340006FE080E00E945D2D86EF9EE2EDCF2091B0
:10C3500001342D9B47C0F0E8F21BF983F7FF02C0C0
:10C3600020582983E0B1F0E0EE0FFF1FEA51F54DB0
:10C3700045915591EF2DF0E0EE0FFF1FEF5EFF4D61
:10C38000A081B18120E039E10E94567B9A0140E012
:10C3900050E00E942F7B6981A62FB0E00E945D7B58
:10C3A0009B01AC016FE080E00E945D2DC8010E94FE
:10C3B000222D8FE20E94C42C80B1873028F487E1BF
:10C3C0000E94C42C83E70ECF80B18031D8F78AE178
:10C3D0000E94C42C8BE1F4CF86ED9EE20E94222DB8
:10C3E0002091023480E890E0821B910949816F2DF1
:10C3F0009695982F8827979587950E948A2EC80131
:10C4000093CF81ED9EE20E94222D20910334EACF4A
:10C4100086ED9EE20E94222D809109340E94302DEB
:10C42000B5CD81ED9EE20E94222D80910A34F6CF97
:10C430008CEE9EE279CF872DF1CFA0910C34BB27F3
:10C44000A1950CF4B0952AE638E10E94567B9B0139
:10C45000AC016FE080E00E945D2D86E5C3CEA09127
:10C460000F34BB27A1950CF4B09526E33CE0EDCF4B
:10C4700020910E3430E0A7E9B8E90E94DE7A9B01F2
:10C48000AC016FE080E00E945D2D85E2ABCE88E0DC
:10C490008093E0218091FD330E94302D98CF5C9BEA
:10C4A00075CD4CEE5EE26FE0CECE10E480E4898381
:10C4B00089CD612F89810E94BD199981905F9983EF
:10C4C0009038B9F7105F103809F4A5CDE0E1E983A1
:10C4D000F0CF10E1FBCF88E50E94C42C149BC8CD9F
:10C4E0008DE20E94C42C8091E02184508093E02151
:10C4F000BFCD8CE48093E0211092DF218DE20C9B74
:10C5000080E20E94C42C89E597E20E94222D80914E
:10C51000F43325E0829FC0011124099B07C0845495
:10C520009B4D0E94222D8FED9EE2A4CD81529B4D0A
:10C53000F8CF88E50E94C42C149BB8CD8DE20E94F0
:10C54000C42C8091E02184508093E021AFCD8CE415
:10C550008093E02149814093DF218DE2149B80E2AA
:10C560000E94C42C88E697E20E94222D8091F53328
:10C5700055E0859FC0011124119B07C084549B4D39
:10C580000E94222D8FED9EE293CD81529B4DF8CFDC
:10C5900040B195E0499FA0011124425B5B4D698148
:10C5A00080E60E94A92E8AED9EE296CDF09101349C
:10C5B000FB832B9BA5CD629AA3CD09F0B8CD149B2C
:10C5C00008C04B8140954B8310958CB194E089272E
:10C5D0008CB9809106345B81580F5B83A7CD809125
:10C5E000F633809589838091FE339981981B9F83D0
:10C5F0009E3708F4A6CD62983B9B03C00E942A2B6D
:10C600003B980E94A63B0E946B3B8091C20481FF35
:10C6100005C08091C30481110E9454785C990BC0BD
:10C6200080B18B3018F08DB1811105C080B18B3095
:10C6300008F0309BA99A80B18B3028F488B1803201
:10C6400010F00E94332C599902C00C94DD4D0E94C9
:10C650001A270C94DD4D2D9B17C06091013466950F
:10C660006695262F3F813E5F3983432F8F810E943D
:10C67000E91960910134619566956695262F498187
:10C680008F810E94E919B7CF2F9B12C049814D3786
:10C6900048F447EA5EE1629909C0898183508D3789
:10C6A00008F0A9CF48E95EE16299A5CF698188CDFC
:10C6B000898183508A3708F09ECF4DE75EE1F6CF3F
:10C6C0005FEF5F8398CF6FEF6F8396CF92E2909387
:10C6D0001F3D8EE58093203D2FE72093213D109252
:10C6E0001E3D9093243D8093253D1092263D10924F
:10C6F000233D0895CF93DF9390E41092163D9093DD
:10C70000173D1092183D9093193DC0E8D0E00E946B
:10C710001D7A9E01281B310920931A3D30931B3D41
:10C720008D57990B079798F3C0E8D0E00E941D7AC7
:10C730009E01281B310920931C3D30931D3D811122
:10C74000F5CFDF91CF910895CF92DF92EF92FF92D4
:10C75000CF93DF9300D00F92CDB7DEB7FC0191816C
:10C760008281292F280F3327331F359527952B8357
:10C770003C83A3E2BDE33DE3EE31F30711F0AEE10C
:10C78000BDE32481253069F1283089F420911C3DD6
:10C7900030911D3D37FF2CC02091173D3B81231761
:10C7A00048F5911521F091509183815082838DE35A
:10C7B000E332F80739F580911C3D90911D3D97FFBC
:10C7C00006C08091183D9091193D94306CF12496EB
:10C7D000CDBFDEBFDF91CF91FF90EF90DF90CF9084
:10C7E000089520911C3D30911D3D12161306A4F2B0
:10C7F00020E4D4CFE1F2D8F28F37C8F69F5F91835F
:10C800008F5FD4CF3DE3EE31F30709F780911C3DF4
:10C8100090911D3D18161906D4F68091183D9091FF
:10C82000193D81309B479CF24091173D818148170B
:10C8300008F440C082818417E8F180911C3D9091FA
:10C840001D3D22273327281B390B29833A83A091CA
:10C850001A3DB0911B3D20E431E00E94567BC72E6B
:10C86000D82E70931A3D80931B3DA981BA810E94F6
:10C87000567B70931C3D80931D3D8181841306C0BF
:10C88000DA94C0921A3DD0921B3DA1CF82818413CD
:10C8900002C0D394F6CF842F90E02B813C81821B81
:10C8A000930B880F991F8C0D9D1D80931A3D9093BB
:10C8B0001B3D8DCF8C918F5F8D938C918E5F8D936F
:10C8C0008C9182508C932496CDBFDEBFDF91CF91A7
:10C8D000FF90EF90DF90CF900C947A630F931F93AB
:10C8E000CF93DF9300D000D00F92CDB7DEB7809109
:10C8F000173D8F838091193D8E831092E02107E0D0
:10C900000093DF2180EB9BE20E944A318AE0809312
:10C91000E02118E01093DF2180911E3D0E94B43188
:10C920008CE48093E0210093DF2186EA9BE20E9461
:10C930004A3180E68093E0211093DF218091233DEE
:10C940000E94B43120E04091213D6091203D8091D2
:10C950001F3D0E94EE2E20E04091263D6091253D36
:10C960008091243D0E94EE2E8E81835089830F8119
:10C970000150682F802F0E94BD1969818F810E940C
:10C98000BD191F811F5F6981812F0E94BD198E8192
:10C99000825089838F8182508C8369810E94BD1966
:10C9A0008F818E5F8D8369810E94BD198E81815038
:10C9B0008A838F81835089836A810E94BD198F8108
:10C9C0008D5F8B836A810E94BD196E8189810E946F
:10C9D000BD196E818B810E94BD198E818F5F8A8304
:10C9E000682F89810E94BD196A818B810E94BD19BF
:10C9F0008E818E5F8983682F8C810E94BD19698129
:10CA00008D810E94BD198E818D5F8983682F802F53
:10CA10000E94BD1969818F810E94BD196981812F92
:10CA20002796CDBFDEBFDF91CF911F910F910C9460
:10CA3000BD190F931F93CF93DF930E9466630E94EB
:10CA40007A635E98589ACAE1DCEF06EE13E08091B3
:10CA5000A80685FD5E9A84FF0CC090911F3D91153C
:10CA600041F0915090931F3D9091203D91509093B3
:10CA7000203D80FF0CC09091203D9F3740F42091D5
:10CA80001F3D2F5F20931F3D9F5F9093203D87FFA9
:10CA90000CC09091243D911541F091509093243D0C
:10CAA0009091253D91509093253D86FF0CC080913B
:10CAB000253D8F3740F49091243D9F5F9093243D16
:10CAC0008F5F8093253D80911C3D90911D3D81306D
:10CAD00024E092070CF46BC000931C3D10931D3DA5
:10CAE00080911A3D90911B3D813024E092070CF417
:10CAF00066C000931A3D10931B3D80911A3D9091A2
:10CB00001B3D2091163D3091173D280F391F209372
:10CB1000163D3093173D4091183D5091193D60915D
:10CB20001C3D70911D3D460F571F4093183D50937B
:10CB3000193D009709F00CF44AC021303B470CF036
:10CB40004BC00E94492C8EE19DE30E94A46383E2C6
:10CB50009DE30E94A4630E946E648BE18093E021B8
:10CB60002DE02093DF2180911E3D8A3028F05E9ACF
:10CB700088E99BE20E944A318091233D8A3028F067
:10CB80005E9A8AE89BE20E944A310E94A63B0E947C
:10CB90006B3B0E94332C5E9B5ACF5E980E94332CD5
:10CBA0006698589ADF91CF911F910F9108959C3FFD
:10CBB0000CF096CFC0931C3DD0931D3D91CF9C3F70
:10CBC0000CF09BCFC0931A3DD0931B3D96CF09F438
:10CBD000B8CF34300CF0B5CF919581959109809301
:10CBE0001A3D90931B3DADCF0F931F93CF93DF93CF
:10CBF000589A5E980E94492CC4E0D7E002E017E3FF
:10CC0000589B52C05898669B15C066987B99CF5F19
:10CC1000C63008F0C4E07A99DF5FD93008F0D7E079
:10CC2000799B06C0C093223DD093273D0E94196591
:10CC30007D995E9A1093E0211092DF218AEB9BE2AE
:10CC40000E944A311092E0210093DF218BE09DE2A7
:10CC50000E944A318AEF9BE20E944A3184E09DE2C1
:10CC6000C43011F08FEF9BE20E944A311092E02114
:10CC700083E08093DF218BE09DE20E944A3185EFC3
:10CC80009BE20E944A3184E09DE2D73011F08FEFA1
:10CC90009BE20E944A311092E0218FE08093DF21D5
:10CCA0008EEE9CE20E944A310E946B3B0E94A63BA2
:10CCB00088955E9BA5CF589ADF91CF911F910F91D8
:10CCC0000895E6E1FDE380E09CE0DF019C011D9218
:10CCD00021503040E1F7EAE1F9E498E0DF019C01FE
:10CCE0001D9221503040E1F782E0809317418093FC
:10CCF0001641809317458093164522E020931849EA
:10CD00001092194988E0809316498DE180931B4960
:10CD1000808380931B4D80931A4D20931C51109259
:10CD20001D5184E080931A51109220510895CF93A1
:10CD3000C0911E5140911F518C2F90E0439669E2A3
:10CD400070E00E94F97A9C01C82F842F90E04396EE
:10CD50006CE370E00E94F97A482F582F522B503222
:10CD600058F7F90130E2F39FF02DE39FE02DF12910
:10CD70001124E80FF91FEA5EF24C50815111DCCF0B
:10CD800020931E5180931F5181E08083809126085B
:10CD9000909127088B3F910570F0209126083091E3
:10CDA0002708A6EEB0E00E94DE7A672F782F609306
:10CDB000360870933708809120518F5F80932051FF
:10CDC000CF910895EF92FF920F931F93CF93DF932C
:10CDD000EC018C010F5F174FD8018C91853019F051
:10CDE000883009F063C0FE01FC5F208190911F51E3
:10CDF00081E0921720F0291708F080E0880F388131
:10CE000090911E51931708F0BEC08460B0E23B9F22
:10CE1000A0011124FA01EC5EFB4CE20FF11DEF5F63
:10CE2000F64F9081923018F49FE0211101C09EE0EE
:10CE3000FA01E20FF11DE95EF24C4081423010F43C
:10CE40002F3109F49D7F40E2349FF0011124E20F5D
:10CE5000F11DEA50F34C4081423010F4311101C011
:10CE60009B7F50E2359FF0011124E20FF11DEA5C37
:10CE7000F24C2081223010F43F3109F4977F89234E
:10CE80007E01A8E0FA0E811509F482C0F7019081B5
:10CE9000982309F480830E94017AD701EC91F0E095
:10CEA00080FF79C0E152F44DE491EC93DE01AE5F76
:10CEB000B74F8D919D911297F8012081211509F4AA
:10CEC000C1C0FC013197EC0FFD1F8081FC5FE08148
:10CED000F0E28F9FC00111248C5E9B4CE80FF92F6C
:10CEE000F11DEE5FF64F1082ED91FD911297CF018B
:10CEF0000197EC0FFD1FBF0161507109C617D707DD
:10CF000009F04DC0F8014081FE01E80FF91F808152
:10CF1000FC5FE081F0E28F9FC00111248C5E9B4C8E
:10CF2000E80FF92FF11DEE5FF64F4083FE01F85F29
:10CF3000908188819E013C5F943009F446C0E0F501
:10CF4000F90180819130E9F18F5F9230D9F18881C8
:10CF5000F901908150E2859FF0011124EC5EFB4CB9
:10CF6000E90FF11DEE5FF64F5081523018F4892B16
:10CF7000803268F1D8011C92DF91CF911F910F91FF
:10CF8000FF90EF90089509F008F440CF88603ECFFD
:10CF9000D7019C9380CFE153F44DE49186CFFB0100
:10CFA0002291BF0121839F013C5FF90140812F5FE6
:10CFB0003F4FF9014083A2CF8F5F983041F68883BD
:10CFC000C6CF8150F9018083C2CF8150F8CF408312
:10CFD00090911E5188819813CFCF90911F51F901E4
:10CFE00080819813C9CF8D919D9112978130F4E083
:10CFF0009F0710F620E0AC01415051094C0F5D1F16
:10D00000BA017C5F0FC08C01020F111DFA01308143
:10D010000C0F1D1FF8013083FB013081F801FC5F0C
:10D0200030832F5F30912051231768F3830F911DB8
:10D030008D939D93DF91CF911F910F91FF90EF9072
:10D040000C9497668430910508F496CFFC013197D3
:10D05000EC0FFD1F8081FC5FE081F0E28F9FC0013B
:10D0600011248C5E9B4CE80FF92FF11DEE5FF64FFB
:10D0700010828D919D9101979E938E937DCFCF923B
:10D08000DF92EF92FF920F931F93CF93DF9300D025
:10D0900000D0CDB7DEB786E1E82E8DE3F82E1D82F5
:10D0A000FD81FF5FFB838D818E5F8C83ED81ED5F62
:10D0B000E983670102E013E0F1E0FE838E81815095
:10D0C0008A83F60181916F01863018F5843008F06B
:10D0D0006DC0813008F49AC009F449C06A818B811F
:10D0E0000E94BD196A8189810E94BD196E818D815E
:10D0F0000E94BD196E818C810E94BD19602F8B81A9
:10D100000E94BD19602F89810E94BD19612F8D81F8
:10D1100048C08750823010F76A818D810E94BD1906
:10D120006A818B810E94BD196A818C810E94BD1920
:10D130006A8189810E94BD196E818D810E94BD190D
:10D140006E818B810E94BD196E818C810E94BD19F8
:10D150006E8189810E94BD19602F8D810E94BD1949
:10D16000602F8B810E94BD19602F8C8139C06A812C
:10D170008B810E94BD196A818C810E94BD196E81CC
:10D180008D810E94BD196E8189810E94BD19602F19
:10D190008D810E94BD19602F89810E94BD19612F68
:10D1A0008B810E94BD19612F8C812EC06A818D8177
:10D1B0000E94BD196A818B810E94BD196A818C8190
:10D1C0000E94BD196A8189810E94BD196E818D817D
:10D1D0000E94BD196E8189810E94BD19602F8D81C9
:10D1E0000E94BD19602F89810E94BD19612F8D8118
:10D1F0000E94BD19612F8B810E94BD19612F8C8106
:10D200000E94BD19612F89810E94BD19FE81FC5FBA
:10D21000FE830C5F1C5FF13809F050CF8D818C5F6D
:10D220008D83E0E2EE0EF11C803809F039CF2696AE
:10D23000CDBFDEBFDF91CF911F910F91FF90EF9097
:10D24000DF90CF9008950F931F93CF93DF9380913A
:10D2500073008E7F809373008AE09DE3809326089D
:10D260009093270885E0809300080E9461660E94E1
:10D2700097665E98589AC4E0D1E00DE016E2669B8E
:10D2800016C066987D995E9A7C9B65C08091164910
:10D29000813009F051C0C09316497F9B78C08091BE
:10D2A0001A51813009F066C084E080931A51809150
:10D2B0000C0880FF31C0D0930C080E94492C80914B
:10D2C0001749833021F086E191E40E94E266809163
:10D2D0001B51863021F08AE199E40E94E2660E94A7
:10D2E0003F680E94A63B0E946B3B0E94332C8091BA
:10D2F0001749811511F0833079F480911B51811504
:10D3000011F0863049F45E9A1093E0210093DF21FA
:10D310008FEB9BE20E944A315E9BB1CF5E98589A98
:10D320001092000880917300816080937300DF91F8
:10D33000CF911F910F910895823021F488E080935E
:10D340001649ABCF843011F482E0F9CF883009F070
:10D35000A4CF81E0F4CF789BA0CF80911649813093
:10D3600069F3823009F497CF843099F3883009F05B
:10D3700094CFEACF823011F488E097CF843011F453
:10D3800082E093CF883009F092CF81E08ECF7E9BF0
:10D390008ECF80911A51813079F3823009F484CF95
:10D3A000843099F3883009F082CFEACF0F931F932E
:10D3B000CF93DF930E94017A869586958695809318
:10D3C0001E510E94017A86958695869580931F51FD
:10D3D000589A5E980E94492CC4E0D6E002E011E31E
:10D3E000589B5EC05898669B15C066987B99CF5F26
:10D3F000C63008F0C3E07A99DF5FD93008F0D6E094
:10D40000799B06C0C0931749D0931B510E94236992
:10D410007D995E9A1093E0211092DF2189EC9BE2C6
:10D420000E944A311092E0210093DF218BE09DE2BF
:10D430000E944A318AEF9BE20E944A3187EB9EE2CA
:10D44000C33041F084E09DE2C43021F0C53021F4C6
:10D450008FEF9BE20E944A311092E02183E080939B
:10D46000DF218BE09DE20E944A3185EF9BE20E9422
:10D470004A3187EB9EE2D63041F084E09DE2D7301E
:10D4800021F0D83021F48FEF9BE20E944A311092B4
:10D49000E0218FE08093DF218EEE9CE20E944A31F2
:10D4A0000E946B3B0E94A63B88955E9B99CF589A41
:10D4B000DF91CF911F910F91089588950895EC9871
:10D4C0001895EC9A189516F068941895E8941895A4
:10D4D000F8948FB7282F207486FD2CE08091200BC4
:10D4E0009091210B80313EE0930748F430E08C337B
:10D4F000910548F431B922B980B9789408952F5F25
:10D5000080519E40EFCF3F5FCC97F1CF42B14C307E
:10D5100008F04C5021B130E02F5F3F4F5CE3529F49
:10D52000C001539F900D112460E17EE0469F900161
:10D53000479F300D1124820F931F01978093280B72
:10D540009093290B80EF80930C0B82E08093070B64
:10D5500008950F93CF93DF9304B1C091E0210A3077
:10D5600098F10A50DCE0DC0F4AE959E164E08C2FC5
:10D570000E94033223E044E064E088E08C0F0E94C4
:10D58000D631E02FF0E0EE0FFF1FE55DFD4E459137
:10D59000559164E08D2F0E940332EC9B0CC08EB13C
:10D5A000853049F48091E02147E1480F01E027E30D
:10D5B00065E30E945A2F8091E021855E8093E021EF
:10D5C000DF91CF910F910895D6E0DC0F23E048E181
:10D5D00064E08C2FD4CF0F931F93CF93DF9300D0B1
:10D5E000CDB7DEB705B18091E0218A8385B188335C
:10D5F00028F4045DE1E019E01B8208C00853E2E072
:10D6000010E0FACF8B818F5F8B830A500A30D0F7FE
:10D61000F0E0EE0FFF1FE55DFD4E4591559164E092
:10D620008A810E940332E12FF0E0EE0FFF1FE55DDB
:10D63000FD4E459155918A81825F898364E00E9405
:10D6400003328B81E82FF0E0EE0FFF1FE55DFD4E0A
:10D65000459155911A81145E64E0812F0E94033236
:10D66000E02FF0E0EE0FFF1FE55DFD4E4591559177
:10D670008A81865D8B8364E00E940332EC9B20C02C
:10D680008EB18630E9F44A81455F01E027E365E326
:10D690008A810E945A2F4A81475E27E365E3898188
:10D6A0000E945A2F4A81495D27E365E3812F0E943A
:10D6B0005A2F4A814B5C27E365E38B810E945A2FE6
:10D6C0008091E021875C8093E0210F900F900F9074
:10D6D000DF91CF911F910F910895CF938093E02117
:10D6E0006093DF21C7B188E59FE25A9B1BC087B1D9
:10D6F0008C3008F08C50811101C08CE06A9915C003
:10D700000E94B4318AE30E94FD3088B10E949631B4
:10D7100080E69FE26A9906C08FEE9BE2CC3010F45F
:10D7200082EF9BE2CF910C944A318C2FE9CF0F937B
:10D73000CF93DF936C9B58C0CEB1C11155C0659B90
:10D7400025C0659802B16A9906C00C3008F4D8C1AA
:10D750000C5009F4D7C10431B8F1045148E059E143
:10D7600065E080E00E940332E02FF0E0EE0FFF1F43
:10D77000E15CFA4E4591559165E089E10E940332E2
:10D7800045E355E167E081E30E94033201B10A30CD
:10D7900040F5EC2FF0E0EE0FFF1FE15CFA4E4591F3
:10D7A000559165E087E30E940332E02FF0E0EE0F31
:10D7B000FF1FE15CFA4E4591559165E080E5DF91F0
:10D7C000CF910F910C9403320A3020F00A504BEBAA
:10D7D00059E1C6CF26E046E165E080E00E94D631FF
:10D7E000C3CFCF5F0A50D3CF659904C08EB18115E6
:10D7F00009F466C065986A9B48C121E040E169E090
:10D8000089E60E94D63102B16A9906C00C3008F44C
:10D810007BC10C5009F47AC1043108F442C10451AF
:10D8200048E059E169E080E00E940332E02FF0E037
:10D83000EE0FFF1FE15CFA4E4591559169E089E1D9
:10D840000E940332EC9B10C08EB1833069F401E07A
:10D8500027E745E163E780E00E945A2F27E74EE281
:10D8600063E789E10E945A2F8AB1811509F432C118
:10D87000649905C08AB190911634981779F048EFF1
:10D8800051E160E082E00E940332CAB1C15065E01C
:10D8900004E0C11113C18AB18093163460E08AE4B8
:10D8A0000E946D6B86E78093E0211092DF215A9BE6
:10D8B00018C1009902C05F9914C180E80E94FD3030
:10D8C000C1B1E0E0CA3008F00EC1F0E0EE0FFF1F7A
:10D8D000E15CFA4E4591559169E087E30E9403327D
:10D8E000EC2FF0E0EE0FFF1FE15CFA4E45915591F1
:10D8F00069E080E50E940332EC9B10C08EB182305B
:10D9000069F401E027E74CE463E787E30E945A2FBC
:10D9100027E745E663E780E50E945A2F89B1811524
:10D9200009F4E4C040B122E06CE088E60E94503285
:10D93000EC9B10C08EB1813069F401E024E742E72E
:10D9400062E788E60E945A2F24E74FE762E785E7FF
:10D950000E945A2F649904C08EB1843008F4D8C054
:10D96000649845E355E16BE081E30E94033288E26D
:10D970008093E02182E08093DF2186B12AE0829FBC
:10D98000C0011124865C924D0E944A3181E080934F
:10D99000E02168990EC00E94EB6A4FE352E165E016
:10D9A0008091E0210E9403328091E021885F809382
:10D9B000E02169990EC00E94A96A4FE352E165E037
:10D9C0008091E0210E9403328091E021885F809362
:10D9D000E021C3B1E0E0CA3008F08FC0F0E0EE0F04
:10D9E000FF1FE55DFD4E4591559164E08091E0217A
:10D9F0000E940332EC2FF0E0EE0FFF1FE55DFD4EBD
:10DA0000459155918091E02164E0825F0E9403324C
:10DA1000EC9B15C08EB1843091F48091E0214BE0F5
:10DA2000480F01E027E365E30E945A2F8091E0212F
:10DA300049E1480F27E365E3825F0E945A2F8091F6
:10DA4000E021835E8093E021699B0CC04FE352E1AB
:10DA500065E00E9403328091E021885F8093E0219D
:10DA60000E94A96A689B54C04FE352E165E080912F
:10DA7000E0210E9403328091E021885F8093E021C1
:10DA8000DF91CF910F910C94EB6A45E152E10FB613
:10DA900006FC02C040E052E169E089E60E940332E0
:10DAA000B2CE0A3020F00A504BEB59E1BBCE26E053
:10DAB00046E169E080E00E94D631B8CEDFEFD60FB4
:10DAC000802F0E94BD19D13011F40F5FD5E0C150F5
:10DAD0006D2FDFCE44EE51E160E082E00E94033220
:10DAE000DDCE80E2EBCEEF5FCA50ECCE23E048E122
:10DAF0006CE088E60E94D6312DCFEF5FCA506BCF25
:10DB0000011162CE0CE062CE0111CBCF0CE0CBCF85
:10DB1000DF91CF910F910895CF92EF92FF920F93E3
:10DB20001F93CF93DF9300D0CDB7DEB78EB18111B5
:10DB30000E94A63B0E94492C64988DB1982F907149
:10DB4000998384FDAFC08AE38093E02181E08093D4
:10DB5000DF218CE00E94B43182E58093E02102E075
:10DB60000093DF2181E00E94B43184E68093E021BC
:10DB700035E0E32EE092DF2182E00E94B4318CE6B2
:10DB80008093E02118E01093DF2183E00E94B431FC
:10DB900094E69093E0218BE08093DF2184E00E9463
:10DBA000B43180E58093E0214DE0F42EF092DF2146
:10DBB00085E00E94B43187E38093E0215EE0C52ECA
:10DBC000C092DF2186E00E94B4318FE18093E02192
:10DBD000F092DF2187E00E94B4319BE09093E02136
:10DBE0009093DF2188E00E94B43183E08093E021AC
:10DBF0001093DF2189E00E94B431C092E021E092CD
:10DC0000DF218AE00E94B4318EE18093E02100930D
:10DC1000DF218BE00E94B4316FE389810E94407A5A
:10DC2000082F6FE389810E94317A8A836CE38981AE
:10DC30000E94407A182F6CE389810E94317A6FE349
:10DC4000262F201B4A81415C611B815C0E94E919DF
:10DC500089818F5F89838C33F9F66AE08AE20E94BA
:10DC60006D6B84E38093E02184E08093DF21699BE6
:10DC700006C083B10E94302D80E20E94C42C84B182
:10DC80008150990B880F991F880F991F8058924DCA
:10DC90000E94222D699906C080E20E94C42C83B1A3
:10DCA0000E94302D90B1998381B18A83809315347D
:10DCB00082B1809314348C3008F08C50282F220FBE
:10DCC000220F280F8A816CE00E94ED7A082F020F44
:10DCD0006C9923C08CE38093E0218BE08093DF215B
:10DCE0005A9B87C0009902C05F9983C080E80E9458
:10DCF000FD3089B1811589F066E389810E94407AFF
:10DD0000182F66E389810E94317A2FE3211B4FE3AC
:10DD1000480F6FE38FE30E94E91964E2802F0E94AD
:10DD2000407AE82E64E2802F0E94317A898395E060
:10DD3000900F9B8368E0892F0E94407AF82E68E05C
:10DD40008B810E94317A182F095C68E0802F0E9435
:10DD5000407AC82E68E0802F0E94317A9FE39E1996
:10DD6000E92E0981015C2FE32F194FE3410F6FE387
:10DD70006C19CC24C394815C0E94802F62E38A8159
:10DD80000E94407AE82E62E38A810E94317A082F4D
:10DD90001A811C5F68E0812F0E94407AF82E68E0AB
:10DDA000812F0E94317AC82E8A81885C898368E03D
:10DDB0000E94407A182F68E089810E94317A9FE39F
:10DDC0009E19E92E015C2FE32F194FE34C0D6FE3F1
:10DDD000611BCC24C394815C0E94802F0F900F9014
:10DDE0000F90DF91CF911F910F91FF90EF90CF9007
:10DDF000089580E27CCFAF92BF92CF92DF92EF92F4
:10DE0000FF920F931F93CF93DF935E9830EFC32E53
:10DE1000AA24A394F12C00E0D12C42E0E42EC0E02F
:10DE2000D0E010E0BA2C669B42C066987E990B2524
:10DE30007B991F5F7A99DF5FDC3308F0D0E0799936
:10DE4000CF5FCC3308F0C0E08FB180FF2CC001154C
:10DE500009F49FC0D394E39480E1E81610F023E026
:10DE6000E22EB092E021E092DF2181E59FE20E9464
:10DE70004A318D2D0E9496318AE30E94FD3014367E
:10DE800018F480E20E94FD30812F0E9496318AE3CF
:10DE90000E94FD308D2F0E9496318AE30E94FD3052
:10DEA0008C2F0E9496317D995E9A80EFC82E0115C5
:10DEB00009F480C0EC9B03C0F11409F480C0EC9914
:10DEC00013C081E0F81210C0C150F12CCF3F61F4B3
:10DED000D150F12CCBE3DF3F39F4111509F462C0C6
:10DEE0001150F12CCBE3DBE3A11461F00E94492C2B
:10DEF00084E08093E0218FE08093DF218CE39FE238
:10DF00000E944A3183E38093E021B092DF21011522
:10DF100011F080E2EC998AE30E94FD3081E5809364
:10DF2000E021B092DF21011511F080E2EC998AE343
:10DF30000E94FD3022E04C2F60E086E50E945032C6
:10DF400022E04D2F60E088E30E94503223E0412F11
:10DF500060E08DE00E9450320E946B3B0E94A63B25
:10DF600080914009811102C00E945D6A8BB186FBDD
:10DF7000AA24A6F886FF57CF5E98DF91CF911F9114
:10DF80000F91FF90EF90DF90CF90BF90AF900C94E7
:10DF9000492C8170A82ED12CC0E0D0E010E092E096
:10DFA000E92E81CF8AED92E30E94507AF12CC0E0F5
:10DFB000D0E09ACFCA9409F097CF5E9A95CFF02E11
:10DFC00093CFAF92BF92CF92DF92EF92FF920F93D7
:10DFD0001F93CF93DF93809173008C7F80937300A6
:10DFE00080EC8093800110922008109221088FE12C
:10DFF0009EE4809326089093270810926008109260
:10E0000061088FE697E180936608909367085E98B1
:10E0100090EFD92EBB24B394E12CC2E0A12C00E0F8
:10E02000D0E010E0CB2C27E2F22E669B46C066982B
:10E030007E9B09C080914008811509F49BC0109215
:10E040000008109240088FB180FF33C090914008C3
:10E05000911509F495C0E394CF5FC03108F0C3E097
:10E0600086E08093E021C093DF2187E39FE20E9456
:10E070004A318E2D0E9496318AE30E94FD3014367B
:10E0800018F480E20E94FD30812F0E9496318AE3CD
:10E090000E94FD308D2F0E9496318AE30E94FD3050
:10E0A000802F0E9496318AE30E94FD308A2D0E94C3
:10E0B00096317D995E9A80EFD82EB1100E94492C3E
:10E0C000F092E021C092DF218AE30E94FD3085E4D6
:10E0D0008093E021C092DF218AE30E94FD3083E635
:10E0E0008093E021C092DF218AE30E94FD3022E08C
:10E0F0004A2D60E088E60E94503222E0402F60E026
:10E100008AE40E94503222E04D2F60E08CE20E94AF
:10E11000503223E0412F60E081E00E9450320E94A3
:10E12000A63B0E946B3B8091400881113AC0DA9473
:10E1300009F45E9A0E94A63B0E945D6A8BB186FB41
:10E14000BB24B6F886FF71CF5E981092000810923B
:10E15000400880917300836080937300DF91CF91BA
:10E160001F910F91FF90EF90DF90CF90BF90AF90F5
:10E170000C94692CC092000888E08093400863CF1B
:10E1800010922008109221081092600810926108E5
:10E190008170B82EE12CA12C00E0D0E010E0C2E0AC
:10E1A00088CF80914C0880FF08C08FEF80934C0887
:10E1B000DF5FDC3310F01F5FD0E08091600890914A
:10E1C000610800E08436910510F4A82EB7CF0F5FE8
:10E1D00084569109F7CF0F931F93CF93DF93CDB759
:10E1E000DEB76097CDBFDEBF40E150E069E07DE083
:10E1F0008E010F5F1F4FC8010E94F07B86B18F5FB9
:10E20000602F912F873008F080E046B120E430E0A5
:10E21000F90102C0F595E7954A95E2F74E2F02C045
:10E22000359527958A95E2F7322F5A98659AE62F09
:10E23000F92FBE016F5E7F4F228127FF55C080817D
:10E240009181232339F122B1281303C021B1921700
:10E2500018F022B18217F0F45A9907C05A9A87B978
:10E2600098B923812093173415C052B127B15213A6
:10E2700004C021B158B1521720F022B157B1521742
:10E2800048F427B1281303C028B1921740F327B1EF
:10E29000821728F32281242339F122B1281303C0E5
:10E2A00021B1921718F422B12817F0F45A9907C037
:10E2B0005A9A87B998B983818093173415C052B19F
:10E2C00027B1521304C021B158B1521790F322B1B3
:10E2D00057B1521770F327B1281303C028B1921712
:10E2E00040F327B1821728F33496E617F70709F0B1
:10E2F000A3CF6096CDBFDEBFDF91CF911F910F916D
:10E3000008958F929F92AF92BF92CF92DF92EF9239
:10E31000FF920F931F93CF93DF93CDB7DEB7639731
:10E32000CDBFDEBF40E150E069E07DE0CE01019667
:10E330000E94F07B9BB05E98639A10E0812C64E0B1
:10E34000E62E669B79C06698639A2CE329B90E94F1
:10E350006B7A7F99A89A212F30E07E9902C0789B32
:10E3600017C088E08816A0F4F901EE0FFF1FEE0F2A
:10E37000FF1FCE010196E80FF91F928140E850E09F
:10E38000082C02C0559547950A94E2F7942792838A
:10E39000C901880F991F880F991F7E9B0AC0E8E06A
:10E3A0008E129AC0FE013196E80FF91F20812F5F6F
:10E3B0002083789B0AC0E8E08E12A4C0FE0131964B
:10E3C000E80FF91F208121502083FE013196E80FCC
:10E3D000F91F2081283108F01082FE013196E80FE4
:10E3E000F91F21812C3308F01182FE013196E80FCC
:10E3F000F91F83818A3008F013827B9B06C08A94C0
:10E400008BE0881610F03AE0832E799B05C0839448
:10E410009BE0891608F0812C7F9B04C011501430BA
:10E4200008F013E07A9902C07C9B04C01F5F14308F
:10E4300008F010E07D995E9A63997AC0612F629529
:10E44000660F607E8110EAC026E0260F01E04DE2F3
:10E4500082E00E94232F0E946B3B0E94A63B6099A2
:10E46000669A80914009811115C18091000981113E
:10E4700011C163990FC166990DC189B1815089B9E4
:10E4800087E0809348000E945D6A5E9903C089B16D
:10E49000811157CF40E150E069E07DE0CE01019667
:10E4A0000E94947B9BB80E946B7A0E94EB705E98EE
:10E4B0008CE389B90E94492C6396CDBFDEBFDF9102
:10E4C000CF911F910F91FF90EF90DF90CF90BF9071
:10E4D000AF909F908F900895F9E08F1208C0FE01D1
:10E4E0003196E80FF91F21812F5F218362CF2AE047
:10E4F00082125FCFFE013196E80FF91F23812F5F53
:10E50000238357CFF9E08F1208C0FE013196E80F40
:10E51000F91F21812150218358CF2AE0821255CF43
:10E52000FE013196E80FF91F2381215023834DCF3F
:10E5300063980E94492CE092E021EFE0E093DF2114
:10E5400082E29FE20E944A31CE0101966C0197E07F
:10E55000998B21E3B22EF12CE092E021F092DF21A1
:10E560008BE19FE20E944A318B2D0E94FD308AE3AD
:10E570000E94FD30F601828187FF09C001E02989F0
:10E5800021504DE26989675082E00E945A2F5A9AC1
:10E59000F601808187B9818188B96F2D89E30E9456
:10E5A0006D6BF0E7F093E021F092DF2180E80E94AC
:10E5B000FD30F6018381805D0E94FD30E092E02114
:10E5C00081E08F0D8093DF2185E29DE20E944A3138
:10E5D000F989F85FFB8B22E02A8B90E4A92EF601E3
:10E5E00082818A2141F001E02B894A89425F698951
:10E5F0008A890E945A2FA694FA89FE5EFA8BF03817
:10E6000071F724E0F20EB39484E0C80ED11C99890E
:10E61000905E998BE0E1FE129FCF10CFF8E08F164D
:10E6200070F48FEF880D22E1829F802D11242FE05E
:10E63000260F40E1480F695F01E08E5F0ACF26E0B8
:10E64000260F88E0881204C001E045E488E301CF8A
:10E6500099E001E047E589E4891609F4FACE4CE730
:10E660008EE60E94232F809140098111F4CE24E090
:10E67000129FF0011124CE010196E80FF91FE381EA
:10E68000F0E0EE0FFF1FE153F04D859195910E9450
:10E69000507AE1CE80914009811509F4F6CE81E0EF
:10E6A000F0CEFC018581982F20E028130EC06481F4
:10E6B0006150770B40E050E02370461757075CF03D
:10E6C00086E0890F8730B0F40895322F337009F453
:10E6D0009F5F2F5FEACFFA01ED59F04DE4919E0F55
:10E6E000413011F4211521F09C514F5F5F4FE5CF70
:10E6F0009B51FBCF8750E6CF85B190E025B19217B3
:10E7000078F020E030E044B14150550B2417350734
:10E710006CF093B19250980F9730C0F496B9089569
:10E72000292F237009F48F5F9F5FE8CFF901ED591E
:10E73000F04DE4918E0F213019F495B1937021F0D2
:10E740008C512F5F3F4FDFCF8B51FBCF9750E4CFE2
:10E75000DC0114962C911497422F4150550BFA016D
:10E76000ED59F04DE491223029F415968C91837087
:10E7700009F4EF5F8E2F08951F920F920FB60F923C
:10E7800011240BB60F922F933F934F935F936F9388
:10E790007F938F939F93AF93BF93CF93EF93FF9309
:10E7A0008091280B9091290BCC968093280B909305
:10E7B000290B8091280B9091290B803C984A30F0CE
:10E7C0008BE390E08093280B9093290B10B881B1D4
:10E7D0008F5F81B98AB1811105C00E948A408AB9D0
:10E7E0008AE589B981B18C3390F111B882B18F5F1C
:10E7F00082B980E00E948A408AB90E94EB7082B19F
:10E800008831F8F0649A12B886B18F5F86B986B104
:10E81000873008F016B883B18F5F83B9C3B180E049
:10E8200090E00E94A8738C1760F491E093B984B1D2
:10E830008F5F84B984B18D3020F094B985B18F5F3A
:10E8400085B96F9B04C087EE92E30E94507A639A69
:10E85000FF91EF91CF91BF91AF919F918F917F9158
:10E860006F915F914F913F912F910F900BBE0F9041
:10E870000FBE0F901F901895F89488B18C3308F054
:10E8800018B887B1883108F017B880B18F3F11F4FC
:10E890008BE380B980B18C3308F010B881B18F3F21
:10E8A00031F48BE381B982B1815082B9659A81B12B
:10E8B0008C3328F011B882B18F5F82B9659A82B12A
:10E8C0008F3F11F487E182B982B1883108F012B824
:10E8D00084B1811102C08CE084B984B18D3010F014
:10E8E00081E084B980E090E00E94A87393B1911117
:10E8F00001C083B993B1891710F481E083B985B160
:10E900008C3908F015B822B1E8942C3010F06894D6
:10E910002C5041B130B160E17EE0269FC001279FBD
:10E92000900D11242CE3429F800D911D1124830F23
:10E93000911D8093200B9093210B0E947C730E9469
:10E94000866A78940895CF93DF931FB81EB889E143
:10E950009DE00E94FC7B8DB980E00E948A408AB9CC
:10E96000109216348CE389B90E94686A0E94E33BD6
:10E970000E947C730E94EB700E940E3B5E98639A2B
:10E98000649A659A0E942B3CCCE3D1E0669B3BC025
:10E99000C9B966988EB18111A9C07D9B02C05F9BE9
:10E9A0005E9A7B990E94E16F7A990E94FB6E799939
:10E9B0000E9481717E9B09C06B9904C08DB190E16A
:10E9C00089278DB96B980E94692C789B07C06B9B37
:10E9D00004C08DB190E189278DB96B9A7F99A89A6F
:10E9E0007C9B09C0609B07C081E08EB960986C99E0
:10E9F0000E94692C1FB85F9B05C00E94EB700E94AB
:10EA00006B7A5F98639A8EB1811109C0639907C0D0
:10EA1000EC9B03C089B1811102C05F9B44C0639825
:10EA200089B1811519F089B1815089B997B182B145
:10EA30009813C8C098B181B19813C4C05A9BC2C082
:10EA400080B1823008F45F9A5F9B0FC080914009CB
:10EA500081110BC0E0911734F0E0EE0FFF1FE1537E
:10EA6000F04D859195910E94507A8CE389B90E946E
:10EA7000686A6B9BADC00E948C6D0E94A63B0E9491
:10EA80006B3B89B1811539F08EB1811104C0649A54
:10EA9000659A0E94332C8EB1811529F089B18111BC
:10EAA00002C01EB8639A6099669A809140098111EC
:10EAB00092C08091000981118EC063998CC06699C3
:10EAC0008AC00E94A63B87E0809348000E945D6A4E
:10EAD0005E9B5CCF6DB189E19DE00E94117C81E07D
:10EAE0008EB988E789B9DF91CF9108959EB17D995C
:10EAF0001EB87C9B07C08EB18F5F8EB98EB18730F8
:10EB000008F01EB88EB1891729F06C990E94692C03
:10EB10000E94EB70F8948EB18430E1F148F48230B9
:10EB200011F1833059F1813099F00E943C7463CF28
:10EB30008530E1F18630C9F7649A7E9B03C085B1C8
:10EB40008F5F85B9789BF1CF85B1815085B9EDCFC5
:10EB50007E9B03C080B18F5F80B9789BE6CF80B188
:10EB6000815080B9E2CF7E9B03C081B18F5F81B9B4
:10EB7000789BDBCF81B1815081B9D7CF659A7E9BDD
:10EB800003C082B18F5F82B9789BCFCF82B18150B1
:10EB900082B9CBCF649A7E9B03C083B18F5F83B968
:10EBA000789BC3CF83B1815083B9BFCF649A7E9BDA
:10EBB00003C084B18F5F84B9789BB7CF84B1815093
:10EBC00084B9B3CF5F9B53CF0E94EB705F984FCF58
:10EBD0000E94976B52CF80914009811509F478CF3C
:10EBE000D093480073CFCF92DF92EF92FF920F93B2
:10EBF0001F93CF93DF9300D000D00F92CDB7DEB735
:10EC000083B18C8384B18D8385B18E8386B18F83EC
:10EC10005E98639A639B54C063980E94492C4CE1B0
:10EC20004093E0211092DF212D812150330B4BE0E6
:10EC3000429FC001439F900D11248055924D0E9428
:10EC40004A318E81883308F08CC087E19FE20E94B0
:10EC50004A318E81845D0E94963184E08093E02168
:10EC600042E04093DF2185E29DE20E944A311BE1B0
:10EC700020E0412F6EE781E00E94EE2E105F1B38EE
:10EC8000B9F711E02BE7412F6BE1812F0E94E919C1
:10EC90001E5E1139B9F7CE0101960E945173E82E1C
:10ECA000ED81E150FF0BED59F04DF49084E0D82E4A
:10ECB00011E0F11608F05CC00E946B3B0E94A63B7D
:10ECC000669B3FC06698639A7F9B06C08E818C3995
:10ECD00010F48F5F8E83A89A7C9B05C08E8181156E
:10ECE00011F081508E837B9B05C08C81823010F0A7
:10ECF00081508C83799B09C01C81CE0101960E94B2
:10ED0000A873181710F41F5F1C837A9B08C083B187
:10ED10008C8384B18D8385B18E8386B18F83789BFC
:10ED200006C08D81823008F463C081508D837E9B44
:10ED300006C08D818C3008F063C08F5F8D837D9914
:10ED40005E9A0E945D6A5E9B65CF2796CDBFDEBF4F
:10ED5000DF91CF911F910F91FF90EF90DF90CF90B7
:10ED6000089583E19FE20E944A318E81885373CFD8
:10ED700087E0E81203C0D394D394E12C42E1E49EEF
:10ED8000C02C112485E08C0D8093E021D092DF21EE
:10ED9000812F0E94963183B1E394811316C085B10F
:10EDA0009E81981312C084B19D8198130EC06D2D61
:10EDB000660F660F660F2AE0260F645001E042E1FD
:10EDC0004C0D82E08C0D0E945A2F8C8181130EC055
:10EDD0006D2D660F660F660F29E0260F41E14C0D81
:10EDE000635001E083E08C0D0E94232F1F5F61CFF1
:10EDF0008E81811509F49BCF81508E838CE096CF54
:10EE00008E818C3908F09BCF91E09D838F5F8E833C
:10EE100096CFDC0115963C91159740E050E0BA0181
:10EE2000CA0143175105A8F014964C911497E3E6D4
:10EE3000FFE221E033702417E8F013962C91215063
:10EE4000330B032E000C0008620F731F801D901DF2
:10EE50000895E42FE370F0E0EF2B39F063597E4F13
:10EE60008F4F9F4F4F5F5F4FDCCF62597E4F8F4F69
:10EE70009F4FF8CF5491650F711D811D911D223058
:10EE800031F4311104C06F5F7F4F8F4F9F4F2F5F61
:10EE90003196D1CFCF92DF92EF92FF92CF93DF9353
:10EEA0000F920F92CDB7DEB769837A830E940977FC
:10EEB0006B017C0189819A810E9409776C157D051F
:10EEC0008E059F0560F4C601861B970B0F900F906F
:10EED000DF91CF91FF90EF90DF90CF900895CB011D
:10EEE0008C199D09F3CFFF920F931F93CF93DF935C
:10EEF000EC011B810C81FD801F5F0E94A8738117AC
:10EF000030F40F5F0D3010F0F39401E011E01B833B
:10EF10000C83FD82DF91CF911F910F91FF90089597
:10EF2000CF93DF93EC018B81815059F48C819D81CB
:10EF3000815011F491508CE08C839D83CE010E940E
:10EF4000A8738B83DF91CF910895CF93C82F883317
:10EF500048F480E19FE20E944A318CE28C0FCF910D
:10EF60000C9496318DE09FE20E944A3188ECF6CFF6
:10EF70001F93CF93DF93FA01309769F513B1D4B1A2
:10EF8000C5B18093E0216093DF21689906C08C2F82
:10EF90000E94A5778FE20E94FD30699906C08D2FEF
:10EFA0000E9496318FE20E94FD30812F0E9496319F
:10EFB000699B06C08FE20E94FD308D2F0E94963122
:10EFC000689B0DC08FE20E94FD308C2FDF91CF91A6
:10EFD0001F910C94A5771381D481C581D2CFDF9185
:10EFE000CF911F910895982F82B16A9906C08C30F5
:10EFF00008F08C50811101C08CE09093E021609367
:10F00000DF210E94B4318AE30E94FD3081B10E9469
:10F0100096318AE30E94FD3080B10E9496316A9950
:10F0200009C08FEE9BE20FB606FC02C082EF9BE2A6
:10F030000C944A310895292F30E02230310539F1FE
:10F040002330310559F021303105A1F482E190E0FF
:10F050002DEB3FE2FA01208331830895282F30E021
:10F06000813061F02230310579F0E9E9FFE22115C4
:10F07000310531F080E090E020E0ECCFEFE7FFE2F7
:10F08000849190E09F01E6CFEFE6FFE2F9CF80E2C6
:10F0900090E02DE93FE2DECFE0E2F0E28287938765
:10F0A00080858D79808708951F93CF93DF93C0E586
:10F0B000D0E084E08E838CE10E94DA3BE0E6F0E071
:10F0C00083838BE1858387EB868311E010838881BE
:10F0D000826088838AE10E94DA3BC0ECD4E08AAF88
:10F0E0008BE10E94DA3B8BAF83E080934400E0E247
:10F0F000F0E2EE83FF831B82108293E491832BE482
:10F1000034E52483358322E0208791872BE834E59A
:10F110002487358792E2908F93EA918F26E331E539
:10F12000248F358F108A918B2FED30E2248B358B15
:10F13000128A138A20E031E0268B378B91EC98837A
:10F1400092E4988789871983DF91CF911F91089561
:10F15000FC01962FABE8B4E5911104C0862F90E036
:10F160000C944C78915084918D933196F5CF1F92E9
:10F170000F920FB60F9211240BB60F922F933F935D
:10F180004F935F936F937F938F939F93AF93BF93AF
:10F19000EF93FF938091C20480FF04C01092C004DB
:10F1A0000E9454788FEF8093CA04FF91EF91BF9132
:10F1B000AF919F918F917F916F915F914F913F910F
:10F1C0002F910F900BBE0F900FBE0F901F901895B0
:10F1D0001F920F920FB60F9211240BB60F921F932E
:10F1E0002F933F934F935F936F937F938F939F934F
:10F1F000AF93BF93EF93FF93CF93DF930F920F9251
:10F20000CDB7DEB7AA9A8091202084FF97C0809165
:10F210004B54807609F088C0E0914C54EA3008F0F5
:10F2200045C0F0E08827E55FF2488F4F0C944E7B95
:10F2300010928B5410928C5482E090E00E944C7893
:10F2400035C080E090E0FACF10914D541F77809147
:10F2500020208D7E8093202080E090E00E944C78DA
:10F260008091282085FFFCCF1093C30483E0111107
:10F2700001C082E080934A5419C0AE014F5F5F4FD6
:10F2800060914F5480914D5490914E540E941B7840
:10F29000009761F06091515470915254861797070E
:10F2A00008F4682F89819A810E94A8788091202093
:10F2B0008D7C809320201092C50483E08093CC0441
:10F2C000AA980F900F90DF91CF91FF91EF91BF918E
:10F2D000AF919F918F917F916F915F914F913F91EE
:10F2E0002F911F910F900BBE0F900FBE0F901F908C
:10F2F00018958091495480938B5481E090E09ECF83
:10F3000080E090E00E944C7880914D548093495465
:10F3100080914954811511F084E0ACCF8091C304F1
:10F320008111FACF81E0A6CF803409F0BFCF61E030
:10F3300080914C540E94A63390E080CF8091202091
:10F3400085FF04C0809120208D7DB3CF8091302037
:10F3500085FFB1CF109232201092332080E091E0EF
:10F36000809336209093372080913020897C809341
:10F370003020A1CF0F93CF93DF930F92CDB7DEB79D
:10F380009C018FB78983F8941BBEF90108ED04BF77
:10F39000608389818FBF0F90DF91CF910F91089586
:10F3A00090E8980F12F491E8980F892F859580586E
:10F3B0000895813428F0803C28F4880F80580895FF
:10F3C00080E008958FEF0895982F80E3890F8A33A6
:10F3D00010F087E3890F08954091CD545091CE5499
:10F3E0006091CF547091D054480F591F611D711D09
:10F3F0004093CD545093CE546093CF547093D054D7
:10F4000008952091CD543091CE544091CF545091D5
:10F41000D054A5E5B2E60E945D7BDC01CB01875E9E
:10F42000994CAF4FBF4F8093CD549093CE54A0933F
:10F43000CF54B093D0548B2F08954091CD54509118
:10F44000CE5425E532E6429FC001439F900D529F66
:10F45000900D112401968093CD549093CE54892F12
:10F4600008958C3358F4E82FF0E0E950FD4C2491D6
:10F47000A60307FC1394812D112408958C53F1CF1A
:10F48000815F8C3358F4E82FF0E0E950FD4C249173
:10F49000A60307FC1394812D112408958C53F1CFFA
:10F4A0008093CB549093CC54E0E7F0E085818E7F3D
:10F4B000858384818D7F848382E08093040AE0E4E5
:10F4C000F9E010A211A281E090E086A397A38683C1
:10F4D0008EE080830895E0E0FAE010821182E0E49B
:10F4E000F9E01082AC98AD981682E0E7F0E08581F3
:10F4F0008160858384818260848308951F920F9246
:10F500000FB60F9211240BB60F922F933F934F9388
:10F510005F936F937F938F939F93AF93BF93EF937B
:10F52000FF93E091CB54F091CC5484919F012E5FD6
:10F530003F4F2093CB543093CC543196E4918115B6
:10F54000D1F190E08093660990936709E11561F12C
:10F5500081E28093010AE093270AE093260A109241
:10F56000200A1092210AE695E0932B0AE093280ADC
:10F5700080914000811116C084E08093000AFF91C1
:10F58000EF91BF91AF919F918F917F916F915F911B
:10F590004F913F912F910F900BBE0F900FBE0F9088
:10F5A0001F90189585E0E9CF1092010A1092000A89
:10F5B000AC98AD98E4CF0E946B7AE1CFA29FB001E6
:10F5C000B39FC001A39F700D811D1124911DB29F97
:10F5D000700D811D1124911D0895992778E0880FE1
:10F5E000991F961708F0961B881F7A95C9F7809582
:10F5F000089597FB072E16F4009407D077FD09D0E5
:10F600000E94707B07FC05D03EF4909581959F4F3A
:10F610000895709561957F4F0895A1E21A2EAA1B57
:10F62000BB1BFD010DC0AA1FBB1FEE1FFF1FA217B2
:10F63000B307E407F50720F0A21BB30BE40BF50BAF
:10F64000661F771F881F991F1A9469F76095709538
:10F65000809590959B01AC01BD01CF010895052EC9
:10F6600097FB1EF400940E94467B57FD07D00E9432
:10F670000D7B07FC03D04EF40C94467B50954095CF
:10F68000309521953F4F4F4F5F4F0895909580954E
:10F69000709561957F4F8F4F9F4F0895EE0FFF1F1D
:10F6A000881F8BBF0790F691E02D19940E94DE7A97
:10F6B000B7FF0895821B930B08950E94DE7AA59FE1
:10F6C000900DB49F900DA49F800D911D112408955D
:10F6D000B7FF0C945D7B0E945D7B821B930B0895AA
:10F6E000AA1BBB1B51E107C0AA1FBB1FA617B70768
:10F6F00010F0A61BB70B881F991F5A95A9F7809584
:10F700009095BC01CD010895FB01DC0102C005907C
:10F710000D9241505040D8F70895DC0101C06D931F
:10F7200041505040E0F70895CF92DF92EF92FF9260
:10F730000F931F93CF93DF932091CC0128602093E8
:10F74000CC01C0E20FEF1FE0D5E3FF24F394411595
:10F750005105C1F1262F2F713C2F321B232F30E092
:10F760004217530708F49A01D22EF801E21BF30B5B
:10F77000E617F70710F40E94397CE091CF01E7FD0E
:10F78000FCCFC82EDB01B05FFC01E090CF01E7FCAD
:10F79000FCCFE190ED92EE2EEC18ED14B0F3109248
:10F7A000C2017093C1016093C001D093CA01E8ED1A
:10F7B000E4BFF092CB01820F931F620F731F421BB5
:10F7C000530BC5CF8091CC01877F8093CC01DF9113
:10F7D000CF911F910F91FF90EF90DF90CF90089500
:10F7E000E0ECF1E0A785A7FDFDCFA485A860A48784
:10F7F0006050704F0C943E7C03D08081992708950F
:10F80000E0ECF1E0378537FDFDCF34853860348793
:10F81000FC01E050F04F08950E94007C80819181AE
:10F820000895262FE0ECF1E0378537FDFDCF3485D4
:10F83000377F3487378531FF09C036E3328738EDAB
:10F8400034BF31E03387378537FDFDCF33E332876F
:10F85000808391831282248325E3228728ED31E07F
:10F8600024BF3387019608950E94117C272F0C94A2
:10F87000127C81E090E0F8940C94477CFB01DC0161
:10F8800002C001900D9241505040D8F70895F8946D
:10F89000FFCFBE34C933C933C933C933C933C933C0
:10F8A000C933C933C933C933C933C933C933C93378
:10F8B000C933C933C933C933C933C933C933C93368
:10F8C000C933C933C933C933C933C933C933CB3356
:10F8D000E5332034413445344F34523455345834B0
:10F8E0005C347134C9337434C933C93385348734D3
:10F8F000C933C933C9338934C9339F34AB34D55480
:10F900005E55AC55CB55DB555E55AC55EC55455663
:10F91000F1562F576D577C578757A457C457E05758
:10F92000F657035817582858375846585A586758A2
:10F930007458B058C158CE58DB58EA58F75809598E
:10F94000245931594D598859A059B559C959E359C4
:10F95000FD59175A285A3D5A485A5A5A6C5A7E5AD3
:10F96000905AAF5ACE5ADB5AF65A135B3B5B4C5B4C
:10F97000865BA25BBE5BD65BEE5B0B5C205C325CA5
:10F98000465C5A5C6E5C875CA05CB75CCE5CE15CFC
:10F99000F45C075DB65FC65FC65FC65FC65FC65FE5
:10F9A000EA60F56026615C61A761EC610162086252
:10F9B000116218621B621D622F6238624762455DE8
:10F9C000585D5F5D665D765D885D985DA85DBA5D3A
:10F9D000C35DD75DE85DF65D045E4A5D4A5D125E1B
:10F9E000255E4A5D4A5D335E4A5D445E545E4A5D13
:10F9F000645E745E845E965EA65EB65EC75ED85E2A
:10FA0000E95E4A5DF75E0B5F1B5F235F335F435F19
:10FA1000575F4A5D6B5F187921795679217956795C
:0AFA200024793D79567979798079CF
:10FA2A0040404748494A4B4C40414042434445467E
:10FA3A0000E803F401FA007D0024F4127A093D007B
:00000001FF
